:1080000000000020BD870000758500008585000008
:108010008585000085850000858500008585000038
:108020008585000085850000858500008585000028
:108030008585000085850000858500008599000004
:108040008585000085850000858500008585000008
:1080500085850000858500008585000085850000F8
:1080600085850000858500008585000085850000E8
:1080700085850000858500008585000085850000D8
:1080800085850000858500008585000085850000C8
:1080900085850000858500008585000085850000B8
:1080A00085850000858500008585000085850000A8
:1080B0008585000085850000858500008585000098
:1080C0008585000085850000858500008585000088
:1080D0008585000085850000858500008585000078
:1080E0008585000085850000858500008585000068
:1080F00085850000858500008585000015950000B8
:108100008585000085850000858500008585000047
:108110008585000085850000858500008585000037
:108120008585000085850000858500008585000027
:1081300085850000858500000DE80000858500002C
:108140008585000085850000858500008585000007
:1081500085850000858500008585000085850000F7
:10816000BDED000085850000858500008585000047
:1081700085850000858500008585000085850000D7
:1081800085850000858500008585000085850000C7
:1081900085850000858500008585000085850000B7
:1081A00035DC0000A5DC00008585000015DD000041
:1081B0008585000085850000858500008585000097
:1081C0008585000085850000858500008585000087
:1081D0008585000085850000858500008585000077
:10840000FFFFFFFFFFFFFFFFFFFFFFFF7EFFFFFFFD
:1084100010B5054C237833B9044B13B10448AFF3BE
:1084200000800123237010BD2821FF1F00000000E1
:1084300054A201000C4B43B10C480D4910B5AFF3E9
:1084400000800C48036823B910BD0A48036833B99B
:108450007047094B002BF7D0BDE810401847064B7A
:10846000002BF5D0184700BF0000000054A2010007
:108470002C21FF1F2821FF1F0000000000280346B9
:10848000B8BF00F11F035B11012B2BD0022B15D0BD
:1084900003B170471D4A434203F01F03D2F8801115
:1084A00000F01F0058BF5842012303FA00F00143B7
:1084B000C2F880111368184310607047134A434292
:1084C00003F01F03D2F8881100F01F0058BF584274
:1084D000012303FA00F00143C2F88811936818439E
:1084E00090607047094A414201F01F0100F01F00EF
:1084F00058BF4842D2F8841103FA00F00143C2F891
:108500008411536818435060704700BF00E100E0D9
:1085100080281ADC40280FDC20281FDC434203F0AF
:108520001F0300F01F00124A58BF5842012303FAEC
:1085300000F0C2F88000704700F01F0001230C4AD1
:1085400003FA00F0C2F88800704700F01F00012312
:10855000074A03FA00F0C2F88C00704700F01F00D1
:108560000123034A03FA00F0C2F88400704700BFF9
:1085700000E100E0684620F007018D4601B401BC2F
:1085800085467047684620F007018D4601B4FFBE5E
:1085900001BC8546704700BF4FF0E020F0B5364B78
:1085A000364A374CC0F8084D41F244053549364F3C
:1085B0004CF220544DF628164FF4E970D481D68140
:1085C00041F23804108059511A59304E304831491F
:1085D00042F4D0521A515E5141F248042E4E1A59BB
:1085E00022F00F0242F002021A5141F204024FF04F
:1085F000240E9C5844F480349C501D6825F40025BA
:108600001D60856C3D408564C46C80253C40C4641D
:1086100081F801E03570985820F001009850A223AD
:108620000B70CB78032403F01F030020CB700A46A5
:108630000C71487193799807FCD5164A9379D9063D
:10864000FCD4144A937903F00C03082BFAD140238D
:10865000104953718B7903F00C03082BFAD10D4AA2
:1086600093795B06FCD522230A4913708B7903F0BA
:108670000C030C2BFAD1F0BD007004400020054023
:108680000080000000003301FFF8FFFE000013012E
:1086900000900440004006400050064080F31188DE
:1086A000704700BFF0B41A4D1A4C2B691A4E1B4A82
:1086B0001B481C4923F0807323F4E06341F2140744
:1086C00043F4E0632B610025E55104F582531C68F7
:1086D00044F004041C60336823F0784323F0010362
:1086E0003360137803F08C0343F050031370537816
:1086F00003F09C0343F040035370937803F0EC03C2
:108700009370857081F8145385F31188F0BC70471D
:10871000009004400070044000D0004000D00740AA
:1087200000E0074000E100E0E2B140EA010313F09D
:10873000030F07D1032A05D951F8043B40F8043B45
:10874000043AF1E7DB0707D4012A05D931F9023BE6
:1087500020F8023B023AE7E711F8013B00F8013B41
:10876000013AE1E7704700BF704700BF884201D07F
:1087700002B1D9E7704700BF10B50C4C24B913E023
:1087800070B9A3688BB10C34216860680029F7D0F8
:108790008142A268F7D0002AF5D0FFF7C5FFF2E7C3
:1087A000A268002AEFD0F8E710BD10BDECC30100AD
:1087B000704700BF704700BF704700BF10B5FFF79C
:1087C000F7FF1D4CFFF7E8FE2046002807D085463E
:1087D00081B04FF000006FEA0000009001B0174B2D
:1087E000174AD21A0AD0002113F0030012D1032A2B
:1087F00010D9043A43F8040B002AF5D1FFF7BCFF67
:10880000FFF7DAFF0F4900200FF0D6FA0E4B186081
:108810008047FEE713F0010007D1012A05D0023A94
:1088200023F8020B002ADFD1E8E7013A03F8011B25
:10883000002AD9D1E2E700BF000000202821FF1F55
:108840009486FF1F4421FF1F7838FF1F08B5FFF7EC
:10885000B5FF00BF70B40D4B00220726082501208C
:1088600002214FF4FA741E705D7158709A701A717B
:108870009A711A755A759A75DA75D9701C62986072
:108880001A619A61DA61D96070BC70475438FF1F71
:10889000304B314AF0B506219A65FA260A25082799
:1088A000C8244FF4967247F230505E61DD614FF498
:1088B0007A664FF4FA7583F8251083F8297005213C
:1088C0004FF4FA671C669A6401240022D8654FF4BD
:1088D0007A701E605E60DE639D601D635D631C6276
:1088E00083F8244083F82C40588540F2FF74D86404
:1088F0004FF4827E7826D96019619F619F634FF49F
:10890000C87583F8262083F8272083F8282083F869
:108910002D20A3F8402083F842205A6483F8542085
:10892000186547F6FF7083F8642083F82E2083F8DB
:10893000692083F86A20A3F86E10A3F86CE09E67A4
:10894000DD67A3F87040A3F87240A3F87400A3F8A1
:108950007600F0BDD037FF1FC0B85900F0B5534DB9
:108960005349544A41F238044FF480702B5943F470
:1089700000732B510860C8605369002043F008035E
:108980000825536104462E460A2156604FF47A7337
:1089900000BF013BFCD113699560DF0748BF01347C
:1089A0004FF47A7300BF013BFCD11369DB0758BF5A
:1089B00001300139E9D10A2C3D4C3C4B3E4EDFF8E9
:1089C00018E13E4F41F238024FF4E0652560E56062
:1089D0009C5818BF084644F4806439499C504FF4B1
:1089E00081754FF480740D65CC60756925F4801530
:1089F00075610E6D334D26F020060E650E6D46F046
:108A000002060E650E6D26F001060E65995841F4BA
:108A100000619950CEF83C40CEF840409E582A491B
:108A200046F480569E506E6946F040066E612E6890
:108A300026F040062E60BC619F58244E244D47F41A
:108A400000579F504A69234F42F004024A614A6925
:108A500042F080724A61B460346674660C68B7F89C
:108A6000722041F22C0624F004044FF080770C6051
:108A70008F60995941F48051995195F8213043F014
:108A8000800385F8213095F8213008BF0A38C2F3F9
:108A9000032143F04003D2B285F8213008BFB0FA79
:108AA00080F069702A7008BF4009F0BD0070044072
:108AB0000090044000F00F4040F00F4000C0044020
:108AC00000A00440C0F00F4000F10F4000D004406F
:108AD00000C00C40D037FF1F00B00440044B054AD3
:108AE000B3F87230C3F30321DBB2517013707047D7
:108AF000D037FF1F00C00C402DE9F04F974CDFF836
:108B00007CC2974EDFF878E29648DFF87882964B81
:108B10009649974F41F23C0541F23009625942F0C3
:108B20000062625154F8092042F0006244F80920C2
:108B30000022CCF824204FF00D0ACCF82C204FF066
:108B40001009F2614FF0040CCEF80420012604F560
:108B5000825EC0F808A0C8F808A0C0F80C90C8F859
:108B60000C90C0F820C0C8F820C04262C8F8242089
:108B70000660C8F80060DEF8009049F00209CEF8FF
:108B8000009054F805A003F5845941F2840E4AF090
:108B9000020A4FF0B60B44F805A00A7141F28C05A9
:108BA00081F804B041F29004C9F8007041F2940ACF
:108BB00041F2980923F80E606FF0030B41F2880E22
:108BC00043F805B00126185141F29E0523F80A200A
:108BD00041F2960443F8092041F2860041F29C09D3
:108BE00043F80E6003F5855E23F805C0614E23F857
:108BF00004C041F2A4051A5241F2AC0423F8092042
:108C000041F2B0004FF0A8094A7141F2B40A81F86C
:108C10000590CEF8006041F2B80941F2A80E564E18
:108C20005A531A5141F2BE051E5002206FF007063A
:108C300023F80A0041F2B60443F8096043F80E0035
:108C400048F6040E23F805E041F2A60948F20405AF
:108C50001D5341F2BC0E40F2011423F8094040F2CA
:108C6000224923F80E90D3F80CE0434E03F58659C1
:108C700067444EF0200E4FF0B80AC3F80CE00836F7
:108C80008A7141F2C40E81F806A0C9F8007041F261
:108C9000CC0734464FF0010623F80E6041F2D009AC
:108CA00043F807B041F2D40E41F2D80743F80980E7
:108CB00041F2C80A23F80E2041F2DE09DA5141F2EE
:108CC000D60841F2C60E41F2DC0701264FF0A90B8F
:108CD00043F80A6023F809C003F5875623F808C053
:108CE00041F2E40A23F80E2041F2EC09DA5341F292
:108CF000F008CA7181F807B001F51A2141F2F40CAD
:108D000041F2F80E41F2E8071031316041F2FE0BFA
:108D100023F80A2041F2F60643F8092041F2E60161
:108D200043F8084041F2FC0A6FF0070423F80C00F6
:108D300048F6044943F80E4040F22262D85140F20E
:108D4000011023F80B909D53585223F80A20DA683B
:108D500042F08002DA6062B6BDE8F08F0070044035
:108D600000A0044000B0034000800040001002401A
:108D70000800FF1F10B003406C21FF1F00B004402B
:108D800000C0044000B00B400249034A01230B60BD
:108D90001360704700B0034000B00B40704700BF45
:108DA000704700BF704700BF704700BF704700BFEB
:108DB000704700BF704700BF704700BF704700BFDB
:108DC00009490A4B4A6922F480124A611A6D22F05D
:108DD00020021A651A6D42F002021A651A6D42F0FD
:108DE00001021A65704700BF40F00F4000A0044028
:108DF00009490A4B4A6922F480124A611A6D22F02D
:108E000020021A651A6D42F002021A651A6D22F0EC
:108E100001021A65704700BF40F00F4000A00440F7
:108E2000094B0A4A596941F480115961116D21F0C9
:108E300002011165116D41F0200111651A6822F4DB
:108E400080121A60704700BF40F00F4000A004403D
:108E5000024B1869C0F30050704700BF40F00F404C
:108E60000020704701280ED008D3022804D1084BF7
:108E70001869C0F30050704700207047054B18690F
:108E8000C0F3C0307047034B1869C0F3004070470F
:108E900040F00F4080F00F40704700BF704700BFA8
:108EA0000020704705281CD8DFE800F0070B0F13DF
:108EB00017030D4B588880B270470B4B988980B2CE
:108EC0007047094B588980B27047074B188980B2A8
:108ED0007047054B188880B27047034BD88980B221
:108EE00070470020704700BF6C21FF1F03281BD86C
:108EF000DFE800F0140E08020C4A0D4B927A33F8AA
:108F000012007047094A0A4B527A33F81200704730
:108F1000064A074B127A33F812007047054A044B91
:108F2000127C33F812007047002070470800FF1FC2
:108F30007C38FF1F6C21FF1F032808D8DFE800F0F2
:108F4000140E08020B4A0C4B927A23F81210704749
:108F5000084A094B527A23F812107047054A064B0B
:108F6000127A23F812107047044A034B127C23F83C
:108F7000121070470800FF1F7C38FF1F6C21FF1F75
:108F80000E490B690A6910B50C699209C3F30023F5
:108F900002F00202E408134304F004041C4306D068
:108FA000072C04D0202000F033FF204610BD0128FC
:108FB000F8D1202000F024FFF7E700BF80F00F4039
:108FC00038B50D4C0D4DB4F87410687AFFF7B4FF46
:108FD000B4F87610A87AFFF7AFFFB4F87010287ACB
:108FE000FFF7AAFFB4F87230054AC3F30321DBB2DE
:108FF0005170137038BD00BFD037FF1F0800FF1F2E
:1090000000C00C40024B4FF480425A60704700BFD2
:1090100000F00F40024B4FF480429A60704700BF4F
:1090200000F00F40014B04225A60704700F10F40DE
:10903000014B04229A60704700F10F40024B186800
:10904000C0F38000704700BF00F10F40704700BFC1
:10905000704700BF704700BF704700BF024B4FF41E
:1090600080625A60704700BF40F00F40024B4FF4DF
:1090700080629A60704700BF40F00F40024B4FF093
:1090800080729A60704700BF00F10F40024B4FF0B2
:1090900080725A60704700BF00F10F40034B18699F
:1090A00080F00070C0F34060704700BF00F10F40D7
:1090B00070B5254A254B2648264C41F2380641F228
:1090C0003C01955945F400759551555845F4805526
:1090D0005550555825F4802555505A6C42F400726D
:1090E0005A641A6C42F400721A64DA6B42F4007229
:1090F000DA639A6B42F480729A634369012243F403
:10910000804343612260236843F0004343F440639B
:109110002360FFF777FF4FF06053E360E36843F0AD
:109120002003E360E36843F48033E360E36A43F0E1
:109130008053E362236823F001032360236823F054
:109140000063236070BD00BF0070044000900440C5
:1091500000F00F4000C00240F0B42249224A234CE4
:10916000234B244E244D41F23807C85940F4806007
:10917000C85141F23C000F5847F400570F500F58A8
:1091800027F480270F50516C41F400715164116C29
:1091900041F400711164D16A41F40071D162916AA5
:1091A00041F4807191626269012142F480626261DE
:1091B00019601A6842F0004242F440624FF4806144
:1091C0001A606160DE601D61DA6A42F08052DA6224
:1091D0001A6822F001021A601A6822F000621A600E
:1091E000F0BC70470070044000A0044040F00F4005
:1091F00000D002400000513E0000F13E70B50C4628
:1092000016460546002833D001281ED1FFF720FF5F
:109210001B4BEEB144F000645C63DA6AD200FCD50B
:10922000DA6A42F08052DA62DA6A12F0F00FFBD0AA
:109230009C6B1A6842F44062E4B21A60E5B1012DF9
:1092400001D1FFF703FF204670BD0E4B002EE1D188
:1092500044F000445C63DA6AC2F30332032AFAD8AA
:10926000DA6A12F0F00FFBD09C6BE4B2204670BDBE
:10927000FFF7D0FE034BCCE7FFF7C4FE204670BDDE
:1092800000D0024000C00240012870B505460C46DF
:1092900016463AD035D3022820D1FFF7DDFE214B08
:1092A000FEB144F000645C63DA6AD200FCD5DA6A8D
:1092B00042F08052DA62DA6A12F0F00FFBD09C6B57
:1092C0001A68012D42F44062A4B21A6025D020D35E
:1092D000022D01D1FFF7BEFE204670BD124B002EBD
:1092E000DFD144F000445C63DA6AC2F30332032A3C
:1092F000FAD8DA6A12F0F00FFBD09C6BA4B22046C9
:1093000070BDFFF787FE084BCAE7FFF7A1FE054BCC
:10931000C6E7FFF777FE204670BDFFF797FE2046B1
:1093200070BD00BF00D0024000C00240134AA8B187
:109330004FF000635363D36ADB00FCD5D36A0F4957
:1093400043F08053D362CB6A13F0F00FFBD0886BED
:109350000B6843F4406380B20B6070474FF00043EA
:109360005363D36AC3F30333032BFAD8034AD36A94
:1093700013F0F00FFBD0906B80B2704700D002402A
:10938000344B9842F0B438D0334B98423DD0334BF5
:1093900098424FD0324B984254D0324B984219D019
:1093A000072A96BF304B4FF4165353F8223000294A
:1093B000B8BF0F310911B1FBF3F1C1F30423C9B2F6
:1093C00003704170C37843F02C03C370F0BC2F20AE
:1093D000FFF754B8254F264C41F228064FF440754C
:1093E000BB5943F48063BB51256600236566C37097
:1093F00083708371C3724371D2E71C4D41F2340410
:109400002B5943F480632B51CAE7A3F5103341F283
:10941000340641F238079C59154D44F400649C51C0
:10942000DC594FF4407644F40054DC512E600023A4
:109430006E60DCE70D4D41F234042B5943F4805348
:109440002B51ADE7094D41F234042B5943F400533D
:109450002B51A5E700A0064000B0064000C0064022
:1094600000D0064000A00E40D483010000700440EC
:1094700000D00440024602490248FFF781BF00BF06
:1094800000D8B80500B006400A4A13685168013395
:10949000202B08BF00238B420AD010B41168064C61
:1094A000114408721360E37843F08003E37010BC4A
:1094B000704700BF8021FF1F00B006400B4B996A28
:1094C000DA6A91420FD09A6A511C1A44996292F852
:1094D00030109A6A0170202A01D0012070470022C2
:1094E0009A62012070470020704700BF8021FF1F53
:1094F000044A137803F0FF0013B100231370012016
:10950000704700BF8838FF1F014B1865704700BFC8
:109510008021FF1F684620F007018D4631B52A499A
:109520000C79E4B2A00615D5284AD36A906A0133B3
:10953000202B08BF0023834206D0D06ACD791118B2
:10954000E8B281F83000D3622149224B052008603F
:10955000126D1A60620625D4230603D4BDE831409B
:10956000854670471B4B1D68002DF7D1174C2268AC
:1095700063689A421ED0FFF755FD6368124A591C72
:10958000234461601B7ADBB2D37163680E4A202BDF
:1095900008BF6560D37843F04003D370BDE8314025
:1095A00085467047FFF744FD074AD37803F0BF03B1
:1095B000D370D1E7044AD37803F07F03D370BDE8BA
:1095C00031408546704700BF00B006408021FF1F34
:1095D0008C38FF1F9038FF1FF8B52D4C2D4F617050
:1095E000002241F23C062270BD592B4B45F000751C
:1095F000BD515D6D45F004055D651D6825F01805DC
:109600001D605D6D25F001055D65D3F8845001385E
:1096100045F0C005C3F88450DA645A609860D3F806
:10962000802042F00102C3F88020D3F8802049B3A3
:1096300022F02002C3F88020D3F8802022F010020C
:10964000C3F88020144A134D516D144B144E41F051
:1096500001015165116841F2380041F008011160C3
:109660002A584FF4C06142F4806240272A501960A2
:1096700058205960C3F8A0709E61FEF7FFFE0123D9
:109680002370F8BD42F02002C3F88020DAE700BF63
:10969000D421FF1F007004400090034000A004404C
:1096A00000010900024A034B11801860704700BF97
:1096B0009838FF1F9438FF1F014B1880704700BF78
:1096C0009838FF1F014B1860704700BF9438FF1F88
:1096D000084B187820B1084B586880B2C0EB0040A6
:1096E000064B074A1B881268B0FBF2F000FB03F040
:1096F00080B27047D421FF1F009003409838FF1FAD
:109700009438FF1F034B187808B1034B586880B298
:10971000704700BFD421FF1F00900340014B5888C1
:10972000704700BFD421FF1F024B0022D8645A604B
:10973000DA64704700900340014B1879704700BF0E
:10974000D421FF1F014B00221A717047D421FF1F43
:10975000014B1870704700BF2400FF1F014B1878A1
:10976000704700BF2400FF1F014B9860704700BF87
:10977000D421FF1F014B9868704700BFD421FF1F01
:10978000014B187B704700BFD421FF1F024B012201
:1097900018611A7358697047D421FF1F38B50C4CF3
:1097A00025690122290C0220FFF76EFDA9B20122D2
:1097B0000220FFF769FD074B054659880122022068
:1097C000FFF762FD002340EA05402373606138BD66
:1097D000D421FF1F2400FF1F704700BF014B1883D7
:1097E000704700BFD421FF1FF0B4114D114B41F25F
:1097F000380420272A59802642F400624FF48071F1
:109800002A51C3F8A070C3F8A060C3F8A01030B903
:1098100059615920D961F0BC1962FEF72FBE064A82
:109820005A615920DA61F0BC1A62FEF727BE00BF08
:109830000070044000B0044000010B0008B5FFF7C1
:109840009FFB0138C0B205289ABF024B33F91000C4
:10985000002008BDF483010038B500F13B03762BEE
:109860000B4C08D80020208042F6AA22094906F0B5
:109870007BF8208038BD2388074D01FB02F180036F
:1098800095FBF1F190FBF1F0181A00B22080EBE7A4
:10989000F421FF1F56D5FFFFE0930400014BB3F9FD
:1098A00000007047F421FF1F884210D0204B002297
:1098B00001381A80052808D8DFE800F03321032793
:1098C0002D1A012932D0022916D0002070478B1E94
:1098D000042BFAD801A252F823F000BFFF98000031
:1098E000C39800000B99000017990000F198000040
:1098F00002291BD00429E8D14FF0FF30704703291B
:1099000014D00629F8D00020704706290ED005296A
:10991000F2D000207047042908D00129ECD00020A3
:109920007047052902D00329CFD1E5E70120704710
:10993000F421FF1F014B5860704700BFF421FF1F47
:10994000014B5868704700BFF421FF1FFEF7AABE05
:10995000044B0548002207211A6058609A6019607C
:10996000704700BF10E000E000770100014B0022CB
:109970001A60704710E000E0014B1868704700BFA4
:10998000FC21FF1F684620F007018D460E490F4A53
:109990000B6801B5106801330B6020B11368013BFF
:1099A000136013685BB10A4B1A6812B11A68013A66
:1099B0001A6009F079FFBDE8014085467047054B04
:1099C00001221A70EFE700BFFC21FF1F8C38FF1F38
:1099D0009038FF1F8838FF1F044B00221A619A61DC
:1099E0001A629A621A639A63704700BF008003404C
:1099F0005D4AF8B541F23C0441F2380115595B4B20
:109A000045F080751551155945F480051551545888
:109A100044F400645450545844F4805454505A6DE3
:109A200042F004025A65002879D1D3F884205049C5
:109A3000504C42F0C002C3F884205A6D40F6C31562
:109A400042F061025A659D60D864D3F88C2042F0E0
:109A50008002C3F88C209A6D42F002029A659A6DDA
:109A600042F080029A650A883F20024018665C66D0
:109A70009A66FFF7B1FF3D4B3F49DA683F48404ED9
:109A8000404C42F00802DA605A6942F008025A611A
:109A9000DA6942F00802DA615A6A42F008025A6250
:109AA000DA6A42F00802DA625A6B2A2742F00802A8
:109AB0004FF400755A631F67C3F89850DA6E42F08E
:109AC0004002DA665A6D42F002025A651D6840F2A1
:109AD0000442002745F008051D6042608260C260B4
:109AE000026132617261CF600A6842F40A6242F038
:109AF000010240F6C3100A6048601F661A683E20E3
:109B000042F040021A60FEF7B9FC302384F83E337D
:109B10004820FEF7B3FC202384F84833F8BD5A6D83
:109B20001349144842F061026FF49C6440F2E1452D
:109B30005A659D60DC649A6D42F002029A659A6DE6
:109B40003F2442F080029A651C665866088840F2FD
:109B500071226FF41C712040986619619A61196234
:109B60009A6219639A6386E700700440008003409C
:109B70001600FF1F737373000060034000B00440C1
:109B800000C0044000E100E0014B3F221A6670472C
:109B90000080034058B1064B6FF41C7140F27122F3
:109BA00019619A6119629A6219639A63704713E79F
:109BB00000800340F0B444F2A8324DF6F00510FBEB
:109BC00002F310FB25F5EC1A2B445A1082B04FEA31
:109BD000640143D40029C0F2838002F51C52103284
:109BE000521A44BF02F57F3202F2FF32002CBCBF92
:109BF00004F57F3404F2FF349214181EB8BF00F548
:109C00007F3002F2E24292B2B8BF00F2FF3002EBC4
:109C1000A444A2EBA040A4B280B20225624B197802
:109C2000012907D16149624F0A8000264C80888053
:109C30003D701E705F4963085208400857425E42FB
:109C400045424FF400748A610F618B620E62886333
:109C50000D63C1F8984002B0F0BC704700291DDBCD
:109C6000002D5EDDC5F51C5110318A1844BF02F588
:109C70007F3202F2FF329214002BB8BF03F57F331C
:109C800002F2E24292B2B8BF03F2FF33A2EBA34367
:109C900098B200EB65439CB20325BFE702F51C5266
:109CA0001032521A44BF02F57F3202F2FF32002C0A
:109CB000BCBF04F57F3404F2FF349214002BB8BF0C
:109CC00003F57F3302F2E24292B2B8BF03F2FF33F0
:109CD00002EBA444A2EBA343A4B298B205259DE7EE
:109CE000002D41DD05F51C521032521A231E4FEA99
:109CF000A242B8BF03F57F3302F2E242B8BF03F2DB
:109D0000FF3392B2281EB8BF00F5FF3002EBA34329
:109D10009CB2B8BF00F2FF10A4EB604080B20125F6
:109D20007CE705F51C521032521A44BF02F57F320F
:109D300002F2FF329214231EB8BF03F57F3302F202
:109D4000E242B8BF03F2FF3392B2281EB8BF00F55B
:109D5000FF3002EBA3439CB2B8BF00F2FF10A4EBAC
:109D6000604080B2042559E7C5F51C5110310A4402
:109D7000002B4FEAA242B8BF03F57F3302F2E24262
:109D8000B8BF03F2FF3392B2002DB8BF05F5FF351F
:109D9000A2EBA343B8BF05F2FF1598B200EB6543F1
:109DA0009CB206253AE700BF0022FF1F9C38FF1F28
:109DB0002E00FF1F00800340014B01221A707047E4
:109DC0000022FF1F014B33F8100070479C38FF1F23
:109DD000064A074B1088518892880844104483FB38
:109DE0000023A3EBE07080B2704700BF9C38FF1FD8
:109DF00056555555014B1878704700BF2E00FF1F70
:109E0000024A136818431060704700BF0422FF1F06
:109E1000024A136823EA0000106070470422FF1F03
:109E2000044A136819B923EA000010607047184308
:109E3000106070470422FF1F034B1B68034214BFCE
:109E400001200020704700BF0422FF1F024A136850
:109E500023F06D03136070470422FF1F034B186843
:109E60001A6822F06D021A60704700BF0422FF1FBB
:109E7000044B18681A6822F06D0200F06F001A6037
:109E8000704700BF0422FF1F2DE9F041174F184D06
:109E9000184E04463878FFF705F880463878FFF703
:109EA00025F8294647F6FF72A8EB000005F05CFD97
:109EB00007B23078FEF7F6FF80463078FFF716F8E5
:109EC0002946A8EB000047F6FF7205F04DFD06B2EB
:109ED000B819294647F6FF72404205F045FD278034
:109EE000A08066802046BDE8F08100BF1100FF1F02
:109EF0000180FFFF1200FF1F38B5084C2078FEF7E5
:109F0000D1FF05462078FEF7F1FF47F6FF72281AC9
:109F10000021BDE8384005F027BD00BF1000FF1F3D
:109F2000002210B5032104461046FFF767F900220E
:109F3000C4F307211046FFF761F90022E1B2104691
:109F4000FFF75CF9002108460122BDE81040FFF749
:109F500055B900BF38B5012204460D460020062140
:109F6000FFF74CF9002210460521FFF747F90021C1
:109F700001220846FFF742F98207F3D50022104676
:109F80000221FFF73BF900221046C4F30721FFF737
:109F900035F90022E1B21046FFF730F929460122D7
:109FA0000020FFF72BF9002210460521FFF726F9C4
:109FB000002108460122FFF721F9C307F3D438BD79
:109FC000F8B51646002204460D4610460321FFF759
:109FD00015F90022C4F307211046FFF70FF90022FC
:109FE000E1B21046FFF70AF97EB1013D771E002469
:109FF0003A1B0021B2FA82F208465209FFF7FEF836
:10A000000134A64205F8010FF2D1F8BD2DE9F04167
:10A0100004460E461746062101220020FFF7EEF8FF
:10A02000002210460521FFF7E9F800210846012229
:10A03000FFF7E4F88107F3D5002210460221FFF76D
:10A04000DDF800221046C4F30721FFF7D7F80022FD
:10A050001046E1B2FFF7D2F8002F4AD0013E0025AA
:10A0600007F1FF380AE0A8EB0502B2FA82F25209C2
:10A070000020FFF7C3F80135AF423AD0013414F0A5
:10A080003F0016F8011FEED10122FFF7B7F8A845EF
:10A09000F1D9002210460521FFF7B0F8002108464B
:10A0A0000122FFF7ABF810F00100F2D101220621E6
:10A0B000FFF7A4F8002210460521FFF79FF80021C2
:10A0C00001220846FFF79AF88207F3D500221046CE
:10A0D0000221FFF793F800221046C4F30721FFF78F
:10A0E0008DF800221046E1B20135FFF787F8AF4244
:10A0F000C4D1002210460521FFF780F80021084650
:10A100000122FFF77BF8C307F3D4BDE8F08100BF5D
:10A1100038B50D46C0EBC00404F500600978FFF7C0
:10A1200019FF697804F60100FFF714FFA97804F617
:10A130000200FFF70FFF297904F60300FFF70AFF7B
:10A14000697904F60400FFF705FFA97904F6050014
:10A15000FFF700FFE97904F60600BDE83840FFF795
:10A16000F9BE00BF002238B50C46C0EBC005032184
:10A170001046FFF743F805F500650022C5F30721F7
:10A180001046FFF73BF80022E9B21046FFF736F819
:10A19000002211461046FFF731F8002211462070C8
:10A1A0001046FFF72BF80022114660701046FFF7AB
:10A1B00025F800221146A0701046FFF71FF8002274
:10A1C000114620711046FFF719F800221146607100
:10A1D0001046FFF713F80021A07101220846FFF78F
:10A1E0000DF8E07138BD00BFF0B5002283B00D4618
:10A1F000C0EBC00403211046FFF700F804F500642B
:10A200000022C4F307211046FEF7F8FF0022E1B256
:10A210001046FEF7F3FF002211461046FEF7EEFF50
:10A220000022114606461046FEF7E8FF00221146BE
:10A2300004461046FEF7E2FF00221146074610468C
:10A24000FEF7DCFF002211468DF804001046FEF7F1
:10A25000D5FF002211468DF805001046FEF7CEFF0F
:10A2600000218DF8060001220846FEF7C7FF8DF891
:10A2700000608DF80140BDF800202B888DF80700A4
:10A280009A4202D0002003B0F0BDAB78BB42F9D1B6
:10A290006B680198C01AB0FA80F04009F3E700BF7C
:10A2A00038B54FF40065012206210020FEF7A6FF15
:10A2B000002210460521FEF7A1FF002101220846D9
:10A2C000FEF79CFF8207F3D5002210460221FEF71D
:10A2D00095FF00221046C5F30721FEF78FFF0022ED
:10A2E0001046E9B2FEF78AFF0024A4F13F020021E4
:10A2F000B2FA82F2084652090134FEF77FFF402C81
:10A30000F3D1002210460521FEF778FF0021084610
:10A310000122FEF773FFC307F3D44035B5F5804F34
:10A32000C1D138BD70B5054640F2FF700C461646E7
:10A33000FFF7F6FD902821D0002140F2FF70FFF7D3
:10A3400009FEFFF7ADFF242229460020FFF75EFE3D
:10A35000214640208022FFF759FE902140F2FF70F5
:10A36000FFF7F8FD294624220020FFF729FE2146A9
:10A3700080224020BDE87040FFF722BE002EDBD1D6
:10A38000F0E700BFF0B51D4C1D4FA569E369DFF88C
:10A3900074E003FB05F387FB0327421ADE17002A4C
:10A3A000C6EB6736B8BF5242B242B8BF44F620632C
:10A3B000DEF80060B8BF5343114A334482FB0362A6
:10A3C000DF175213A2EB070C44F6206606FB1C3382
:10A3D000CEF8003085B1884208DB0EDD2168BA1A5C
:10A3E000494210448842B8BF0846F0BD2168604425
:10A3F0008842A8BF0846F0BD0846F0BDD037FF1F11
:10A40000AD8BDB680822FF1F2DE9F84F5C4D95F8F6
:10A4100025E02E68BEF1060F0746884691461C4689
:10A4200002D0BEF1000F73D195F82900D7F800B023
:10A4300040080DF04FF85946824658460DF09EF8F8
:10A4400050490DF09BF8014650460DF097F88246B2
:10A45000A869C0EB0010C0000DF03CF80146504662
:10A460000DF040F90DF0DEFAA4EB09024C45B8BF3F
:10A470007642002AB8BF524290424FEAE27371EB33
:10A4800003034FF48040A8BF0026FFF7D5FC012846
:10A4900058D030460DF01EF83C68804601462046F4
:10A4A0000DF00AFAC8B1002E38D1EB69A86903EBA8
:10A4B000830203EB420300FB03F00DF00BF832497B
:10A4C0000DF010F9014620460CF050FF04463860AC
:10A4D00020460DF019FABDE8F88F414620460DF0F0
:10A4E00009FA0028F4D00EB3AB69E86900FB03F069
:10A4F0000CF0F0FF25490DF0F5F8014620460CF070
:10A5000033FF0446386020460DF0FEF9BDE8F88FB1
:10A51000BEF1070F20D000200021A5E7AB69E86954
:10A5200000FB03F00CF0D6FF1849C9E7EB69A869F6
:10A5300003EB830203EB420300FB03F00CF0CAFFC2
:10A540001149D8E740460CF0C5FF04463860204664
:10A550000DF0DAF9BDE8F88F016808460DF00EF845
:10A560000B490DF0BFF80DF05DFAEB6BAA698E4652
:10A57000A3FB000103FB0E11D3170DF0EBF973E7FA
:10A58000D037FF1F0000C0400050434800409C46A9
:10A590000000F042014B1878704700BF0C22FF1FEB
:10A5A000014B1870704700BF0C22FF1F38B50E4DCD
:10A5B000AB6C1361401A00231446536110600B49C1
:10A5C0004FF6FF7205F0D0F92369206003FB00F01D
:10A5D00000282A68B8BFFF300012A0615142BDE8D0
:10A5E000384005F0C1B900BFD037FF1F0100FFFFA1
:10A5F0002DE9F84F394FD7F84C803E6D5661C2F8BF
:10A600001080144697F82520054699464AB9B8F1B6
:10A610000003B8BF0733002EB8BF03364FEAE30884
:10A62000B610681A20602E494FF6FF7205F09CF9AB
:10A63000D4E902AB616920601AEB000A4BEBE07BC6
:10A64000C4E902AB71B34FEA094292FBF6F2514200
:10A65000504605F089F92368824603FB08F34FEA68
:10A66000E07B002BC4E902AB80FB06ABB8BFFF3335
:10A67000BAF1000F4FEA23207BF100031EDB4FEA03
:10A680001A4343EA0B431844A06197F82530082B7E
:10A690000ED1002D08DDB86BBD6F000290FBF5F008
:10A6A000BDE8F88F0A46D3E710D12846BDE8F88FF9
:10A6B0004A465142BDE8F84F05F056B94FF6FF72D1
:10A6C00000231AEB020A4BEB030BD8E7B86BBD6F04
:10A6D000000290FBF5F04042BDE8F88FD037FF1F35
:10A6E0000100FFFF2DE9F04114460E461A4659427B
:10A6F00005F03AF9244A136B516B2361002BB8BF64
:10A700000733DD10D4E90223801B00298846B8BF37
:10A7100001F10308161843EBE077616120604FEA0E
:10A72000A808C4E9026739B3184A92FBF8F251420B
:10A73000304605F019F9236803FB05F3002B0646A4
:10A740004FEAE07780FB0801B8BF03F2FF3300282F
:10A7500071F10002C4E902674FEAA3230EDB000C8B
:10A7600040EA01401844A06140F6C312084905F0D0
:10A77000FBF800B2BDE8F0810A46D9E74FF6FF7654
:10A78000002780197941EAE7D037FF1F0000C3098D
:10A790003DF6FFFFF8B514460D461A46594205F03E
:10A7A000E3F8D4E902231F4E00B2451B716B306BF6
:10A7B0002061561943EBE57725606161C4E90267C2
:10A7C00039B3194A92FBF1F25142304605F0CCF808
:10A7D0002269236803FB02F36269002B06464FEAF5
:10A7E000E07780FB0201B8BFFF33002871F100025F
:10A7F000C4E902674FEA23230DDB000C40EA014065
:10A800001844A06147F6FF72084905F0ADF800B2A0
:10A81000F8BD0A46D9E74FF6FF760027801979413F
:10A82000EBE700BFD037FF1F0000FF7F0180FFFF75
:10A8300082B02DE9F04F1DB21C1487B005EBD57620
:10A8400004EBD475B94CDDF864E0139F01977610E2
:10A85000A680159E05966D10169EE5800296179EA1
:10A8600004968146189E606811930EEBDE7703967E
:10A87000DFF8CC82149D8A46934605F0C5F8019B0B
:10A880001E6898F82530A06006EBD676063B7F1050
:10A8900046F34F06032B00F22181DFE813F0B500E9
:10A8A000F9005E0004000020FEF7C8FF98F8282099
:10A8B000012A834600F070815846FFF73BF8029B5F
:10A8C0001B68029318460DF01FF8D8F8142080EA90
:10A8D000E07EAEEBE07E964580F20C8198F8293060
:10A8E000D8F820609249934A0EFB03F006FB00F073
:10A8F000000381FB0013C117C1EB6311236A1944E4
:10A9000082FB01325211CB17D61A642000FB1610BD
:10A91000206200210298049303920CF0EBFF0028C0
:10A9200000F01382039A049BE18BD8F838609B1ADD
:10A930000B449BB203F58041E38309B23302F60175
:10A94000D8F8782093FBF2F3019A7B481360D8F88B
:10A95000783096FBF3F636B26BE0029BD3F800B08A
:10A9600058460CF0D1FF98F829307149714A80EAB5
:10A97000E07EAEEBE07E03FB0EF0D8F8203003FB68
:10A9800000F0000381FB0013C117C1EB6311236AC0
:10A99000194482FB01325211CB17D01A4FF0640ECA
:10A9A0000EFB101E039000215846C4F820E00293CD
:10A9B00001920CF09FFF002800F0A980019A029BF1
:10A9C000E18B9B1A0B449BB203F58041E38309B2F0
:10A9D000594805F009F9C0F30F4328806B80012026
:10A9E000FEF72CFF98F82830012B00F0DB80FEF7F3
:10A9F000A1FFFEF76DFEA0F5FF407F3800B2FEF725
:10AA0000B3FE4FF0000B1CE00120FEF717FF98F893
:10AA10002E20012A834600F0CA8098F82820012AB7
:10AA20007ED05846FEF786FF0020FEF79DFE424886
:10AA3000594605F0D9F8C0F30F4328806B804FF0DA
:10AA4000000B3B464A46B5F900103046FFF7A2FE20
:10AA50003B46208252465846B5F90210FFF79AFE4F
:10AA6000237860827BBB238AA384344804F0F4FFFC
:10AA7000324805F01BF82A886B88A06252005B0000
:10AA80002A806B8007B0BDE8F04F02B0FFF792B8A4
:10AA9000FEF764FE012855D0FEF71AFE98F82C3018
:10AAA000A0F5FF407F38012B0FFA80F800F04781B6
:10AAB0000020FEF73FFF4046FEF756FE41461E4887
:10AAC000A4F81E80B5E7A18C21820022002300217A
:10AAD000C9E902236182CAE90223C6E700211648B8
:10AAE00005F082F84FF0000BC0F30F4328806B8015
:10AAF0005E46A6E75946104805F076F8C0F30F42C7
:10AB0000A4F81EB028806A804FF0000B99E75846E1
:10AB100000210CF0D1FE002857D1B4F91E1057E7E0
:10AB20000BF5FF437F330FFA83FB7AE70C22FF1FFD
:10AB3000F11976051F85EB511422FF1F1C22FF1F00
:10AB4000D037FF1F4FF48060FFF776F9012811D04E
:10AB50004FF40070FFF770F9012801D1049B4BB945
:10AB60004FF40060FFF768F90128B7D1019B1B681B
:10AB7000002BB3D098F82C30012B00F03C81C0F0B2
:10AB8000FE80022B40F02C816369032B3FF657AF08
:10AB9000DFE803F0A445242400F5FF437F330FFAD8
:10ABA00083FB89E600F5FF407F3000B21FE798F88D
:10ABB0002910D8F8202003984908FEF74DFEFEF72B
:10ABC0006DFE83440FFA8BFB27E7E38B039A1A444D
:10ABD00093B2A3F58041E38309B2F9E65846002613
:10ABE0002682668205F06CF8484605F069F8504602
:10ABF00005F066F80599626900230B600299022A44
:10AC00000B6000F0B4818020FFF7FAF80020FEF717
:10AC100091FEA069FEF7A8FDB4F918105FE7D4F81B
:10AC200018B098F829308BEAEB715B08C3EB03424C
:10AC3000A1EBEB71914280F29581D8F86010D8F8C1
:10AC40002020CF4E01FB03F3C2EBC23202FB03F321
:10AC5000B8F8662086FB0316B2F5007F4FEAE3736F
:10AC6000C3EBA64600F09481B2F5806F00F09081AE
:10AC7000B2F5006F00F0AC81E368D8F83820C14825
:10AC8000D8F878104FEAC21B9BFBF1FB03FB0BFBD0
:10AC9000A0FB0B3B0020FEF74DFEA069FEF764FD14
:10ACA000B4F91810B84804F09FFFB8F8663028804F
:10ACB000B3F5007FC0F30F404BF34F3B688000F0CB
:10ACC0007981B3F5806F00F0758198F8423013F008
:10ACD000020332D102221E466261B2E6E26842F20B
:10ACE00010739A4200F23081D8F83830A548D8F86D
:10ACF000781001324FEAC31B9BFBF1FB02FB0BFBFD
:10AD0000A0FB0B3B0020E260FEF714FE0020FEF7E4
:10AD10002BFD00219C4804F067FFB8F866302880BE
:10AD2000B3F5007FC0F30F404BF34F3B688000F05A
:10AD30003C81B3F5806F00F03881002681E618462B
:10AD4000FEF77CFDFEF7F6FDB5E6029800210CF05B
:10AD5000B3FD20B90646B4F91E100346F0E5E28BB8
:10AD6000D8F83800324492B2C0EB0063A2F58041BB
:10AD7000C0EB4060E28309B21B02C601E0E5E36874
:10AD800042F2107201339342E36000F2A180D8F8DE
:10AD900038207C48B8F86610D8F878604FEAC21BB3
:10ADA0009BFBF6FB03FB0BFBA0FB0B3BB1F5007F12
:10ADB0004BF34F3B00F08780B1F5806F00F083804C
:10ADC0000020FEF7B7FD0020FEF7CEFC00216E4804
:10ADD00004F00AFFC0F30F4328806B80002630E6A2
:10ADE0000021694804F000FF0026C0F30F432880CB
:10ADF0006B80B34625E618460393FEF7C1F801467B
:10AE00000290207FFEF750FD039B029A01901846A6
:10AE10002277FEF713FD98F82820012A034604BF85
:10AE200000F5FF437F3318460293FEF783FD019B35
:10AE3000002B029B76DB39D003F515435433B8F968
:10AE40003C1098F829205148520803FB01F393FB6A
:10AE5000F2F380FB03201844DB17C3EBE03080B231
:10AE6000FEF762FCFEF734FC00230FFA80F8584628
:10AE700023826382019304F023FF484604F020FFFD
:10AE8000504604F01DFF019B1846FEF761FC4FF48D
:10AE90000040FEF7B5FFA8F5FF437F3B0FFA83F8AC
:10AEA0004046FEF761FC41463748C2E50120FEF707
:10AEB000C5FC98F82830012B41D000F5FF437F33C3
:10AEC0000FFA83F8E7E7019A4FEA4B03136077E73D
:10AED00000231846E360FEF727FC98F82C302BBBC4
:10AEE00098F8423043F0010388F8423058464FF05A
:10AEF000000BA4F810B0A4F812B004F0E1FE48462C
:10AF000004F0DEFE504604F0DBFE059A00231360D9
:10AF1000029A58461360FEF71BFC4FF40040FEF700
:10AF20006FFF8EE503F5D5432A3388E7022BDDD189
:10AF300098F8423043F0020388F84230D6E700F533
:10AF4000FF437F3318B2B8E70020FEF7EDFB98F817
:10AF50004230012243F0020388F8423062614FF030
:10AF6000000B6EE5032363614FF0000B69E530468B
:10AF7000FEF7EEFB4FF40040FEF742FF46E600BF4F
:10AF8000851DD96F5917B7D11422FF1F018000808A
:10AF9000029B1B680293184600210CF0ABFC029B3D
:10AFA00060B1ABEB0606A66166E6019B0026C3F81E
:10AFB00000B046E5019BC3F800B086E618460021C4
:10AFC0000CF07AFC00283FF457AE5E44A66153E6CD
:10AFD000019B1B68002BE4DC3FF44EAEF5E700BF9D
:10AFE000024B00225A61DA609A6170470C22FF1FFF
:10AFF000014BB3F91E0070470C22FF1F08B5054B2B
:10B00000054918600422FEF7DBFF044B01221A7089
:10B0100008BD00BFCC3CFF1FD03CFF1F3822FF1FE4
:10B02000024A136801331360704700BFD03CFF1F12
:10B030002DE9F04B2D4B2E4D1E6ADA6D2D4C2E4F07
:10B0400080EAE07EAEEBE07E85FB0E314FEAEE73E8
:10B05000C3EB21130EFB03F085FB0013C017C0EBFD
:10B06000231306FB03F3D4E9020187FB037E02EB03
:10B070008207DB176268C3EBEE0310EB030B02F1F0
:10B0800001024FEA8707B7FBF6F6A5FB063641F14A
:10B09000000CB2EB561FC4E902BC626023DBD4F89B
:10B0A0001080DFF85890676959F8286000234FF442
:10B0B000C872584661460CF09DFC08F1010185FB01
:10B0C0000135CB17C3EB651500220023BE1BC4E975
:10B0D0000223642303FB15150644002349F82800C6
:10B0E000666125616360BDE8F08B00BFD037FF1F4C
:10B0F0001F85EB513822FF1F67666666D43CFF1F31
:10B10000014B5869704700BF3822FF1F014B186878
:10B11000704700BFD03CFF1F014B1860704700BF55
:10B12000D03CFF1F054B1B78012B00D07047044B10
:10B13000044918680422FEF769BF00BF3822FF1FC8
:10B14000CC3CFF1FD03CFF1F044B93F8643003B18D
:10B1500070474FF40030FEF75BBE00BFD037FF1FD3
:10B16000431E18B100BF13F1FF33FBD2704700BF7D
:10B1700041F238010E480F4A435830B443F480631B
:10B180000D4C43504FF48075A56453694FF48021F2
:10B190000B43536142F23413916000BF013BFCD179
:10B1A000044A536923F48023536130BC704700BFC5
:10B1B0000070044040F00F4000A00440F8B5384D46
:10B1C000384C394F00232B70FEF7DEFCFDF728FECC
:10B1D00041F2380135486658354B364A46F4006628
:10B1E0006650665846F4805666504FF48071416050
:10B1F0008160C160016139617961596941F01E0165
:10B200005961516941F030015161196821F0020121
:10B210001960196821F008011960116821F0100106
:10B220001160196841F004011960196841F01001BA
:10B230001960136843F02003136042F2341300BF17
:10B24000013BFCD141F2380116481B4C43581B4AC4
:10B2500043F4806343504FF48076A66453694FF4FF
:10B2600080210B43536142F23413916000BF013BD4
:10B27000FCD1124A536923F48023536142F2341300
:10B2800000BF013BFCD10A490C4A4B6923F004037F
:10B290004B615369012143F4802353612970F8BD48
:10B2A0005022FF1F0070044000C0044000B0044062
:10B2B00080F00F40C0F00F4000A0044040F00F406D
:10B2C000014B1878704700BF5022FF1F064B074AFA
:10B2D0001B691B0703D4936801339360704753685D
:10B2E00001335360704700BF40F00F405022FF1FF2
:10B2F000084909484B688A681A44A0FB020203EB1C
:10B30000830300205B0052094860B3FBF2F38860BE
:10B31000CB6070475022FF1F1F85EB51014BD8684F
:10B32000704700BF5022FF1F0023194640FA03F266
:10B3300012F0010F03F1010318BF01310F2BF5D1FA
:10B34000CB0754BF40F40040C0F30E00704700BF6D
:10B350000023194640FA03F212F0010F03F1010332
:10B3600018BF01310F2BF5D181EAD03000F0010078
:10B37000704700BF204B2149F0B500224FF48025D3
:10B380001024DFF87CE09D60074626461046202505
:10B390004FF0010C47FA02F3DB078E6040F25233A4
:10B3A0004CBFCEF80450CEF8085000BF013BFCD192
:10B3B0004C6040F2A91300BF013BFCD10B695B0755
:10B3C00003D50CFA02F3184380B240F2A91300BF70
:10B3D000013BFCD10132102ADCD10849084B8A60BC
:10B3E00020229A6040F2523300BF013BFCD1024B55
:10B3F0004FF480225A60F0BD40F00F4080F00F40C3
:10B40000C0F00F4038B5002485B22946234641FAE2
:10B4100003F212F0010F03F1010318BF01340F2BE7
:10B42000F5D1E30754BF45F40045C5F30E052846A2
:10B43000FFF7A0FF42F2341300BF013BFCD12846C6
:10B44000BDE83840FFF796BF0220FFF7DBBF00BF23
:10B450000320FFF7D7BF00BF0420FFF7D3BF00BF13
:10B4600070B520F48055ADB2002104460B4645F47A
:10B47000006040FA03F212F0010F03F1010318BF5C
:10B4800001310F2BF5D1C80745BF46F6FF752540A2
:10B4900045F4084545F400652846FFF76BFF6A4B05
:10B4A00000BF013BFCD124F40066B6B246F48050E4
:10B4B0001A4640FA02F111F0010F02F1010218BF21
:10B4C00001330F2AF5D1D90745BF47F2FF7020405D
:10B4D00046F4104040F48050FFF74CFF002319461B
:10B4E00040FA03F212F0010F03F1010318BF01311A
:10B4F0000F2BF5D1C0F3CF364E40F643420406F091
:10B50000010648BF46F0020683040BD4684046F0AB
:10B51000040610F4FE6FB6B202D046F00806B6B2CA
:10B52000304670BD2D0985EA10104006F5D1002E79
:10B53000F6D142F2341300BF013BFCD11A4644F469
:10B54000C05040FA02F111F0010F02F1010218BFE0
:10B5500001330F2AF5D1D9074ABFC4F30E0044F4D2
:10B56000184040F4C050FFF705FF00210B4640FA99
:10B5700003F212F0010F03F1010318BF01310F2B89
:10B58000F5D181EAD03111F0010F08BF1026420435
:10B5900044BF46F02006B6B283040BD485EA1015EA
:10B5A00046F040066906B6B2BAD046F08006B6B29A
:10B5B000304670BD85EA10104206F6D1002EAFD19C
:10B5C00042F2341300BF013BFCD124F4C0501A46B0
:10B5D00080B240FA02F111F0010F02F1010218BF2E
:10B5E00001330F2AF5D1DB074ABF46F2FF7040F462
:10B5F00000402040FFF7BEFE00210B4640FA03F258
:10B6000012F0010F03F1010318BF01310F2BF5D127
:10B6100081EAD03111F0010F08BF4FF48076410468
:10B6200044BF46F40076B6B2820458BF46F4806642
:10B6300085EA101558BFB6B26B061CBF46F400660B
:10B64000B6B2304670BD00BF1C7E06004FF6FA73DE
:10B65000034043F00200FFF703BF00BF4FF6FB7348
:10B66000034043F00300FFF7FBBE00BF4FF6FC733F
:10B67000034043F00400FFF7F3BE00BF10B54B7862
:10B6800082B0FE2B00F2A986DFE813F04606CA0559
:10B69000BD05B3052304A7060F04FB03A706E703B4
:10B6A000FA04E6047606DD04A706A706A706A706A1
:10B6B000A706A70679036A03A706A706A706FD053E
:10B6C000560359054B058A06A7064305A706A70694
:10B6D000A706A706A706A706A706A706A706A70602
:10B6E000A706A706A706A706A706A706A706A706F2
:10B6F0009B0625062F06AD039206E40553065B0460
:10B7000011030803FF02A706A706A706A706A706B8
:10B71000A706A706A706A706A706A706A706A706C1
:10B72000A706A706A706A706A706A706A706A706B1
:10B73000A706A706A706A706A706A706A706A706A1
:10B74000A706A706A706A706A706A706A706A70691
:10B75000A706A706A706A706A706A706A706A70681
:10B76000A706A706A706A706A706A706A706A70671
:10B77000A706A706A706A706A706A706A706A70661
:10B78000A706A706A706A706A706A706A706A70651
:10B79000A706A706A706EB028B05A706A706A7061E
:10B7A000A706A706A706A706A706A706A706A70631
:10B7B0007705A706A706A7066D056305DE03A7069E
:10B7C000A706D203C903A706A706B503A706BE04AA
:10B7D000A706AA04A70679046504A706A706A70674
:10B7E000A706A706C9044203A7062E031A032F05BE
:10B7F0001B051106A706A706A706A706A706A70604
:10B80000A706A706A706A7060E05D705A103950359
:10B8100089034F044304F005370439069F05A90541
:10B82000E2027302A7065F02A706A706A2024B0266
:10B8300098018F019902A70687010702FD01D60230
:10B84000F1016901A706A706A706A706A706A7068E
:10B850006101A70690025901DD01A706A706A70608
:10B86000C9017C02A706B50123020F02A706370211
:10B87000A706A7067401A706A706A706A7064601FE
:10B880003301A10120010D01FF00052800F084878C
:10B89000062800F0F087072801F09280082800F0C1
:10B8A0004F8702B010BD052800F0FA86062801F087
:10B8B0009680072801F0A2800828F2D1CE49012203
:10B8C000692002B0BDE81040FEF77ABB052800F001
:10B8D000B386062801F0FD80072801F01F810828A3
:10B8E000DFD1C64901226E2002B0BDE81040FEF74C
:10B8F00067BB052800F0C086062801F008810728EC
:10B9000001F014810828CCD1BD4904227C2002B06A
:10B91000BDE81040FEF754BB052800F0DF8606287E
:10B9200000F0C787072801F0BD800828B9D1B549C4
:10B9300001226C2002B0BDE81040FEF741BB062892
:10B94000AFD1019203F084FA019A5060A9E706286A
:10B95000A7D1019202F054FF019A5060A1E7052897
:10B9600000F0348706289CD10192FFF775FD019AFB
:10B97000506096E7052800F0C586062801F084800F
:10B98000072801F04B8008288BD19F4902226A20AA
:10B9900002B0BDE81040FEF713BB062881D101922A
:10B9A000FFF7BCFC019A50607BE706287FF479AF73
:10B9B0000192FDF7DFFE019A506072E706287FF4DE
:10B9C00070AF0192FDF7BCFF019A506069E705284E
:10B9D00000F0BE86062800F03987072801F016809F
:10B9E00008287FF45EAF894901226D2002B0BDE8CE
:10B9F0001040FEF7E5BA052800F03486062801F06D
:10BA00007F80072801F06C8008287FF44AAF8049C6
:10BA10000122AA2002B0BDE81040FEF7D1BA0528E5
:10BA200000F03486062800F0D387072801F06080F4
:10BA300008287FF436AF774904228C2002B0BDE895
:10BA40001040FEF7BDBA052800F02B85062801F04E
:10BA50009380072801F0088008287FF422AF6E4900
:10BA60000422882002B0BDE81040FEF7A9BA0528DC
:10BA700000F0988606287FF414AF0192FFF7E8FCE7
:10BA8000019A50600DE705287FF40BAF03F0D0F961
:10BA900002B0BDE81040FFF791BB05287FF401AF6D
:10BAA00002B0BDE81040FFF763BB052800F00C862C
:10BAB000062800F05187072800F03F8708287FF408
:10BAC000F0AE56490222AE2002B0BDE81040FEF7AB
:10BAD00077BA052800F0A685062800F0F387072826
:10BAE00001F0688008287FF4DCAE4D490222AC20CA
:10BAF00002B0BDE81040FEF763BA052800F0F885F3
:10BB0000062800F0DD86072801F0DC8008287FF495
:10BB1000C8AE44490422A02002B0BDE81040FEF7A0
:10BB20004FBA052800F0C685062800F00E870728C2
:10BB300000F0AF8608287FF4B4AE3B490422BC2055
:10BB400002B0BDE81040FEF73BBA052800F097842C
:10BB5000062800F02087072800F0A38608287FF435
:10BB6000A0AE32490122A92002B0BDE81040FEF784
:10BB700027BA06287FF495AE019203F081F9019A65
:10BB800050608EE6052800F0C785062800F0838700
:10BB9000072800F08F8708287FF483AE2449042209
:10BBA000902002B0BDE81040FEF70ABA06287FF4E4
:10BBB00078AE019203F046F9019A506071E60628CA
:10BBC0007FF46FAE0192FFF713FA019A506068E6B6
:10BBD000052800F0AB85062800F0EB86072800F06A
:10BBE0004B8708287FF45DAE12490422B82002B0CA
:10BBF000BDE81040FEF7E4B9F937FF1FFE37FF1F1D
:10BC00000C38FF1FFC37FF1FFA37FF1FFD37FF1FE0
:10BC10003A38FF1F1C38FF1F1838FF1F3E38FF1F20
:10BC20003C38FF1F3038FF1F4C38FF1F3938FF1FCB
:10BC30002038FF1F4838FF1F052800F0F38506282D
:10BC40007FF42FAE0192FFF7FFFB019A506028E6C8
:10BC500006287FF426AE019203F00CF9019A506099
:10BC60001FE6052800F07184062801F024800728CB
:10BC700001F0308008287FF414AECB4904225C2008
:10BC800002B0BDE81040FEF79BB906287FF409AE6C
:10BC9000022002F071F8C54B586002E606287FF4D6
:10BCA00000AE012002F068F8C04B5860F9E50628A4
:10BCB0007FF4F7AD002002F05FF8BC4B5860F0E570
:10BCC000052800F0E583062800F06C86072800F0C0
:10BCD000FE8508287FF4E5ADB5490222B22002B006
:10BCE000BDE81040FEF76CB9052800F091840628E5
:10BCF00001F00F80072800F0FD8708287FF4D1AD00
:10BD0000AC490222B02002B0BDE81040FEF758B99D
:10BD1000052800F03884062800F09A87072800F0EC
:10BD2000E18708287FF4BDADA3490422742002B046
:10BD3000BDE81040FEF744B9052800F0CD83062881
:10BD400000F0FC86072800F0CA8508287FF4A9AD1A
:10BD50009A490422982002B0BDE81040FEF730B99D
:10BD6000974C94F82F309A0740F13B830120FDF760
:10BD700079F801280FD08D4B00225A6091E5904C44
:10BD800094F82F3013F0010000F037830020FDF706
:10BD900069F80128EFD1854B01225A6081E5052819
:10BDA00000F0488506287FF47CAD019203F01EFC6C
:10BDB000019A506075E5052800F0D08406287FF4CC
:10BDC00070AD019203F00CFC019A506069E5052802
:10BDD00000F0D08406287FF464AD019203F0FAFBF2
:10BDE000019A50605DE506287FF45BADFDF7F0FF3A
:10BDF0006E4B586055E5052800F0F683062800F0E4
:10BE00004C87072800F01C8708287FF44AAD6D494D
:10BE10000122652002B0BDE81040FEF7D1B8062827
:10BE20007FF43FAD0192FEF719F8019A506038E5B2
:10BE3000052800F0B28306287FF433AD019202F0AA
:10BE400017FA019A50602CE506287FF42AAD01927A
:10BE500002F04CFA019A506023E5052800F0A78310
:10BE6000062800F00487072800F0F98608287FF4E8
:10BE700018AD55490422502002B0BDE81040FEF72D
:10BE80009FB8052800F0BA83062800F03B870728F2
:10BE900000F0808608287FF404AD4C490422482035
:10BEA00002B0BDE81040FEF78BB8052800F0028311
:10BEB000062800F06886072800F0748608287FF4BA
:10BEC000F0AC43490422442002B0BDE81040FEF724
:10BED00077B8052800F00983062800F03686072881
:10BEE00000F03A8608287FF4DCAC35490422402073
:10BEF00002B0BDE81040FEF763B8052800F05A8490
:10BF000006287FF4CEAC019203F088FB019A5060C2
:10BF1000C7E4052800F0548406287FF4C2AC0192DF
:10BF200003F070FB019A5060BBE4052800F05C84CC
:10BF300006287FF4B6AC019203F05EFB019A5060D4
:10BF4000AFE406287FF4ADAC224B1878FCF7AAFFCB
:10BF5000164B5860A5E4052800F06382062800F01F
:10BF60007F82072800F0DC8608287FF49AAC1A4903
:10BF700001226F2002B0BDE81040FEF721B805286D
:10BF800000F07482062800F07D84072800F0EC851C
:10BF900008287FF486AC11490222802002B0BDE857
:10BFA0001040FEF70DB800BFEC37FF1FB838FF1F79
:10BFB0004238FF1F4038FF1F0438FF1F2838FF1F7B
:10BFC000D037FF1FF537FF1FE037FF1FD837FF1FA0
:10BFD000D437FF1F1200FF1FFF37FF1F1038FF1F4E
:10BFE000052800F0D383062800F03E84072800F0DF
:10BFF0002F8208287FF455ACD3490122942002B047
:10C00000BDE81040FDF7DCBF052800F0FF830628DF
:10C01000ECD1019203F0AEF9019A506041E4052899
:10C0200000F0A782062800F0DC85072800F0CA850A
:10C0300008287FF436ACC5490422702002B0BDE860
:10C040001040FDF7BDBF06287FF42BAC019202F033
:10C050003FF9019A506024E4052800F03482062854
:10C0600000F08A84072800F08E8408287FF419AC39
:10C07000B7490422582002B0BDE81040FDF7A0BF28
:10C08000052800F06C82062800F0A485072800F03F
:10C090003C8408287FF405ACAE4904224C2002B051
:10C0A000BDE81040FDF78CBF052800F06983062825
:10C0B0007FF4F7AB019203F081FA019A5060FFF729
:10C0C000F0BB052800F0B681062800F04C84072854
:10C0D00000F02B8408287FF4E4AB9F490222B420AF
:10C0E00002B0BDE81040FDF76BBF052800F01882D4
:10C0F000062800F07D85072800F08A8508287FF44F
:10C10000D0AB96490422782002B0BDE81040FDF77C
:10C1100057BF05287FF4C5AB02B0BDE8104002F060
:10C12000EFBA052800F08C83062800F096830728D4
:10C130007FF4B7AB02B0BDE81040FEF7F3BF0628AE
:10C140007FF4AFAB0192FEF7DBFF019A5060FFF77F
:10C15000A8BB06287FF4A5AB019202F0C1F8019AB2
:10C160005060FFF79EBB06287FF49BAB019202F064
:10C1700001FB019A5060FFF794BB052800F02A826A
:10C18000062800F08385072800F0788508287FF4CA
:10C1900088AB73490122642002B0BDE81040FDF76E
:10C1A0000FBF052800F0AA81062800F0A083072809
:10C1B00000F03E8508287FF474AB6A4904226020B1
:10C1C00002B0BDE81040FDF7FBBE06287FF469AB66
:10C1D000019202F043FE019A5060FFF762BB06280D
:10C1E0007FF45FAB019202F03FFE019A5060FFF7CF
:10C1F00058BB06287FF455AB019202F0B5FA019ABC
:10C200005060FFF74EBB052800F0DB8106287FF465
:10C2100048AB019202F0B6F9019A5060FFF741BBBA
:10C22000052800F0A18206287FF43BAB019202F0C2
:10C23000A3F9019A5060FFF734BB052800F0CE82C5
:10C2400006287FF42EAB019203F0BEF9019A5060EC
:10C25000FFF727BB052800F0DB8006287FF421AB21
:10C26000FEF798F9404B5860FFF71BBB052800F01C
:10C27000C78206287FF415AB019203F0C9F9019A31
:10C280005060FFF70EBB052800F04181062800F042
:10C290003583072800F0418308287FF402AB334937
:10C2A00004229C2002B0BDE81040FDF789BE05289D
:10C2B00000F03F81062800F0A284072800F0968352
:10C2C00008287FF4EEAA2A490222B62002B0BDE86F
:10C2D0001040FDF775BE06287FF4E3AA0120FDF7A4
:10C2E00071FD214B5860FFF7DCBA06287FF4D9AA0C
:10C2F0000220FDF767FD1C4B5860FFF7D2BA0528F6
:10C3000000F08A8206287FF4CCAA019203F08CF90F
:10C31000019A5060FFF7C5BA052800F06B82062825
:10C320007FF4BFAA019201F0CDFF019A5060FFF7A0
:10C33000B8BA06287FF4B5AA0E4B1878FCF7B2FD00
:10C34000094B5860FFF7ADBA2438FF1F0038FF1FB4
:10C35000E837FF1FDC37FF1F4438FF1F0838FF1F77
:10C36000F437FF1FF037FF1FB838FF1F2C38FF1FAF
:10C370004638FF1F1100FF1F052800F0DD8006284A
:10C3800000F09284072800F04B8408287FF489AAE3
:10C39000AE490422542002B0BDE81040FDF710BEA3
:10C3A00005287FF47EAA02B0BDE81040FEF7CCBE9F
:10C3B00006287FF476AAFDF71DFDA54B5860FFF710
:10C3C00070BA06287FF46DAAFDF7F6FC0020FDF791
:10C3D000F9FC9F4B5860FFF764BA03231370FFF713
:10C3E00060BA0120FCF73EFD00283FF4D4AC94F87D
:10C3F0002F309B077FF5BFACB8E4FCF733FD002876
:10C400003FF4C9AC94F82F30D9073FF5BFACB2E484
:10C410004868012840F28C848D4B04221A70FFF783
:10C4200040BA4B68032B0FD88A4B0A7983F82F2028
:10C43000FFF737BA884B01924968187803F072F811
:10C44000019A00287FF42DAA04231370FFF729BA5C
:10C4500082490122942002B0BDE81040FDF7D6BD0C
:10C460007C4B93F82F305360FFF71BBA486801925A
:10C4700002F0A4FD019A0028E6D0FFF712BA48683E
:10C48000019202F0F9FF019A0028DDD0FFF709BA06
:10C490004868019203F024F8019A0028D4D0FFF7ED
:10C4A00000BA4868019202F01BFF019A0028CBD025
:10C4B000FFF7F7B94868019202F0EEFC019A0028F4
:10C4C000C2D0FFF7EEB94868019202F0F5FE019A7A
:10C4D0000028B9D0FFF7E5B94868019202F0B8FF2B
:10C4E000019A0028B0D0FFF7DCB94868019202F049
:10C4F00049FE019A0028A7D0FFF7D3B948680192F6
:10C5000002F0F6FD019A00289ED0FFF7CAB94868EC
:10C51000019202F089FF019A002895D0FFF7C1B976
:10C520004868019202F0CCFC019A00288CD0FFF7F9
:10C53000B8B901924A4B7FE74868019202F00EFEBB
:10C54000019A002880D0FFF7ACB94868019202F048
:10C5500041FE019A00283FF477AFFFF7A2B948687F
:10C56000019202F0E3FE019A00283FF46DAFFFF75D
:10C5700098B94868019202F0CDFD019A00283FF475
:10C5800063AFFFF78EB94868019202F0D5FD019ABA
:10C5900000283FF459AFFFF784B94868019201F0D1
:10C5A00085FE019A00283FF44FAFFFF77AB948683B
:10C5B000019202F0FBFD019A00283FF445AFFFF71E
:10C5C00070B94868019201F0EDFD019A00287FF4EE
:10C5D00068A939E74868019202F058FE019A0028DC
:10C5E0003FF432AFFFF75DB94868019202F052FDA7
:10C5F000019A00283FF428AFFFF753B94868019229
:10C6000002F080FE019A00283FF41EAFFFF749B9FF
:10C610004868019202F046FF019A00283FF414AFE7
:10C62000FFF73FB94868019202F0D6FE019A002850
:10C630003FF40AAFFFF735B94868019202F092FC67
:10C64000019A00283FF400AFFFF72BB9E437FF1F32
:10C65000B838FF1FD037FF1F1100FF1F2438FF1FFE
:10C660001200FF1F4868019202F0A4FE019A002800
:10C670003FF4EAAEFFF715B94868019202F084FC76
:10C68000019A00283FF4E0AEFFF70BB94868019229
:10C6900002F0D8FD019A00283FF4D6AEFFF701B9A9
:10C6A0004868019202F020FC019A00283FF4CCAEC9
:10C6B000FFF7F7B84868019202F074FF019A00286A
:10C6C0003FF4C2AEFFF7EDB84868019202F09AFE5F
:10C6D000019A00283FF4B8AEFFF7E3B8486801922A
:10C6E00002F09AFC019A00283FF4AEAEFFF7D9B8E9
:10C6F0004868019202F0A2FC019A00283FF4A4AE1F
:10C70000FFF7CFB84868019202F0B0FC019A002808
:10C710003FF49AAEFFF7C5B84868019202F0A4FD55
:10C72000019A00283FF490AEFFF7BBB84868019229
:10C7300002F0ECFE019A00283FF486AEFFF7B1B894
:10C74000BA490122682002B0BDE81040FDF738BCAC
:10C75000486802B0BDE8104002F044BC486802B02E
:10C76000BDE8104002F078BF486802B0BDE8104054
:10C7700001F0EABF486802B0BDE8104002F066BFB1
:10C78000486802B0BDE8104002F054BF486802B0EB
:10C79000BDE8104002F0F6BD486802B0BDE81040A8
:10C7A00002F0CCBB88880192FEF758FF019A5060D6
:10C7B000FFF777B8486802B0BDE8104002F06ABFE2
:10C7C000486802B0BDE8104002F058BF8888019266
:10C7D000FEF74CFF019A5060FFF763B8486802B05B
:10C7E000BDE8104002F02CBF486802B0BDE8104020
:10C7F00002F03EBF486802B0BDE8104001F000BD45
:10C80000486802B0BDE8104002F03EBF486802B080
:10C81000BDE8104002F09EBD486802B0BDE810407F
:10C8200002F03EBF88880192FEF710FF019A506027
:10C83000FFF737B8486802B0BDE8104002F012BFF9
:10C84000486802B0BDE81040FEF766BC019202F0F5
:10C85000D9FB019A5060FFF724B80192FEF756FC0D
:10C86000019A5060FFF71DB8019202F09BFD019AFA
:10C870005060FFF716B8019202F06AFB019A50600F
:10C88000FFF70FB8019202F0A7FB019A5060FFF783
:10C8900008B867490422BC2002B0BDE81040FDF78B
:10C8A000B5BB64490122A92002B0BDE81040FDF7E4
:10C8B000ADBB019202F0BCFB019A5060FEF7F1BFE4
:10C8C000019202F0CDFB019A5060FEF7EABF5A498F
:10C8D0000222B22002B0BDE81040FDF797BB5749D5
:10C8E0000422982002B0BDE81040FDF78FBB0192F2
:10C8F00002F00AFC019A5060FEF7D3BF019202F0E9
:10C90000A1FD019A5060FEF7CCBF4D4904224C2096
:10C9100002B0BDE81040FDF779BB4A4904229C20D3
:10C9200002B0BDE81040FDF771BB47490222B420B8
:10C9300002B0BDE81040FDF769BB44490222AE20B9
:10C9400002B0BDE81040FDF761BB019202F030FE7D
:10C95000019A5060FEF7A5BF019202F05FFD019AB7
:10C960005060FEF79EBF3A4B0192187802F002FE2B
:10C97000019A5060FEF795BF019202F0ABFC019A5C
:10C980005060FEF78EBF33490422582002B0BDE844
:10C990001040FDF73BBB019202F07AFD019A506016
:10C9A000FEF77FBF019202F0ABFD019A5060FEF7E7
:10C9B00078BF019202F0B0FD019A5060FEF771BF9E
:10C9C0001A490122682002B0BDE81040FDF71EBBE5
:10C9D000019202F043FC019A5060FEF762BF01929F
:10C9E00002F07CFA019A5060FEF75BBF1A490222FE
:10C9F000B62002B0BDE81040FDF708BB1749012280
:10CA0000692002B0BDE81040FDF700BB14490122C7
:10CA10006D2002B0BDE81040FDF7F8BA11490222BE
:10CA20006A2002B0BDE81040FDF7F0BAF837FF1FEA
:10CA30004C38FF1F3938FF1F4238FF1F2838FF1FAF
:10CA4000DC37FF1F2C38FF1F4438FF1F3E38FF1F05
:10CA50001100FF1FE837FF1F4638FF1FF937FF1F80
:10CA6000FD37FF1FFA37FF1FB4490422882002B0A8
:10CA7000BDE81040FDF7CABAB1490422B82002B09F
:10CA8000BDE81040FDF7C2BA019202F0FDFA019A2A
:10CA90005060FEF706BF019202F0F2FB019A50606F
:10CAA000FEF7FFBEA74901226C2002B0BDE810408E
:10CAB000FDF7ACBAA4490422902002B0BDE81040B2
:10CAC000FDF7A4BA019202F097FC019A5060FEF7BC
:10CAD000E8BE019202F052FA019A5060FEF7E1BE00
:10CAE0009A490122AA2002B0BDE81040FDF78EBA93
:10CAF000974904228C2002B0BDE81040FDF786BAA9
:10CB0000019202F063FC019A5060FEF7CABE0192E6
:10CB100002F04EFA019A5060FEF7C3BE8D49012221
:10CB20006E2002B0BDE81040FDF770BA8A490422B9
:10CB30007C2002B0BDE81040FDF768BA019202F017
:10CB400095FC019A5060FEF7ACBE019202F028FB02
:10CB5000019A5060FEF7A5BE80490422402002B031
:10CB6000BDE81040FDF752BA7D490222802002B094
:10CB7000BDE81040FDF74ABA019202F0BDFB019AF0
:10CB80005060FEF78EBE019202F080F9019A50606B
:10CB9000FEF787BE73490422482002B0BDE810406A
:10CBA000FDF734BA70490422442002B0BDE81040B9
:10CBB000FDF72CBA6D490222AC2002B0BDE810404E
:10CBC000FDF724BA6A490422702002B0BDE8104083
:10CBD000FDF71CBA019202F0B7FB019A5060FEF714
:10CBE00060BE019202F0A2FA019A5060FEF759BEAF
:10CBF000019202F05FF9019A5060FEF752BE5D4B60
:10CC00000192187802F0B6FC019A5060FEF749BE16
:10CC100059490422782002B0BDE81040FDF7F6B96A
:10CC200056490422542002B0BDE81040FDF7EEB989
:10CC300053490422602002B0BDE81040FDF7E6B978
:10CC400050490122652002B0BDE81040FDF7DEB971
:10CC5000019202F07DFA019A5060FEF722BE4A4925
:10CC60000422502002B0BDE81040FDF7CFB9019278
:10CC700002F0AAFA019A5060FEF713BE434901225E
:10CC8000642002B0BDE81040FDF7C0B9019202F087
:10CC900009FB019A5060FEF704BE019202F00CFA03
:10CCA000019A5060FEF7FDBD019202F065FA019A0B
:10CCB0005060FEF7F6BD019202F0BEFA019A506094
:10CCC000FEF7EFBD32490422A02002B0BDE81040BB
:10CCD000FDF79CB92F4904225C2002B0BDE810404A
:10CCE000FDF794B92C490422742002B0BDE810402D
:10CCF000FDF78CB929490222B02002B0BDE81040EE
:10CD0000FDF784B9019202F00BFB019A5060FEF727
:10CD1000C8BD019202F0DEFB019A5060FEF7C1BD72
:10CD20001F4901226F2002B0BDE81040FDF76EB927
:10CD3000C0B202B0BDE81040FDF732BC1838FF1F8A
:10CD40004838FF1FFC37FF1F2038FF1F3A38FF1FEE
:10CD50001C38FF1FFE37FF1F0C38FF1FD037FF1F87
:10CD60001038FF1FD837FF1FD437FF1F3C38FF1F75
:10CD70000038FF1F1200FF1F0838FF1FE437FF1F96
:10CD8000F037FF1FF537FF1FE037FF1FF437FF1F96
:10CD90003038FF1FEC37FF1F0438FF1F4038FF1FDC
:10CDA000FF37FF1F70B51049104C114B00224FF494
:10CDB00080700880227003F5806143F8042F8B4255
:10CDC000FBD10C4BDB7D73B90B4E40F21A7440F271
:10CDD000FA75A4F21A710422204631441444FDF776
:10CDE000EFF8AC42F5D170BD6846FF1F663EFF1FED
:10CDF000C838FF1F5438FF1FCC38FF1F014B18786D
:10CE0000704700BF643EFF1F8B780BB9FEF736BC3E
:10CE100010B40423137010BC704700BF08B5874AD4
:10CE20009378002B40F0C7805378403BBF2B00F233
:10CE3000CE80DFE813F0BF018601A401CC004001E1
:10CE4000CC00CC00CC00CC006601CC0057017701AF
:10CE50002301EE01CC00CC00CC00CC009501CC002D
:10CE6000CC01CC003101CC00CC00DF01CC00CC00E7
:10CE7000CC00CC00CC00CC00CC00CC00CC00CC0052
:10CE8000CC00CC00CC00CC00CC00CC00CC00CC0042
:10CE9000CC00CC00CC00CC00CC00CC00CC00CC0032
:10CEA000CC00CC00CC00CC00CC00CC00CC00CC0022
:10CEB000CC00CC00CC004F01B201CC0019010F0115
:10CEC000CC00CC00CC00CC00CC00CC00CC00CC0002
:10CED000CC00CC00CC00CC00CC00CC00CC00CC00F2
:10CEE000CC00CC00CC00CC00CC00CC00CC00CC00E2
:10CEF000CC00CC00CC00CC00CC00CC00CC00CC00D2
:10CF0000CC00CC00CC00CC00CC00CC00CC00CC00C1
:10CF1000CC00CC00CC00CC00CC00CC00CC00CC00B1
:10CF2000CC00CC00CC00CC00CC00CC00CC00CC00A1
:10CF3000CC00CC00CC00CC00CC00CC00CC00CC0091
:10CF4000CC00CC00CC00CC00CC00CC00CC00CC0081
:10CF5000CC00CC00CC00CC00CC00CC00CC00CC0071
:10CF6000CC00CC00CC00CC00CC00CC00CC00CC0061
:10CF7000CC00CC00CC00CC00CC00CC00CC00CC0051
:10CF8000CC00CC00CC00CC00CC00CC00CC00CC0041
:10CF9000CC00CC00CC00E900CC00CC00CC00CC0014
:10CFA000CC00CC00CC00CC00CC00CC00CC00CC0021
:10CFB000CC00E900FA00012B0CD0022B0BD0204B47
:10CFC00004221A7008BD1F490988994223D81C4BB6
:10CFD00003221A7008BD5378372BF4D80A2800F0C2
:10CFE000268109281CD00B2800F082810C28F1D161
:10CFF0001549042240F21A7001EB830102FB030081
:10D00000BDE80840FCF7DCBF0A28E3D10F4A0C4B0F
:10D0100012785A6008BD0A2800F009810928D9D180
:10D020000949526841F8232008BD0A2800F04981C7
:10D030000928CFD1064B12791A7008BDC438FF1FDA
:10D04000B838FF1F6846FF1FCC38FF1F5038FF1F3E
:10D05000B138FF1F0A2800F0FF800928BAD1AE4A74
:10D06000AE4B52681A6008BD0A2800F01D810928DD
:10D07000B0D1A94AAA4B52681A6008BD0A2800F02C
:10D08000FF800928A6D11379A64A537519461520A1
:10D09000BDE80840FCF75EBF0A2800F0D3800928ED
:10D0A00098D1A049137901F8023F01220220BDE87E
:10D0B0000840FCF7ABBF0A2800F0D880092889D1C6
:10D0C0009849536841F8183F04221820BDE80840E9
:10D0D000FCF79CBF0A287FF47DAF934A8E4B1278F1
:10D0E0005A6008BD0A2800F0DA8009287FF472AF80
:10D0F00013798C4A137119460420BDE80840FCF7E7
:10D1000029BF0A2800F0D58009287FF463AF117980
:10D11000002940F0E780834B99751620BDE8084050
:10D12000FCF718BF0A2800F0888009287FF452AF66
:10D1300013797C4AD37019460320BDE80840FCF7F8
:10D1400009BF0A2800F0A18009287FF443AF1379B2
:10D15000744A137019460020BDE80840FCF7FABE77
:10D160000A2874D009287FF435AF6E49536841F816
:10D17000103F04221020BDE80840FCF747BF0A28F2
:10D180006FD009287FF426AF1379664A5370194689
:10D190000120BDE80840FCF7DDBE0A287FF41AAF85
:10D1A000614B5D4A1B78A3F10403B3FA83F35B0977
:10D1B000536008BD0A2800F0A78009287FF40AAF51
:10D1C000117940F2FF70BDE80840FCF7C3BE0A28A1
:10D1D00051D009287FF4FEAE5368012B3FF6EFAE25
:10D1E0005049137901F8173F01221720BDE8084084
:10D1F000FCF70CBF0A284DD009287FF4EBAE494953
:10D20000536841F8203F04222020BDE80840FCF785
:10D21000FDBE0A285DD0092860D00B287FF4DAAE65
:10D22000404B0720D979BDE80840FCF793BE3F4941
:10D23000394A51F82330536008BD3A4A364BD27808
:10D240005A6008BD374A344B92785A6008BD354A57
:10D25000314B12695A6008BD304A2F4B12685A6030
:10D2600008BD304A2C4B52785A6008BD2D4A2A4BD3
:10D2700092695A6008BD2B4A274BD27D5A6008BD7F
:10D28000284A254B527D5A6008BD264A224B127807
:10D290005A6008BD234A204B126A5A6008BD214AD1
:10D2A0001D4B12795A6008BD1D4A1B4B12685A600B
:10D2B00008BD1C4B184A9B7D003318BF01235360E7
:10D2C00008BD1B4B144A1B78003318BF0123536061
:10D2D00008BD144A104BD2795A6008BD114B12791F
:10D2E000DA7108BD0F4A0C4B01219175596014E7A2
:10D2F0000E49042240F21A7001EB830102FB030085
:10D30000BDE80840FCF782BE40F2FF70FCF708FE63
:10D31000014B586008BD00BFB838FF1F6C46FF1FA7
:10D320007046FF1F5438FF1FB238FF1FCC38FF1F55
:10D33000B138FF1F074B9A78022A04D15A685878EF
:10D340002AB9FBF7A9BD044B04221A707047FBF7FA
:10D35000A5BD00BFC438FF1FB838FF1F38B5184B34
:10D360009A78012A14D00BD3022A05D15878FBF7FA
:10D3700097FD144B586038BD124B04221A7038BD0B
:10D380005878FF280AD0FBF76DFD0E4B586038BD6A
:10D390005878FBF787FD0B4B586038BD0120FBF731
:10D3A00061FD05460020FBF75DFD44000220FBF710
:10D3B00059FD44EA8504034B2043586038BD00BF43
:10D3C000C438FF1FB838FF1F034B9A7802B170476B
:10D3D0005868404200F0E6BEC438FF1F034B9A78FD
:10D3E00002B17047586800F0DDBE00BFC438FF1FAF
:10D3F000024B987800B1704700F0D4BEC438FF1FCC
:10D400000A4B9A7832B95A7862B1012A06D1586823
:10D4100000F026BF064B04221A707047044B03220B
:10D420001A707047586800F0EBBE00BFC438FF1F89
:10D43000B838FF1F10B4124B5B789BB91149124BDF
:10D440000868124A1249DB7802F8013B0124431EA6
:10D450000C70073013F8011F02F8011B8342F9D149
:10D4600010BC7047012BFBD10A4BC1246020042162
:10D470000022DC71987159711A7110BC704700BF9D
:10D48000C438FF1F2000FF1F5438FF1FA838FF1F9C
:10D49000A438FF1FB838FF1FF8B50D490D4B01E048
:10D4A0008B4207D053F8042F0132F9D00A4B0822DF
:10D4B0001A70F8BD094C0A4F04F50066C4F5FE2544
:10D4C000281954F8041FB847B442F9D1F8BD00BF79
:10D4D000FCF70700FCEF0700B838FF1F643EFF1F92
:10D4E0006DA201000C4A5378012B10D009D3FF2BF9
:10D4F00006D15368094A03F5FE231B685360704741
:10D5000070474FF4FE22054B12685A607047044A78
:10D51000024B12685A607047C438FF1FB838FF1FAB
:10D5200004F007004FF0E02318B9044AC3F80C2DAB
:10D530007047034AC3F80C2D704700BF0100FA057D
:10D540000400FA05194A1A4938B5136823F07F43D5
:10D5500023F0FF038B4203D0164B04221A7038BD10
:10D560005268154B9A42F7D1FBF742FC72B6FCF7B2
:10D57000FDF9124C124B134D13484FF0E0214FF0C0
:10D58000FF32C3F88020C3F88021C3F88420C3F899
:10D590008421C3F88820C3F88821C3F88C20C3F8FD
:10D5A0008C212560C1F80C0D38BD00BFC438FF1FA9
:10D5B00000819200B838FF1FD6C5B4A30000FF1F3A
:10D5C00000E100E0785634120400FA05044B5A6872
:10D5D00040F2D2439A4202D1024B01221A707047A4
:10D5E000C438FF1F663EFF1F10B52B4B98785A7842
:10D5F00038B1032A0FD0042A49D0284B04221A70CC
:10D6000010BD0A2A3FD8DFE802F00D121706421CAF
:10D61000202A2F3439000146586802F0BBF81F4B0E
:10D62000586010BD02F0B0F81C4B586010BD02F0FD
:10D63000A7F81A4B586010BD02F0AAF8174B5860B3
:10D6400010BDBDE8104002F03FB802F045F80446B6
:10D6500002F048F8114B2043C0B2586010BD586822
:10D66000BDE8104002F0A6B802F0BCF80B4B5860C1
:10D6700010BD5868BDE8104002F0BAB802F0BEF81C
:10D68000064B586010BD054B03221A7010BD596837
:10D69000BDE8104002F00AB8C438FF1FB838FF1FB9
:10D6A00010B54849484A08784B68507064240E28E1
:10D6B0001470536079D00ED98E2837D01BD9D22858
:10D6C0006FD021D9F22868D0FF281AD140F2D24277
:10D6D000934272D010BD042838D02FD8022819D018
:10D6E00038D801280DD18A78002AF3D11846BDE830
:10D6F000104000F057BD882814D0892836D00F2854
:10D7000018D002231370E5E7D128FAD1BDE8104004
:10D71000FFF7C2BE8A78002ADCD15842BDE810402B
:10D7200000F040BDBDE81040FFF784BEBDE81040EA
:10D73000FFF75ABFBDE81040FFF710BE082810D908
:10D740000C28DED8BDE81040FFF768BBBDE81040EC
:10D75000FFF756BE88780028BCD1BDE8104000F025
:10D7600021BD8B782BB30423137010BD096821F001
:10D770007F4121F0FF010029ACD140F2D242934217
:10D78000A8D140F2FF70FCF7E5FBFCF789FD4FF0F4
:10D79000E0230E4AC3F80C2D10BDBDE81040FFF782
:10D7A000D1BEBDE81040FFF79DBEBDE81040FFF7B9
:10D7B000C1BDBDE81040FDF761BF054B01221A70E5
:10D7C00010BD00BFC438FF1FB838FF1F0400FA05A2
:10D7D000663EFF1F2DE9F043954B964D1B7883B0B5
:10D7E00053B92B7843B9944C2378032B33D0042BB3
:10D7F00000F0AD80914E07E0914B1B78063BDBB209
:10D80000192B1FD98C4C8D4E8E4B1A780023237008
:10D8100033702B7022B14FF0E0238B4AC3F80C2DEC
:10D820000DF10700FBF74AFE002850D1874B1B780B
:10D83000042B7BD02278082A41D9FFF731FF03B0AF
:10D84000BDE8F083824A22FA03F3DA07DAD57A4C8C
:10D850002378032BCBD1794E3378002B00F0A580B1
:10D86000012BD1D17B4F07F1090817F8010FFBF706
:10D870000BFE4745F9D1C7E7714D6379617AA27A0A
:10D88000A779E679207A2B70E37AA9716A712B71F6
:10D890006F70AE70E871FCF76FF86C4A6E4B1278DF
:10D8A0006E491860042A4FF000004FF0030308701F
:10D8B0002370C2D195F90020002A3DDA1A4640F2C1
:10D8C0005113D340DB07B8D503B0BDE8F083FBF7B5
:10D8D0000FFE002835D162789DF80710531CDBB28B
:10D8E0002244092B63701171A0D15D4B21795A78C4
:10D8F00060708A429B7800F09680002B96D0994207
:10D9000094D101232B70574A0023D01D01E012F857
:10D91000011B0B448242DBB2F9D1227B9A42ABD08D
:10D920004A4B1B78042293422270CDD1444B93F989
:10D930000030002BFFF67EAF01F07AFA03B0BDE8AD
:10D94000F08301229DF80730627023716EE7DFF8E3
:10D950001091454F99F8030099F80180374E012343
:10D960003B7000237B707B608044FBF78DFD99F852
:10D970000100FBF789FD3878FBF786FD7878FBF727
:10D9800083FDF879FBF780FDB879FBF77DFD08F1A1
:10D9900001087879FBF778FD5FFA88F83879FBF7AA
:10D9A00073FD4046FBF770FD2EE7DFF8B490DFF81B
:10D9B000B88099F8030099F8017098F8002098F859
:10D9C00001300744174498F807201F4498F80630A0
:10D9D000174498F805201F4498F8043017441F4452
:10D9E000FBF752FD99F80100FBF74EFD98F8000097
:10D9F000FBF74AFD98F80100FBF746FD98F8070091
:10DA0000FBF742FD98F80600FBF73EFD98F805008D
:10DA1000FBF73AFDFFB298F80400FBF735FD3846F6
:10DA2000FBF732FDF0E68B427FF46DAF69E700BF94
:10DA3000B138FF1F653EFF1F6022FF1FA438FF1F84
:10DA4000C438FF1F663EFF1F0400FA05B238FF1FEF
:10DA500011020002A738FF1FB438FF1FC038FF1F94
:10DA60005438FF1F6522FF1FB838FF1FF0B5254B44
:10DA7000254C0246007992F801E09678D778D87163
:10DA8000507998710D469179597194E8030083B0EB
:10DA9000D2795E7083F800E09F701A718DE8030000
:10DAA000FFF7FEFD194B1B786E46B3B1012B05D075
:10DAB00096E8030084E8030003B0F0BD144A6B1E2F
:10DAC000073512F8011B03F8011FAB42F9D196E8A4
:10DAD000030084E8030003B0F0BD2B706B70637823
:10DAE0002278AA70EB70E3792B71A3796B7163795B
:10DAF000AB7196E803002379EB7184E8030003B06F
:10DB0000F0BD00BFC438FF1FB838FF1FA438FF1F87
:10DB1000A938FF1FF0B50D4C0D4E05460F4694E891
:10DB2000030083B03570B27073608DE803007770C6
:10DB3000FFF7B6FD9DE8030063682578054A84E891
:10DB400003001846157003B0F0BD00BFB838FF1FC2
:10DB5000C438FF1F643EFF1F08B50C4B196821F045
:10DB60007F4121F0FF0121B95A6840F2D2439A4225
:10DB700000D008BD40F2FF70FCF7ECF9FCF790FB19
:10DB80004FF0E023024AC3F80C2D08BDC438FF1F34
:10DB90000400FA050000000010B50D4CFBF7B2FDC3
:10DBA00094F82920E36B21465208B3FBF2F3B0FB53
:10DBB000F3F202FB130021F8400F02228020FCF751
:10DBC00025FA94F8423023F0010384F8423010BD66
:10DBD000D037FF1F10B5064CB4F84000FBF7A4FD8A
:10DBE00094F8423023F0020384F8423010BD00BFA5
:10DBF000D037FF1F38B50020FBF7C2F90B4B93F865
:10DC00002520092A054602D9094C257038BD40F265
:10DC10004123D340DB07064CF7D501462078FBF7BC
:10DC200043FE636825701844606038BDD037FF1F1D
:10DC30007022FF1F684620F007018D4619B5164B6C
:10DC4000D3F8A030590609D5144C94F82530072B89
:10DC500008D0114A936943F080739361BDE819407D
:10DC60008546704794F84230DA0703D5FFF794FFF2
:10DC700094F84230980701D5FFF7ACFF94F8543080
:10DC8000D907E6D5064A002151605A07E1D523F0AD
:10DC9000010384F85430DCE700A00440D037FF1FB4
:10DCA0007022FF1F1A4B6846D3F8A02020F007010E
:10DCB0008D46910601B503D4D3F8A020120617D5DE
:10DCC000FFF798FF0020FBF75BF904281BD0104BEF
:10DCD0005A6942F080725A61DA6942F08072DA6100
:10DCE0001A6A42F080721A62BDE8014085467047A8
:10DCF000D3F8A030DB05F7D5FFF77CFF0020FBF75A
:10DD00003FF90428E3D101210220FBF757F8DEE7B1
:10DD100000B00440114B684620F00701D3F8A02062
:10DD20008D4601B4D00703D51A6842F080721A609C
:10DD30000A4BD3F8A020910703D55A6842F08072AD
:10DD40005A60064BD3F8A020520703D59A6842F0D8
:10DD500080729A6001BC8546704700BF00D00440C5
:10DD60000346044A00EBD070C0F34F0082F829301C
:10DD7000FBF7A2BCD037FF1F01280CD007D3022825
:10DD800003D1074BB3F90400704700207047044BE0
:10DD9000B3F900007047024BB3F90200704700BFAF
:10DDA000D846FF1FFBF70CB800B585B001F094FC16
:10DDB00010B905B05DF804FB01F014FD0328F8D19B
:10DDC0000020FBF76FF800900120FBF76BF8019043
:10DDD0000420FBF767F802900520FBF763F804AB1B
:10DDE000039013E90F0001F099FCE2E770B50A4CCB
:10DDF0000A4DE06909F06AFB0146094809F072FC26
:10DE0000064694F8290009F061FB0146304609F006
:10DE100069FC286070BD00BFD037FF1F3000FF1FB6
:10DE20000050C34870B5094C094DE06909F04EFB3C
:10DE30000146084809F056FC0646E06B09F046FB2F
:10DE40000146304609F04EFC686070BDD037FF1FB8
:10DE50003000FF1F007C924938B5054600200C4673
:10DE6000FBF78EF8314B93F8283013B180F00700A0
:10DE7000C0B214B980F00700C0B22D4B0022C3F825
:10DE8000902007280FD8DFE800F01D212B313C47F8
:10DE9000041D274B27490C24002202201C668860A1
:10DEA0009D619A629A63224B9A6D4FF4007042F022
:10DEB00004029A650021C3F898000220BDE83840AA
:10DEC000FAF77CBF1A4B3F221A66ECE7184B194948
:10DED00000220C2018668A609A619A629D63E2E7CC
:10DEE000134B1449302400220120D7E7104B11496D
:10DEF0000022032401201C6688609A619A629D6357
:10DF0000D1E70B4B0B490022032402201C668860DA
:10DF10009A619D629A63C6E7054B0649002230204C
:10DF200018668A609A619D629A63BCE7D037FF1FCA
:10DF3000008003407022FF1FF8B5514C514E94F8F9
:10DF40002500FBF755FDE06909F0C0FA01460546DA
:10DF50004D4809F0C7FB074694F8290009F0B6FAC6
:10DF60000146384609F0BEFB29463060474809F0B3
:10DF7000B9FB0546E06B09F0A9FA0146284609F00D
:10DF8000B1FB94F825507060062D30D0072D3CD0A1
:10DF9000082D5BD0092D12D06DB94FF40040FBF76E
:10DFA0002FFF8020FBF734FF0120FBF71DFC2946E3
:10DFB0002846FFF751FFBDE8F840FAF701BF4FF4DC
:10DFC0000040FBF71DFF8020FBF722FF0120FBF73D
:10DFD0000BFC94F82D10E06BFBF7FEFA94F8291077
:10DFE000E06B4908FBF75EFB94F82550D4E74FF44B
:10DFF0000040FBF705FF8020FBF70AFF0120FBF73D
:10E00000F3FB94F82550072DC2D14FF40040FBF7E5
:10E01000FFFE8020FBF7FCFE94F82C30012B2AD069
:10E0200094F82D10E06BFBF7D7FA94F82910E06B09
:10E030004908FBF737FBFBF785FBFCF7D1FF012015
:10E04000FBF786FB94F82550082DA3D14FF4004030
:10E05000FBF7D6FE0020FBF7C7FB94F82D10E06B12
:10E06000FBF7BAFA94F82910E06B4908FBF71AFBA2
:10E0700094F825508EE70020FBF7B6FBD0E700BFF1
:10E08000D037FF1F3000FF1F0050C348007C92496B
:10E09000014B01221A7370477022FF1FB0F5007FF9
:10E0A00010B504464AD02CDDB0F5806F1CD0B0F519
:10E0B000006F16D1FBF7A4FE4FF48070FBF7A8FEAB
:10E0C0004FF48060FBF7A4FE4FF40070FBF7A0FE56
:10E0D0004FF48040FBF79CFE1D4BA3F86640FAF717
:10E0E00063FE1C4B1C6010BDFBF78AFE4FF4807072
:10E0F000FBF78EFE4FF40070FBF78AFE4FF40060D2
:10E10000E4E7B0F5807FECD1FBF77AFE4FF4806056
:10E11000FBF77EFE4FF40070FBF77AFE4FF40060D1
:10E12000FBF776FE4FF48040FBF772FE084BA3F836
:10E130006640FAF73BFE074B1C6010BDFBF760FE24
:10E140004FF48070FBF764FE4FF48060D4E700BFAB
:10E15000D037FF1FC846FF1F08B50F4B93F8252087
:10E1600012B993F8692082B90C4A9B6F000290FBA8
:10E17000F3F010604FF40060FFF790FF084B0022AF
:10E180001A60FAF71DFE012008BD044ADB6F000289
:10E1900090FBF3F01060EDE7D037FF1FD046FF1F74
:10E1A0000047FF1F00F54333104A03F5A073934265
:10E1B00001D9002070470E4A0E4B10B51468186044
:10E1C0004FF40070FFF76AFFB4F5006F03D0FAF761
:10E1D000F7FD012010BD084B084C186809F07AF9CA
:10E1E0002060FAF7EDFD012010BD00BF801A060087
:10E1F000C846FF1F3847FF1FC446FF1F0047FF1FC9
:10E20000124A134B10B510611C684FF48060FFF781
:10E2100045FF4FF48040FBF7FBFDB4F5007F0CD0C9
:10E22000B4F5006F05D10B4B0B4C186809F052F98F
:10E230002060BDE81040FAF7C3BD084A064B1268DB
:10E240001A60BDE81040FAF7BBBD00BF7022FF1F87
:10E25000C846FF1FC446FF1F7846FF1F0047FF1F29
:10E26000024B5B681844FFF7CBBF00BF7022FF1F53
:10E270000C4B93F8252012B993F8692042B90A4A49
:10E280009B6F106800FB03F0002808DB001270474A
:10E29000054ADB6F106800FB03F00028F6DAFF3058
:10E2A00000127047D037FF1FC046FF1F00F5AF3385
:10E2B000034A03F5C873934200D84DE70020704726
:10E2C00020BF0200014B1869704700BF7022FF1F7A
:10E2D00008B5024B186809F017FB08BD0047FF1F7F
:10E2E000014B5869704700BF7022FF1F014B9869AE
:10E2F000704700BF7022FF1F10B5164B164C1878E0
:10E30000FAF7D0FD4FF4C673144A03FB00F082FB0A
:10E3100000320244C017C0EBE230B0F58C7F606180
:10E320004FF004000ADBFBF76BFD63693C2B4FF0F9
:10E3300002000ADDBDE81040FBF76ABDFBF768FD8F
:10E3400063693C2B4FF00200F4DCBDE81040FBF7A2
:10E3500057BD00BF1900FF1F7022FF1F0180008002
:10E3600010B5454B454C1878FAF79CFDC0F30F10DB
:10E3700009F0B0F808F0A0FC02460B4632A1D1E942
:10E38000000108F017FE32A3D3E9002308F034FBA4
:10E3900008F096FF3A4909F0A5F908F08DFC09F05C
:10E3A00099FD2DA3D3E9002308F0DAFC2CA3D3E9CF
:10E3B000002308F023FB02460B462BA1D1E9000104
:10E3C00008F0F8FD2AA3D3E9002308F015FB08F0B4
:10E3D00077FF09F099FAA0610820FBF72DFDA369EA
:10E3E00048B9772B4FF0080022DCFBF711FDFAF754
:10E3F0002FFD48B110BD6D2BFCDC0820FBF708FD9C
:10E40000FAF726FD0028F5D1FBF732FD0028F1D1FF
:10E410004FF40050FBF710FD0028EBD14FF4807053
:10E42000FBF70AFD0028E5D1BDE81040FAF7C8BCAB
:10E43000FBF7E6FCFAF7DCFC4FF48070BDE8104017
:10E44000FFF72CBEAFF300809A9999999999C14032
:10E450009A999999999901400000000000A0724092
:10E460000000000000D4AA4000000000C83A2F417C
:10E4700000000000001071401800FF1F7022FF1FF5
:10E480000000204138B5374DFBF776FAEB69C31A27
:10E49000002BB8BF5B42B3F57A7F50DA324CFFF7FE
:10E4A0002BFFFCF713FFFCF72BFEA36D98422DD832
:10E4B000FBF762FA6B6AE26DC01A0028B8BF4042EF
:10E4C00090420ED394F86420012A03D001F00AF997
:10E4D00098B938BD0023254984F86430A420FBF79F
:10E4E00095FD94F86430012BF0D14FF40030FBF728
:10E4F00087FC01F0F7F80028EBD01D4A1D4B10688F
:10E5000019686A68BDE8384001F07EB9FBF734FA53
:10E510002B6AC01A0028B8BF4042B0F57A7FC7DB2B
:10E52000FCF77EFD4FF40030FBF76AFC94F8643092
:10E5300063B1FCF7F7FDFBF71FFA2862B8E7044662
:10E54000FCF7D6FEFFF70CFFEC61A7E7214601229E
:10E5500001F8642FA420FBF759FDFBF70DFA686260
:10E56000E7E700BF7022FF1FD037FF1F3438FF1FBF
:10E57000CC46FF1FC446FF1F014B5868704700BFC1
:10E580007022FF1F014B1868704700BF3847FF1FFC
:10E590002DE9F041414C94F8253082B00546092B15
:10E5A00025D8DFE803F0322424242424320527323E
:10E5B000FBF7A8F8E16B3A4C8A10904202EB420656
:10E5C000636B2CDA9E422ADAC31A0B44354E61681B
:10E5D00032686063C91AD01A3060616013B1324A80
:10E5E0005B429360002D3FD0304BA26A1A6002B0AC
:10E5F000BDE8F0812E4B186809F086F92B4A284BAC
:10E600001060986202B0BDE8F08178B1244B274ACF
:10E610005868996AD862116002B0BDE8F081B042D2
:10E6200020DD9A421EDDC31A5B1ACFE71C4C1F4D3A
:10E63000E36A60682E68C01A08F04CFF1A4B19682C
:10E6400008F09CFF09F060F9082301460093324668
:10E65000052304F1300001F0C9F963682860A06265
:10E66000E362C4E7C31AB1E708F034FF0E4B0F4F63
:10E670005968D7F8008008F081FF09F045F90823B0
:10E680000146424600930B48022301F0AFF90A4BC2
:10E6900032683860A0621A603560A8E7D037FF1F83
:10E6A0007022FF1F2847FF1F3000FF1FC446FF1FB7
:10E6B0000047FF1FA022FF1FD446FF1F08B50120FF
:10E6C000FFF766FFFFF738FC0120FFF761FF034A01
:10E6D000034B92F825201A7308BD00BFD037FF1FE7
:10E6E0003000FF1F044A054B92F825201B7B9A42FD
:10E6F00000D0E3E7704700BFD037FF1F3000FF1F97
:10E70000F8B50B4B0B4F58680B4E0C4D0C4C0D498C
:10E7100018610022002301203B6033602B602260DF
:10E720000A60FFF735FFBDE8F840FFF705BC00BF02
:10E730007022FF1F3847FF1FC046FF1FD046FF1F34
:10E740007846FF1F0047FF1F10B504464FF4804076
:10E75000FBF75EFB034B01205C601C61BDE81040D1
:10E76000FFF716BF7022FF1F014B1868704700BFEC
:10E77000C446FF1F0C4B93F8252012B993F869206B
:10E7800042B90A4A986F136800FB03F0002808DBBF
:10E7900000127047054AD86F136800FB03F0002889
:10E7A000F6DAFF3000127047D037FF1FCC46FF1F4C
:10E7B000034A92F8423023EA000082F84200704790
:10E7C000D037FF1F034B93F84230184214BF01208B
:10E7D00000207047D037FF1F034A92F8543023EAD5
:10E7E000000082F854007047D037FF1F034B93F8A6
:10E7F0005430184214BF012000207047D037FF1F4B
:10E80000014B1868704700BFE046FF1F684620F0C4
:10E8100007018D462DE9F14FB94D8EB00121002041
:10E82000FAF7CCFA95F82530002B35D1B54CB64A1D
:10E83000B4F9381081EAE173A3EBE1739B10D36064
:10E84000136843F001031360B048E26B0168236C66
:10E8500021F080010160217B01320133E2632364F6
:10E8600051B1AB4A95F82510127B914202D0FFF7C7
:10E8700025FF236C00222273EA699A4240D92A6A52
:10E88000E36B9A4211D900210846FAF797FA0EB0C5
:10E89000BDE8F14F854670479B4B9A4C0022DA60E9
:10E8A0001A6842F001021A60CEE70023E36301F028
:10E8B0004BFA4FF48060FBF7BFFA002800F03E816E
:10E8C00095F82560002E40F0558195F86930012BB0
:10E8D00000F0838008A8FBF7D7FAA2688D4B089850
:10E8E000BDF824109980012A186000F00882022ADD
:10E8F00000F00182002A73D11E88764236B26FE0A2
:10E900000026854F266401F02FFA3046FFF740FEBF
:10E910003A682B6982EAE271A1EBE27183EAE37261
:10E92000A2EBE37291424FF0100053DDFBF770FA57
:10E930004FF48060FBF780FA002840F0898195F859
:10E940002430012B00F0B0812A68744B744E186893
:10E95000514201F009F808F0BDFD30604FF400703D
:10E96000FBF76AFA002800F0978195F82530002B14
:10E9700040F0B98095F86930002B00F0B4806B68E6
:10E98000EE6F1B0293FBF6F6DFF89481D7F8009048
:10E99000D8F8000008F0B8FF33464946614AFBF753
:10E9A00027FE614B186000F097FE00283FF467AF28
:10E9B00000F018FF01287FF462AFD8F8000008F0DB
:10E9C000A3FF3B680B930A900EAB13E90F0000F016
:10E9D000A5FE54E7FBF714FAAAE7FBF78DFA06B297
:10E9E00094F84430012B95F8693004BF764236B272
:10E9F000002B7ED06B68EA6F1B0293FBF2F34A4F49
:10EA00004A4A3868DFF830813146FBF76BFE3B68D5
:10EA100020870028C8F80030C0F26181002384F804
:10EA20004430434F43483A68082331460093042357
:10EA300000F0DCFFB4F93830386083EAE37094F812
:10EA40004410A0EBE370FFF707FA00F045FE002842
:10EA500040F0E680FFF7A8F995F82530002B3BD170
:10EA600095F86930002B37D039686B68EA6F81EA16
:10EA7000E176A6EBE1761B0293FBF2F39E42D4BF54
:10EA80000026012631460120FBF7CAF93046FAF785
:10EA900089F995F86A30626913B3B5F86C3093421E
:10EAA00040F32181B5F86E105B1A934200F3C880E1
:10EAB000FFF760FEFCF7BCFA4FF40030FBF7BCF93F
:10EAC000002853D1FAF7C4F900287FF4DCAE4FF4E4
:10EAD0008070FFF7E3FAD6E639686B68AA6FC6E77D
:10EAE000B5F86C30DEE76B68AE6F1B0293FBF6F691
:10EAF0004AE76B68AA6F1B0293FBF2F37FE700BF44
:10EB0000D037FF1F7022FF1F0060034000800340CA
:10EB10003000FF1FD846FF1FC446FF1F3847FF1FA6
:10EB20000047FF1FA046FF1FD046FF1F0847FF1FDB
:10EB3000CC46FF1FB822FF1FC046FF1F4FF40070D6
:10EB4000FBF77AF900287FF4BBAE4FF40060FBF7C7
:10EB500073F9064600287FF4B3AE4FF48070FBF7DC
:10EB60006BF9002840F0E980824F75E70020FFF73D
:10EB7000F3FAA7E7DFF838B27F4EDFF838A2DFF804
:10EB80003892DFF824827B4F08A8FBF77DF9089ABA
:10EB90007A48BDF82430CBF8002079496A680068CB
:10EBA000ABF804300968BBF804E006901202A86FC5
:10EBB00092FBF0F273480792734AADF800E0DBF87D
:10EBC0000030059104900392CDF804A06F4A70497B
:10EBD00070480296FBF72CFEDAF80030B6F9001008
:10EBE000D9F80020C8F800304FF0080A02236A481C
:10EBF000CDF800A000F0FAFEB6F90230B6F9001028
:10EC0000C9F800003A686548CDF800A0194404230B
:10EC100000F0ECFE386000F05FFD00283FF41AAF12
:10EC200000F0E0FD00287FF415AFD8F800203B6825
:10EC30000B930A920EAB13E90F0000F06FFD09E78A
:10EC4000574B40229A604FF48020FBF7E1F82FE702
:10EC5000544A61682069FBF7A9FC494B186000F031
:10EC60003BFD00284FD123696168EA68591A81EA9F
:10EC7000E173A3EBE17393423FF761AE3B68AA688F
:10EC800083EAE371A1EBE37191423FF758AE4FF491
:10EC90008040FBF7B5F852E64FF48060FBF7CCF804
:10ECA00000287FF462AEEAE54FF48060FBF7C4F819
:10ECB000002836D14FF40070FBF7BEF800283FF46F
:10ECC0004DAE2F4B2F4ED3F80080306808F01CFE5D
:10ECD0004146FBF757FB08F0FDFB30603EE60123A1
:10ECE00084F844309DE62E4B40225A604FF4802039
:10ECF000FBF786F8DCE69E88764236B270E65E88E0
:10ED0000764236B26CE600F06DFD0228ABD1226986
:10ED100063680B930A920EAB13E90F0000F0FEFC40
:10ED2000A1E7174A2369116817486268154EFBF777
:10ED30006BFB08F0CFFB3060BCE714480D4F00F0D0
:10ED4000BFFF184800F0BCFF124800F0B9FF1048A0
:10ED500000F0B6FF0B4B144995F825000E60002219
:10ED60001A603E60FAF716FF104B4FF40072C3F8BA
:10ED700098206FE6CC46FF1F2C47FF1FC446FF1F9D
:10ED80003847FF1F0047FF1F7846FF1FA046FF1FA1
:10ED90008046FF1F0847FF1FBC22FF1FC022FF1F26
:10EDA000C0F00F40E046FF1FC046FF1F0080034039
:10EDB000D846FF1FD046FF1F3047FF1F684620F090
:10EDC00007018D4601B5F9F7DFFF044ABDE80140B0
:10EDD000136823F0400313608546704700600340CA
:10EDE000034B93F84230DB0701D5FEF7D5BE7047E1
:10EDF000D037FF1F034B93F842309B0701D5FEF736
:10EE0000E9BE7047D037FF1F074A92F85430D80741
:10EE100008D5064900204860590744BF23F0010384
:10EE200082F85430704700BFD037FF1F7022FF1F99
:10EE300008B5F9F7DDFF4FF48070BDE80840FFF733
:10EE40002DB900BF014B1868704700BFA046FF1FD7
:10EE5000014B9868704700BFA046FF1F014B186820
:10EE6000704700BF0847FF1F014B9868704700BFFD
:10EE70000847FF1F014B1868704700BF8046FF1FFF
:10EE8000014B9868704700BF8046FF1F014B5868D0
:10EE9000704700BFD037FF1F044A904298BF044A12
:10EEA00003469ABF5360012000207047905F010025
:10EEB000D037FF1F014B986B704700BFD037FF1F43
:10EEC000044A904298BF044A03469ABF93630120C4
:10EED00000207047905F0100D037FF1F014B93F86F
:10EEE00029007047D037FF1F831EFC2B02D9002357
:10EEF0001846704770B50E4C0E4D84F82900C0F3CB
:10EF00004F00FAF7D9FBE06908F0E0FA01460A4839
:10EF100008F0E8FB064694F8290008F0D7FA014605
:10EF2000304608F0DFFB01232860184670BD00BFA3
:10EF3000D037FF1F3000FF1F0050C3480030034B85
:10EF400018BF012083F82800704700BFD037FF1F8B
:10EF5000034B93F82800003018BF0120704700BF12
:10EF6000D037FF1F012898BF034A03469ABF82F893
:10EF70002E30012000207047D037FF1F014B93F83F
:10EF80002E007047D037FF1FB0F5803F0BD208B579
:10EF9000064BDA6BD863904203D0FFF7B1FB012038
:10EFA00008BD012008BD0020704700BFD037FF1FFB
:10EFB000014BD86B704700BFD037FF1FB0F5803FC3
:10EFC00038BF044A03463ABFA2F84030012000206F
:10EFD000704700BFD037FF1F014BB3F840007047A8
:10EFE000D037FF1F064B003093F82D2018BF0120AB
:10EFF000824283F82D0001D0FFF782BB704700BF2B
:10F00000D037FF1F034B93F82D00003018BF0120AD
:10F01000704700BFD037FF1F022898BF034A03463E
:10F020009ABF82F82C30012000207047D037FF1F94
:10F03000014B93F82C007047D037FF1F00F5433386
:10F04000054903F5A0738B4298BF044B02469ABF53
:10F050001A66012000207047801A0600D037FF1F73
:10F06000014B186E704700BFD037FF1F42F210727D
:10F07000904298BF034A03469ABF5385012000205F
:10F08000704700BFD037FF1F014BB3F92A0070470C
:10F09000D037FF1F831F032B00D930B9044A054B1B
:10F0A00082F825000120187370470020704700BFC8
:10F0B000D037FF1F7022FF1F014B93F825007047C8
:10F0C000D037FF1F094BB3F86630B3F5806F08D017
:10F0D000B3F5006F07D0B3F5007F0CBF022000200E
:10F0E0007047032070470120704700BFD037FF1FD3
:10F0F0000A2898BF034A03469ABF136201200020E2
:10F10000704700BFD037FF1F014B186A704700BF20
:10F11000D037FF1FB0F5803F38BF034A03463ABFE0
:10F120001363012000207047D037FF1F014B186B7D
:10F13000704700BFD037FF1FB0F5803F38BF034A8C
:10F1400003463ABF5363012000207047D037FF1FAA
:10F15000014B586B704700BFD037FF1F044A9042E5
:10F1600098BF044A03469ABF5361012000207047AC
:10F17000400D0300D037FF1F014B5869704700BF97
:10F18000D037FF1F044A904298BF044A03469ABFF3
:10F190001360012000207047400D0300D037FF1F8F
:10F1A000014B1868704700BFD037FF1F044A9042D8
:10F1B00098BF044A03469ABF13610120002070479C
:10F1C000400D0300D037FF1F014B1869704700BF87
:10F1D000D037FF1F1428F8B523D8134C134DE06126
:10F1E00008F074F901460646114808F07BFA074614
:10F1F00094F8290008F06AF90146384608F072FAD6
:10F20000314628600B4808F06DFA0646E06B08F0BE
:10F210005DF90146304608F065FA0123686018463A
:10F22000F8BD00231846F8BDD037FF1F3000FF1F80
:10F230000050C348007C9249014BD869704700BF19
:10F24000D037FF1FB0F5803F38BF034A03463ABFAF
:10F25000D364012000207047D037FF1F014BD86CCA
:10F26000704700BFD037FF1FB0F5803F38BF034A5B
:10F2700003463ABF1365012000207047D037FF1FB7
:10F28000014B186D704700BFD037FF1F012898BF92
:10F29000034A03469ABF82F82430012000207047B9
:10F2A000D037FF1F034B93F82400003018BF012014
:10F2B000704700BFD037FF1F044A904298BF044AEE
:10F2C00003469ABF9361012000207047A086010089
:10F2D000D037FF1F014B9869704700BFD037FF1F21
:10F2E000B0F5803F38BF034A03463ABF936401201C
:10F2F00000207047D037FF1F014B986C704700BF4C
:10F30000D037FF1F044A904298BF044A03469ABF71
:10F310009360012000207047400D0300D037FF1F8D
:10F32000014B9868704700BFD037FF1F044A9042D6
:10F3300098BF044A03469ABFD3600120002070475B
:10F34000A0860100D037FF1F014BD868704700BF6F
:10F35000D037FF1F064A92F8543020B923F001033A
:10F3600082F85430704743F0010382F854307047FC
:10F37000D037FF1F024B93F8540000F00100704794
:10F38000D037FF1F064A92F8543020B923F0040307
:10F3900082F85430704743F0040382F854307047C9
:10F3A000D037FF1F024B93F85400C0F38000704722
:10F3B000D037FF1F012898BF034A03469ABF82F83F
:10F3C0006A30012000207047D037FF1F014B93F8AF
:10F3D0006A007047D037FF1FA0F13202B2F5D77F25
:10F3E00098BF044A03469ABFA2F86C30012000205F
:10F3F000704700BFD037FF1F014BB3F86C00704758
:10F40000D037FF1F322898BF034A03469ABFA2F89D
:10F410006E30012000207047D037FF1F014BB3F83A
:10F420006E007047D037FF1F044A904298BF044ACD
:10F4300003469ABFD365012000207047E093040083
:10F44000D037FF1F014BD86D704700BFD037FF1F6B
:10F45000044A904298BF044A03469ABF936501202C
:10F460000020704780DF1710D037FF1F014B986DC9
:10F47000704700BFD037FF1F012898BF034A0346DB
:10F480009ABF82F86930012000207047D037FF1FF3
:10F49000034B93F86900003018BF0120704700BF8C
:10F4A000D037FF1F08B54FF6FE73984201D90020F0
:10F4B00008BD03460549064A08789BB21946A2F8DA
:10F4C0007030F9F739FD012008BD00BF1000FF1FA3
:10F4D000D037FF1F014BB3F870007047D037FF1FC4
:10F4E000B0F5805F01D30020704708B5034BA3F847
:10F4F0007200F9F7F3FA012008BD00BFD037FF1FF3
:10F50000014BB3F872007047D037FF1F014B98676B
:10F5100001207047D037FF1F014B986F704700BF25
:10F52000D037FF1FB1F5803F0AD208B50E4A1278D6
:10F53000824210D00D4A1278824203D0002008BDCA
:10F54000002070478BB20A4A1946A2F87630F9F7C4
:10F55000F3FC012008BD8BB2054A1946A2F87430AD
:10F56000F9F7EAFC012008BD1100FF1F1200FF1F80
:10F57000D037FF1F084B1B78834208D0074B1B78FE
:10F58000834206BF064BB3F8760000207047044B59
:10F59000B3F87400704700BF1100FF1F1200FF1F77
:10F5A000D037FF1F014BD86701207047D037FF1FAE
:10F5B000014BD86F704700BFD037FF1F014B186851
:10F5C000704700BFE085FF1F014B1868704700BF00
:10F5D000D885FF1F014B1868704700BFD485FF1FF7
:10F5E000014B1868704700BFCC85FF1F014B18689E
:10F5F000704700BFDC85FF1F014B1868704700BFD4
:10F60000C085FF1F014B1868704700BFC885FF1FEA
:10F61000014B1868704700BFC485FF1F014B186875
:10F62000704700BFD085FF1F014B1868704700BFAF
:10F630003C47FF1F014B1860704700BFE085FF1F6C
:10F64000014B1860704700BFD885FF1F014B186041
:10F65000704700BFD485FF1F014B1860704700BF83
:10F66000CC85FF1F014B1860704700BFDC85FF1F72
:10F67000014B1860704700BFC085FF1F014B186029
:10F68000704700BFC885FF1F014B1860704700BF5F
:10F69000C485FF1F014B1860704700BFD085FF1F56
:10F6A000014B1860704700BF3C47FF1F054B10B46B
:10F6B0000022012418705C721A725960DA6010BC62
:10F6C000704700BFC822FF1F024B00225A721A72F5
:10F6D000DA607047C822FF1F014B187A704700BFDD
:10F6E000C822FF1F014B587A704700BFC822FF1F76
:10F6F000014BD868704700BFC822FF1F064BDA686D
:10F7000001320021B2F57A7FDA60196102D15972B3
:10F710001972D960704700BFC822FF1FF0B4154DA1
:10F72000154E2C693668013484B004AFB44207E941
:10F730000F002C6117DB2B7AABB1EB68B3F57A7F46
:10F7400011DA1F010D4A009ED65101333A44019C43
:10F7500002980399EB600026B3F57A7F54609060BD
:10F76000D1602E6102D004B0F0BC70476E722E7270
:10F77000EE60F8E7C822FF1F4000FF1F4047FF1F51
:10F780004FF47A70704700BF4FF47A50704700BF53
:10F7900004207047B0F57A7F07DA032905D801EB1A
:10F7A0008001034B53F8210070470020704700BFD1
:10F7B0004047FF1F032803D8DFE800F0020A060EC7
:10F7C000074B00225A617047054B02225A6170476D
:10F7D000034B01225A617047014B03225A61704763
:10F7E000C822FF1F014B5869704700BFC822FF1F86
:10F7F000014B1860704700BF4000FF1F014B1868A5
:10F80000704700BF4000FF1F10B5144B1C78062C3A
:10F8100010D8DFE804F00704170C1B1F1300596809
:10F82000914207DD01221A7200225A7210BD5A68F5
:10F830008A42F7DC1A7A012AF6D010BD5A68904243
:10F84000F0DCF7E759688A42ECDCF3E75A6891424A
:10F85000E8DCEFE75A688242E4DCEBE7C822FF1FEE
:10F86000B0F5803F1DDBB0F1807F33DBB0F1805F0E
:10F870003BDAB0F1806F3A4A4FDB0315D35C9B0152
:10F880005A1C90FBF3F31A445210531C90FBF2F2F3
:10F8900013445B1003FB03F2904209DA013B184664
:10F8A0007047FF2806DC002857DB2D4B1B5C1B092B
:10F8B00018467047B0F5805F294A26DBB0F5804FC7
:10F8C00041DB0312D35C013303FB03F29042E5DB1F
:10F8D00018467047B0F5801F214A0FDBB0F5800F46
:10F8E00029DB0314D25C1201CFE7B0F1804F18DBA3
:10F8F0001C4B98422CDD4FF6FF73D9E7B0F5802FF3
:10F900001DDB0313D25C9200BFE7B0F5806F0DDB07
:10F910000311D35C9B080133D6E78314D35C5B01EE
:10F92000AEE70F4A8315D35CDB01A9E78310D35CF4
:10F93000DB080133C8E78313D25CD200A5E783124A
:10F94000D25C5200A1E78311D35C5B080133BBE7B3
:10F95000034A0316D35C1B0292E74FF0FF33A7E77D
:10F96000008401000080FE7F904203DC8842B8BF23
:10F970000846704710467047904203D8884238BF07
:10F98000084670471046704730B5DDE903458442AC
:10F9900075EB010E07DB904271EB030400DB30BD19
:10F9A0001046194630BD2046294630BD70B5144674
:10F9B0000E4607F08FFD0546204607F087FD0446FA
:10F9C0000146284607F08EFE0146284607F0CCFC8B
:10F9D0000546304607F07EFD214607F083FE0146CE
:10F9E000284607F0C3FC07F08FFF70BD30B4029CBF
:10F9F0000568E31A8A1A02FA03F32B44036043FAF8
:10FA000004F030BC704700BF44F6E612030C13FB51
:10FA100002F3002B00B2B8BF03F5FF4310FB02F264
:10FA2000B8BF7F33002A84B0B8BF02F5FF42C3F3EA
:10FA3000CF33B8BF7F32ADF80C0003EBE232134492
:10FA4000BDF80C205B4200209BB262F30F0063F311
:10FA50001F4004B0704700BFB0F90210B0F9003089
:10FA600010B401FB01F20F4C03FB0322A24216D992
:10FA7000120E3A3A0C4C34F8122002FB03F3002B1E
:10FA800002FB01F2BCBF03F5FF437F33002ABCBF7A
:10FA900002F5FF427F32DB13D2130380428010BC99
:10FAA000704700BF0044FA3A008501001F49B0F9D1
:10FAB0000020B1F90030B1F9021010B4B0F90240E1
:10FAC00002FB03F00028B8BF00F5FF4002FB01F283
:10FAD00004FB01F1B8BF7F300029B8BF01F5FF4139
:10FAE00003FB04F3B8BF7F31002B83B0B8BF03F52D
:10FAF000FF434FEAE03000EBE131B8BF7F33002A2B
:10FB0000B8BF02F5FF42ADF80410B8BF7F32BDF8B0
:10FB10000410DB13A3EBD23300209BB261F30F0080
:10FB200063F31F4003B010BC704700BFE022FF1F0B
:10FB3000A0F50040C0F3891000F44073B3F5807F56
:10FB400082B03FD029D9B3F5007F19D0B3F5407FFB
:10FB500035D1244BC0B203EB4002400080F4FF706B
:10FB6000B2F88C2018445242B0F98C3012B292B2E2
:10FB700000209BB262F30F0063F31F4002B0704796
:10FB8000C0B2184A430083F4FF73134402EB4000F1
:10FB9000B3F98C20B0F98C30E9E783B9C0B2114ACF
:10FBA000430083F4FF73134402EB4000B3F88C204E
:10FBB000B0F88C3052425B4212B21BB2D7E700233E
:10FBC0001A46D4E7C0B2074A430083F4FF731344D4
:10FBD00002EB4000B3F88C30B0F98C205B421BB2D2
:10FBE000C5E700BF0085010010B5044682B0084695
:10FBF000FFF79EFF1C4AB4F90030106002B203FB0D
:10FC000002F1B4F9024000294FEA2040B8BF01F5E3
:10FC1000FF4103FB00F304FB00F0B8BF7F31002875
:10FC2000BCBF00F5FF407F30002BB8BF03F5FF439A
:10FC300002FB04F24FEAE131A1EBE030B8BF7F33C1
:10FC4000002AADF80400BCBF02F5FF427F32BDF8C8
:10FC50000410DB1303EBD23300209BB261F30F00DF
:10FC600063F31F4002B010BDE022FF1F032923D819
:10FC7000DFE801F01C140C02104B400080F4FF7010
:10FC80001844B0F88C00404200B270470B4B03EBB5
:10FC90004000B0F88C00404200B27047074B400073
:10FCA00080F4FF701844B0F98C007047034B03EBED
:10FCB0004000B0F98C0070470020704700850100BB
:10FCC00000230022C0E90223002303608361704700
:10FCD00070B5144C2368C31A002BB8BF5B42632B6A
:10FCE0001EDD0546606800EB80004000FFF7A2FCC7
:10FCF000A06800EB8000002640006660FFF7A0FCD3
:10FD0000E068A66000EB80004000FFF79FFC2069E0
:10FD1000E66000EB80004000FFF79EFC2661256056
:10FD200070BD00BFE422FF1F024A536801335360D5
:10FD3000704700BFE422FF1F024A936801339360BB
:10FD4000704700BFE422FF1F024AD3680133D3602B
:10FD5000704700BFE422FF1F024BD86800EB800011
:10FD600040007047E422FF1F024A13690133136108
:10FD7000704700BFE422FF1F024B186900EB8000B0
:10FD800040007047E422FF1F124B1A88013A12B25A
:10FD9000002A02DA00231846704770B45E6800211A
:10FDA000541804EBD474641004EB440506EB85038B
:10FDB00036F82550854209D004F1FF3304F10104DF
:10FDC0008CBF1AB221B28A42EADA0023184670BC0C
:10FDD000704700BF3C23FF1FCB071DD5002A18BF6B
:10FDE00001301F4B00EBC00040009A68135A591EA7
:10FDF00010441D2912D8DFE801F01E1E201C1E2011
:10FE00001C1C2222111111111111111111111111AA
:10FE1000111111111111111E1044E2E71E2B17D8F8
:10FE20000120104A00FA03F3134205D113F4C87FEE
:10FE300010D00420704701207047022070470379DA
:10FE4000C289022B0CBF084B084B53F822007047A5
:10FE50000020704713F0480F0CBF002002207047AD
:10FE60003C23FF1F26000040A014FF1FA48D0100AB
:10FE7000F8B50C4615461E46FFF786FF00283DD014
:10FE80000279A242034602D84FF48170F8BD027A8B
:10FE9000D20736D4B0F802C0BD4904EB0C0202EB25
:10FEA000C20288685200811891F804E0CF88BEF140
:10FEB000000F39D1835A1E2B3DD8DFE813F0230100
:10FEC0004701410161015A0154014D0134012901E9
:10FED0003C003C003C003C003C003C003C003C0042
:10FEE0003C003C003C003C003C003C003C003C0032
:10FEF0003C003C003C003C003C003B0140F2011057
:10FF0000F8BD4288A249002C0CBF1346531C03EBDA
:10FF1000C30388685B00C11891F804E0CF88BEF184
:10FF2000000F0BD1C35AC6E7BEF1020F00F0A48048
:10FF3000BEF1010F18D000232B60A5E7002C0CBFE9
:10FF40001146511C01EBC101490043181B79022BDA
:10FF50004ED0002C0CBF1446541C04EBC4046200A9
:10FF600083181B79012BE6D1835A1E2BE3D801A2FB
:10FF700052F823F005010100570201004B02010075
:10FF80003D0201002F020100370301002903010097
:10FF90001B0301000D030100FD020100ED02010041
:10FFA00037FF000037FF000037FF000037FF000079
:10FFB00037FF000037FF000037FF000037FF000069
:10FFC00037FF000037FF000037FF000037FF000059
:10FFD00037FF000037FF000037FF000037FF000049
:10FFE00037FF000037FF000037FF0000E10201008B
:10FFF000435A1E2B9FD801A252F823F0050101009D
:020000021000EC
:100000000F0201000B0201000702010003020100C0
:10001000FF010100E7010100E3010100CB01010044
:1000200037FF000037FF000037FF000037FF0000F8
:1000300037FF000037FF000037FF000037FF0000E8
:1000400037FF000037FF000037FF000037FF0000D8
:1000500037FF000037FF000037FF000037FF0000C8
:1000600037FF000037FF000037FF000037FF0000B8
:1000700037FF0000B9010100825A1E2A3FF65BAF2C
:1000800001A151F822F000BF05010100C5020100E5
:10009000B7020100A90201009B0201008D020100CC
:1000A0007F02010071020100630201002B020100C6
:1000B0001302010037FF000037FF000037FF000088
:1000C00037FF000037FF000037FF000037FF000058
:1000D00037FF000037FF000037FF000037FF000048
:1000E00037FF000037FF000037FF000037FF000038
:1000F00037FF000037FF000037FF000037FF000028
:10010000D302010000232B6040F215203360F8BDBC
:10011000204B042203EB87032B603260002B3FF45B
:10012000B3AE0020F8BD1C4B042203EB87032B6009
:100130003260F3E7194B01223B442B603260EDE75C
:10014000174B01223B442B603260E7E7154B01223D
:100150003B442B603260E1E7134B022203EB470381
:100160002B603260DAE7114B01223B442B60326096
:10017000D4E70F4B042203EB87032B603260CDE7FB
:100180000C4B022203EB47032B603260C6E700BF33
:100190003C23FF1F2C23FF1FA014FF1F2423FF1F3E
:1001A0003823FF1F2823FF1F2815FF1F4815FF1F97
:1001B0003023FF1F3423FF1F624B53F82730013CCD
:1001C000234401222B603260A8E75F4B53F82730AD
:1001D00004F18044013C03EB840304222B60326071
:1001E0009CE75A4BF2E75A4B53F8273004F100448E
:1001F000013C03EB440302222B6032608EE7554B37
:10020000DBE7554BE2E7554BEEE7554BD5E7554B52
:10021000D3E7554A52F827702F60197A2246604674
:10022000FFF7DAFD3B46306078E7504AF2E7504B83
:10023000042203EB87032B6032606FE74D4B0222F1
:1002400003EB47032B60326068E74B4B01223B44D2
:100250002B60326062E7494B01223B442B603260E5
:100260005CE7394B042253F827302B60326055E7A6
:10027000364B042253F827302B6032604EE7344B64
:10028000022253F827302B60326047E7314B0122BE
:1002900053F827302B60326040E72F4B042253F88D
:1002A00027302B60326039E72C4B022253F827307D
:1002B0002B60326032E72A4B012253F827302B6043
:1002C00032602BE7274B012253F827302B60326036
:1002D00024E71C4B012253F827302B6032601DE7C6
:1002E000274B01223B442B60326017E7254B53F824
:1002F0002700286006F074FB306012E7224B53F8A9
:100300002700286006F06CFB30600AE71F4B0422D0
:1003100003EB87032B60326000E71D4B042203EBE5
:1003200087032B603260F9E61A4B022203EB470386
:100330002B603260F2E6184B01223B442B603260A6
:10034000ECE600BFE88B0100F08B0100F48B0100AC
:10035000748C0100B08C0100D48C0100548D01001C
:100360007C8D0100EC8B0100D88B0100DC8B01003F
:10037000448E0100648E0100788E01009C8D010086
:10038000988D0100888D01008C8D0100A08D0100E9
:10039000A48D0100188E0100348E01001E2807D89C
:1003A00001230A4A03FA00F0104203D008207047E4
:1003B0000020704710F4C87F01D02020704710F053
:1003C000480F0CBF00201020704700BF26000040DF
:1003D00038B50D461446FFF7D7FCC0B1037A184A6A
:1003E00013F0010F438813D15919936801EBC10130
:1003F00003EB41014888082C06D8DFE804F0081C0C
:100400001C0518050505140020F03F0080B238BD1A
:10041000002D0CBF1946591C936801EBC10103EB79
:1004200041014888E7E720F01B0080B238BD20F08A
:100430002D0080B238BD20F0360080B238BD00BF3C
:100440003C23FF1F2DE9F04182B0154601AA064664
:100450000F469846FFF70CFD044618B1204602B03F
:10046000BDE8F08100F0A6FD394602463046FFF7B0
:10047000AFFFC30405D4019B2B60204602B0BDE84A
:10048000F081D8F800200199284607F00FFDE5E734
:100490002DE9F04383B000240E469146984601941E
:1004A0000746FFF771FC48B10379B34204460BD805
:1004B0004FF48175284603B0BDE8F08340F2011582
:1004C000284603B0BDE8F08301AB6A4631463846A2
:1004D000FFF7CEFC05460028ECD100F06BFD31465D
:1004E00002463846FFF774FFC30409D43246217A26
:1004F0006088FFF771FC804523D940F20315D9E7E6
:10050000237A194A13F0010F638822D0002E0CBF02
:100510001E465E1C06EBC606936833F816301E2B8B
:1005200015D80122114902FA03F30B4218D113F432
:10053000C87F17D113F0480F0CBF00230223984542
:10054000DBD142464946009807F0B0FCB2E70023F1
:10055000F5E71E4406EBC606936833F81630DEE76F
:100560001346ECE70423EAE73C23FF1F2600004084
:1005700070B50C4615461E46FFF706FC40B30379DE
:10058000A34203D84FF48173184670BD037A4188A3
:1005900013F0010F2A4B1FD10C4404EBC4049B68D9
:1005A00064001A191B5B1289013B1D2B45D8DFE83B
:1005B00003F042403E3C3A3230281F444444444415
:1005C0004444444444444444444444444444441817
:1005D00040F20113184670BD002C0CBF0C464C1C99
:1005E000DBE7184B1A4401212A6000233160CBE776
:1005F000154B53F82200286006F0F2F90023306012
:10060000C2E7124B03EB820204212A60002331600F
:10061000BAE70F4BF6E70F4B03EB420202212A60C9
:1006200000233160B0E70C4BDCE70C4BEAE70C4BE6
:10063000F2E70C4BD6E70C4BD4E700232B60A3E783
:100640003C23FF1F988D01008C8D0100A08D0100BF
:10065000A48D0100188E0100348E0100448E01002B
:10066000648E0100788E01009C8D010038B50D4626
:100670001446FFF789FB50B14289074B53F822001B
:10068000286006F0ADF900232080184638BD40F2FE
:100690000113184638BD00BFA48A010070B50E468C
:1006A00015461C46FFF770FB08B3037A124A13F095
:1006B000010F438810D19919936801EBC10103EB35
:1006C00041010A8A0D4B53F82200286006F088F990
:1006D00000232080184670BD002E0CBF1946591CFF
:1006E000936801EBC10103EB41010A8AEAE740F29A
:1006F00001132860184670BD3C23FF1F8C87010042
:1007000001282DE9F04F59D0DFF85CB1BBF80C801F
:10071000BBF800A0D04543D2DBF80430DBF808601A
:1007200008EB480903EB89094FF6FF7C99F804E0D0
:10073000BEF1000F2CD099F80870B9F802500020D3
:1007400007F00107044609E001306145528883B291
:1007500019D031EA020216D0734518D282B2002AAB
:100760000CBF2A466A1C2B1802EBC20203EBC30320
:1007700006EB420206EB4303002FE5D10130614551
:100780005A8883B2E5D101347345A4B2E6D364B983
:1007900008F101081FFA88F8D04509F10C09C5D104
:1007A0004FF000084046BDE8F08F08F10108ABF8B3
:1007B0000C80B9F800804046BDE8F08F4FF6FF731B
:1007C000DFF8A4B09942BBF8008047D0B8F1000F21
:1007D00044D008F1FF391FFA89F909F10109DBF862
:1007E00004C0DBF8086009EB49090CEB89094FF0FC
:1007F00000089CF804E0BEF1000F2BD09CF8080024
:10080000BCF80250002400F0010027460BE052889B
:1008100031EA020204F1010408BF0137A3B208BFA4
:10082000BFB2734511D2A2B2002A0CBF2A466A1C7D
:100830002B1902EBC20203EBC30306EB420206EBE9
:1008400043030028E3D15A88E2E71FB108F1010809
:100850001FFA88F80CF10C0CE145CAD10023ABF863
:100860000C304046BDE8F08F3C23FF1F70B50E46AC
:1008700015461C46FFF788FA40B1C288437932809A
:100880002B700279013A2270002070BD40F20110F5
:1008900070BD00BF70B50C4615461E46FFF774FAD2
:1008A00028B30379A34202D84FF4817070BD037A54
:1008B000184913F0010F43881CD1234403EBC302F2
:1008C0008B6833F812202A80027A4188D2071AD521
:1008D000002C0CBF0C464C1C04EBC40403EB44047A
:1008E000638833802B88002BDED0002070BD40F25F
:1008F000011070BD002C18BF013303EBC3028B68DD
:1009000033F81220DFE70C4404EBC40403EB440487
:100910006388E6E73C23FF1F30B5A0F5E052103AAC
:10092000032A83B01D4603D8E9B9002003B030BDC7
:1009300000F47F43B3F5B05F044602D0B3F5D05F57
:10094000F3D10029F1D0002DEFD101AB294620468B
:100950000DF10302FFF776FD9DF80330002BE4D084
:100960004FF48570E2E701AB0DF103020021FFF7C0
:1009700069FD9DF80330002BD7D0002DD5D140F272
:100980000910D3E7044A054B10880549054A188029
:1009900099605A6000207047C801FF1F3C23FF1F69
:1009A0005C05FF1FCC01FF1F2DE9F0415A4E8768FF
:1009B00032783B7A012A054603F0E0012DD0092A5E
:1009C00002D00020BDE8F081B9BB4288092A40F27C
:1009D0008780C3F34201033A521A746892B2D94332
:1009E000A242C9B2C3F3001353DC4C4F97F800E0A6
:1009F0009E4508D0B2EB040E01F0010118BF4FF084
:100A0000010E8E457FD00A240022284634701146FC
:100A1000434BBDE8F04101F0DFBF602931D8202908
:100A20001ED051BB6B88092B33D80B23284633705B
:100A30000821BDE8F04100F0ABBF602933D1428806
:100A4000092A4DD9354A1178C3F300139942DAD0F7
:100A5000072471683470BDE8F041137002F044BBA4
:100A600013F00204438827D00A2BDED1022333700F
:100A70001146BDE8F04101F0FBBF40293AD06029A2
:100A8000D0D00B23284633700521BDE8F04100F09B
:100A90007FBF0A240022284634701146214BBDE84E
:100AA000F04101F099BF0B220023327073600521E1
:100AB000BDE8F04100F06CBF092BB6D917490323FC
:100AC00007F10C0033700A7001F036F86B880A3BAE
:100AD000C31A214628467360BDE8F04101F0C8BF43
:100AE0000B2200232846327073600821BDE8F041D4
:100AF00000F04EBF43880A2B97D106233370BDE820
:100B0000F04102F007BBA21A042172603B70317001
:100B1000BDE8F04102F028BB4C23FF1F5F15FF1F0B
:100B20000000030501000405034B1A7812B90121E6
:100B30005A601970704700BF4C23FF1F0C490B7897
:100B4000013BDBB20A2B0FD8012202FA03F340F279
:100B500001121A4009D113F4C06004D113F0FE0F42
:100B600002D0087070470A70704700230B707047FE
:100B70004C23FF1F0D4B1A780A2A02D00B2A02D0F1
:100B800070475A6812B901221A707047B2F1004FCB
:100B900002D009221A7070479A681AB901215A6066
:100BA0001970704708221A7001F0FABE4C23FF1F1B
:100BB00010B504468068063000F0BCFF2E4A13785A
:100BC000012B00F4704003D0092B24D0022010BD6B
:100BD000B0F5005F37D0B0F5004F07D020460B23AB
:100BE0000521BDE81040137000F0D2BEA3681B7A47
:100BF00003F07F03012B2AD0032B19D0052BEDD155
:100C000063880A2B2ED020460B230821BDE8104014
:100C1000137000F0BDBEB0F5005F14D020460B2469
:100C2000002314700521BDE81040536000F0B0BEF1
:100C30006388082BE7D120460021BDE810401370DF
:100C4000916001F067BC2046BDE81040ACE66388C7
:100C5000082BD8D120460021BDE8104013709160C8
:100C600001F030BB204600210823BDE81040916010
:100C7000137001F011BD00BF4C23FF1F154B68B16D
:100C80001A78062A0DD0072A12D0082A01D1062880
:100C900017D0082810D00A221A70704701221A7043
:100CA00070470428F5D10C4A596001211170F2E710
:100CB0000528EED15960EEE700225A600A221A7028
:100CC00070470029CCBF4FF00042002299605A6063
:100CD000E1E700BF4C23FF1F5F15FF1F044B1B788C
:100CE00003F0F703012B14BF02200020704700BF60
:100CF0004C23FF1F0349044A044B00200870108056
:100D0000188070475823FF1FE485FF1FE685FF1FEB
:100D100010B54FF4186082B002F0D6FA40F20133F9
:100D20001840B0F5407F32D01A4B00241C7001945B
:100D300002F098FC01280ABF22230123ADF800002D
:100D4000ADF802306A464FF002034FF0010141F660
:100D5000324018BFADF80040FFF79AFB01AA042308
:100D6000022141F63240FFF793FB02230DEB030211
:100D7000012141F63340FFF78BFB01AA0423022136
:100D800041F63340FFF784FB022002B010BD002083
:100D900002B010BD5823FF1F0220704738B50C4B1E
:100DA0001B784BB10B4A13889BB23BB10A4C23888A
:100DB00000250A2B158003D8012038BD002038BD3E
:100DC00000F0F8F80828F9D02580012038BD00BFD0
:100DD0005823FF1FE485FF1FE685FF1F704700BFF4
:100DE000024B1A1D1A605A64002070475C23FF1FD3
:100DF000F0B51C4A91F800E013684F788E78CD78F2
:100E00000C7983B0ADF80000506C8DF802E0191A2F
:100E10003F298DF803708DF804608DF805508DF82A
:100E2000064016DC92F84810012910D00E49581AD5
:100E30003F2812DC6C4603CC0C4C1860012003F1F7
:100E40000805207000205960156003B0F0BD834292
:100E5000ECD140F2092003B0F0BD01200B4682F82E
:100E60004800E7E75C23FF1F6023FF1FE985FF1FA2
:100E7000F0B587B0FFF732FF18B10124204607B064
:100E8000F0BD01A800F0FEFC18B10224204607B016
:100E9000F0BD314D2A686B6CD11A3F293CDD2F4AD9
:100EA000991A3F2904DD00216A64134685F8481029
:100EB000019A18685968946800260A2704AB03C38E
:100EC00057809680A01D96714FF4805100F036FE39
:100ED000019BBDF810109868083000F02FFE3146D5
:100EE00002AB03AA41F20100FEF7C2FF0198039A88
:100EF000836812789A7206AB826853F8061DC2F8AE
:100F00000B101B79D373032100F0D4FC044670B19D
:100F1000019B02241E70B1E79A42C0D195F8482087
:100F2000002ABCD1019B40F203241A70A6E70146B7
:100F30000720FFF7A3FE6B6C2A680833D11A3F29FC
:100F40006B649BDC9A4299D195F84830002B95D17F
:100F5000034B1C7092E700BF5C23FF1F6023FF1F41
:100F6000E985FF1F70B50E4C10F010030D4600F020
:100F70000F06218018BF012301464FF49870E370DB
:100F8000A67002F0C7F929464FF49A7002F0C2F930
:100F90002A46E1783046BDE8704005F021BC00BF2C
:100FA000A623FF1F0123024A184600219370D9E7A8
:100FB000A623FF1F014B9878704700BFA623FF1F91
:100FC000014B1888704700BFA623FF1F10B5194CAE
:100FD000A378A080013B072B2AD8DFE803F0211972
:100FE00029112929290414230120E38000F026FE79
:100FF000A088E38801461846FFF7B4FF002010BD23
:10100000142301461846E380FFF7ACFF002010BD13
:10101000122301461846E380FFF7A4FF002010BD0D
:10102000112301461846E380FFF79CFF002010BD06
:10103000022010BDA623FF1FF8B588B1A34CA378EA
:10104000013B0546072B08D8DFE803F004380726E4
:1010500007070741012D00F0078102263046F8BD41
:101060009A4C4FF4907002F02FF9A378013B072BB4
:10107000F3D801A252F823F0F31001006911010026
:101080005B100100431101005B1001005B100100C7
:101090005B10010019110100012800F07F81022D71
:1010A000DBD1E378002BD8D128461B221423A28061
:1010B000E38002F093F9E088A1883DE00128CCD1DB
:1010C000E578002D00F04481002EC7D132E0012DDB
:1010D00000F04D81022DC0D1E378002BBDD11B2241
:1010E00014230120A280E38000F0A8FDE088A188FD
:1010F00022E010F010014AD000F00F00013807285C
:1011000000F21C81DFE810F09B00A500A000770032
:101110001A011A011A017700E37800F00F00002B82
:101120004ED0022800F0D480042800F05881012815
:1011300000F04881E088A1880026FFF713FF3046C1
:10114000F8BD10F0100349D000F00F000138072857
:1011500000F2F980DFE810F09A0091008C00B000F6
:10116000F700F700F700A50010F010031BD000F007
:101170000F000138072800F2DB80DFE810F04200A2
:1011800050004B005500D900D900D9004B00E3783E
:1011900000F00F00002BB1D0012852D0112021887F
:1011A000E080A180C8E7E27800F00F00002AE0D0DC
:1011B000012800F0528112202188E080A180BBE745
:1011C000431E072B00F2D180DFE813F09A008E0057
:1011D000AB00A100CF00CF00CF00AD00E27800F05F
:1011E0000F00002AB2D0012800F03E81142021888F
:1011F000E080A180A0E711231946A380E380184670
:101200009AE701220023E280A38000F029FBE08816
:10121000A18891E711211220A180E0808CE70220B3
:101220000021E080A18087E7032000F021FD002855
:1012300000F0E8801E211220A180E0807CE70120E0
:101240000021E080A18077E713211120A180E080B8
:1012500072E7022000F0A6FA002800F0F6801621BE
:101260001120A180E08067E702F0CCF90226F5E6C4
:1012700011211420A180E0805EE702220023E28099
:10128000A38000F0EBFCE088A18855E70122002351
:10129000E280A38000F0E4FA00F0E0FCE088A1889E
:1012A0004AE7637A002B00F0A480FFF777FD00285F
:1012B00040F09F800126D1E6042200230220E28034
:1012C000A38002F07DF8E088A18835E7A623FF1F00
:1012D0002388A38001201223E38000F0AFFC00F0FC
:1012E000BDFCE088A18827E702220023E280A380DA
:1012F00000F0B4FC012000F0A1FCE088A1881BE70D
:1013000001250023E580A38000F0AAFAF0E700237E
:1013100004221846A380E28000F090FCE088A188B7
:101320000AE71122DCE608230021E380A18003E71D
:1013300012231946A380E3801846FDE612211120EE
:10134000A180E080F8E612211420A180E080F3E67D
:10135000022000F027FA002840F0B680022602F0B2
:1013600051F9002E7FF47AAEE4E61222B8E6E7786F
:10137000002F7FF4A9AE022000F014FA06460028E0
:101380004AD0162211232846A280E3803E4600F070
:1013900055FC00F063FC00F063FAE0E7E578002D0F
:1013A0007FF4C8AE022000F0FDF90646002841D0C7
:1013B00016221123A280E3802E4600F04FFC00F09D
:1013C0004FFACCE72388A3801123E38000F036FC9A
:1013D00000F044FC00F044FAE088A188ACE62388E1
:1013E000A38001201423E38000F028FCE088A1887A
:1013F000A2E608220023E280A38000F095FDE088A9
:10140000A18899E6022000F033FC002843D01D217A
:101410001220A180E0808FE6032000F029FC28B391
:101420001E221223A280E38000F018FC284600F060
:1014300005FC94E7032000F01BFCF8B11E221223E8
:10144000A280E38000F00AFC89E70223A080E38009
:1014500000F0EAF9E088A1886EE6E080A38000F061
:10146000FFF9E088A18867E6E08012E7022000F03B
:10147000FFFB00283FF472AF1D22D2E7022000F0EC
:10148000F7FB00283FF46AAF1D221223A280E380FD
:1014900000F0E4FB63E7FFF73BFC10B9FFF77CFCCF
:1014A000D0B9FFF735FC08B1237AABB9FFF730FCB0
:1014B000B8B90123637204220023E280A38000F004
:1014C00081FDE088A18837E6162211232E46A280EE
:1014D000E38000F0C5F942E736211220A180E080C8
:1014E0002AE600236372E6E710B5FFF74BFA0446DD
:1014F00008B1204610BD01F029FF00F039F904467B
:101500000028F6D1FFF74EFDFFF76AFC04460028DD
:10151000EFD14FF4A77001F0D7FEC30701D5022425
:10152000E7E7044B21464FF401701C6001F0FEFE1A
:10153000DFE700BFB023FF1F044A136823EA00035C
:1015400019464FF40170136001F0F0BEB023FF1F85
:1015500070B502F087F806464FF4087001F0C2FE3D
:10156000514D6C6810B9002C00F08A80044361066C
:101570002BD42B7A012B00F08E80E10774D4A205C6
:101580003AD4E30544D460054ED4022E55D0E20689
:1015900060D4464C4FF4887001F096FE2388834255
:1015A000054602D005F046F92580414B1A783AB934
:1015B000404B1B7803B970BDBDE87040FFF758BCC5
:1015C00000221A7002F0B0F8F2E74FF4886001F0E0
:1015D0007BFEC2072B7ACDD4002BCBD101232B72FB
:1015E00005F026F90028C4D1FFF7E4FC0828C0D193
:1015F0000220FFF721FDBCE700F092F96B6801289B
:101600000CBF43F4007323F400736B60E305BAD599
:1016100000F0F0F96B6801280CBF43F4807323F4E9
:10162000807360056B60B0D5022001F075FF012E5C
:1016300024F4806405D0022EA9D12105A7D524F475
:10164000006405F0EBF80128A1D1032001F064FF4C
:10165000E2069ED5FFF7B4FC00289AD101F0DEFF28
:101660000120FFF7E9FC94E70020FFF7E5FC6B6839
:1016700001280CBF43F0010323F001036B607EE7F8
:1016800040F6050001F012FE030782D56B6843F4B3
:1016900080736B607DE74FF4886001F015FEC00732
:1016A00044BF00232B7268E7B023FF1F6015FF1FA4
:1016B0002536FF1FE985FF1F2DE9F04182B0002686
:1016C0008DF80760C0B1022304460370012001F0C9
:1016D00093FE8046012001F0A7FE0E4A638815683C
:1016E000A1689C1DA4B245440746224628463346BD
:1016F00001F028FEA74202D802B0BDE8F081781EB2
:101700002844334601220DF1070101F01BFE02B00F
:10171000BDE8F081EC85FF1F38B5044601200D4679
:1017200001F082FE63885A1D824202DB40F20220F1
:1017300038BDA2680D4913701B0A5370A288A068B7
:101740000B788270120AC270A268A0791071072B00
:10175000A26845EA03151ABF0133DBB20123204614
:1017600055710B70FFF7A8FF002038BD6215FF1FF1
:1017700070B40A4B0A4AFF21002003F1280603F245
:10178000EA5503F6AC345170DE609D615C621870FE
:1017900018711874187770BC704700BFBC23FF1F06
:1017A0006215FF1F0238012801D90220704708B5D1
:1017B000002001F039FE21282FD940F6060001F063
:1017C00075FDC2072CD5002001F016FEB0F5805F34
:1017D0001AD3012001F028FE21281ED940F60E0060
:1017E00001F064FDC3071BD5012001F005FEB0F533
:1017F000805F09D3002001F02FFE012001F02CFEB4
:10180000002001F04DFE10B140F20D2008BD012076
:1018100001F046FE0028F7D108BD40F20B2008BDBC
:101820004FF4037008BD00BF10B50B4C2378012B9B
:1018300010D00023094A23711846FF21237423770F
:10184000517001F0BDFD012001F0BAFD01232370AC
:10185000FFF76AF9002010BDBC23FF1F6215FF1FB0
:1018600010B5074C23784BB1FFF768F9002001F061
:10187000B5FD012001F0B2FD0023237010BD00BFB3
:10188000BC23FF1F0A4A137C63B1137F23B10023DB
:101890000360022318467047012102F81C1F0260F2
:1018A00018467047012102F8101F02601846704761
:1018B000BC23FF1F064B1B7813B94FF40070704711
:1018C0000378012B02D040F20120704724E700BFCB
:1018D000BC23FF1F10B5114C237C032B1AD0237F90
:1018E000032B00D010BD012304F81C3F012140F65A
:1018F0000F0001F003FD40F60D0001F0D7FC10F0E1
:101900000801F8D140F60F0001F0F8FC2046BDE8D0
:101910001040D1E6012304F8103FE7E7BC23FF1F86
:1019200030B5194C83B0237800228DF8072013B905
:10193000022003B030BD154B01201D6801F05CFD95
:1019400001231A4628440DF1070101F0FBFC237C1A
:10195000022B07D0227F022A11D0FFF70BF90020BB
:1019600003B030BD03232374237F0222032BF4D161
:1019700002EB420204EB820400232371EDE7032211
:1019800022770122F2E700BFBC23FF1FEC85FF1F77
:1019900038B5174B1A7CC2B91C46012204F8102F27
:1019A0008288A280042565808079A268A0710125C3
:1019B00000209571D0711A78A3680D0A19725D72B2
:1019C0003AB900232370022038BD1A7F5AB1022091
:1019D00038BD2378012BF4D101462046FFF79CFE49
:1019E0000028EED138BD1C46012204F81C2FD7E791
:1019F000BC23FF1F2DE9F047484C82B0237800201C
:101A00008DF805001BB9022002B0BDE8F087444BF9
:101A10001E6801F0F1FC371800F5805539460DF1CC
:101A2000060001230222354401F08EFC26791EB106
:101A3000012002B0BDE8F0874FF00108304684F87D
:101A4000048001F0F1FCA5F6FB7A8146434601A82B
:101A50004246514601F078FC9DF80400DFF8D0E0E2
:101A6000C0F302108DF8040018B19EF801308342D3
:101A700038D001231A468EF8010051460DF10300BB
:101A800001F062FCBDF806209DF80360E0680632B4
:101A9000002392B206F00F0639468DF8036001F07C
:101AA00053FCBDF8063099452CD81E48E38002222D
:101AB0000123A5F6FE7101F047FC01231A46A5F6A5
:101AC000FC71194801F040FC9DF80330032B15D040
:101AD00002211648FFF75CFF01284FF0000093D069
:101AE000207191E709F1FF310DF1060039444346B9
:101AF000424601F029FC2671022085E70B48FFF7DA
:101B000057F8E9E7012309F1FF311A4639440DF18D
:101B1000050001F019FCBDF80630C6E7BC23FF1F25
:101B2000EC85FF1FC423FF1FC623FF1FC023FF1F19
:101B30006215FF1F00887047006870470B0A01702C
:101B40004370704710B40A0C0C0A0B0E44700170FD
:101B50008270C37010BC704749B942B9012826D0C1
:101B6000354B998D09293AD940F207207047F0B5D5
:101B70000E4683B014461F46054601AB6A46214611
:101B80003046FEF775F918B140F2011003B0F0BD10
:101B9000019B3B80082221463046FEF719FC012DAF
:101BA00010D0010616D440F2072003B0F0BD224B3E
:101BB00019880529D8D803EBC1000131426019808A
:101BC000002070474406EED510F0380F24D140F2C3
:101BD0000510DBE7420709D14FF48270D6E703EB2B
:101BE000C1000131026399850020704721463046CB
:101BF0000422FEF7EDFB4307EED00F4B998D092928
:101C0000D1D8009803EBC102106308B138889086E0
:101C1000013199850020B9E7074B19880529C2D8F9
:101C2000009803EBC102506008B13888108101317F
:101C300019800020AAE700BF2C35FF1F10B504460D
:101C4000054801F0DDFD012C01D0002010BD02206F
:101C500001F0C4FB002010BDA435FF1F08B5032010
:101C600001F0BCFB022001F0B9FB002008BD00BF61
:101C70002DE9F04F8FB083460BAB09AA00214FF43A
:101C8000E050FEF7DFFB28B140F2062528460FB0F2
:101C9000BDE8F08FBBF1030F054609D0BBF1020F81
:101CA000F2D17F4B188001234FF0030A039305E024
:101CB0007B4B988502234FF0040A03939DF8243050
:101CC000022BE3D90BF58073DB009A1D07330192D9
:101CD00002930324049506E001349DF82430E4B215
:101CE000A342C0F0D5800BAB0DF1250221464FF485
:101CF000E050FEF7A7FB0028C6D19DF825305345DC
:101D0000EAD1584601F078FBB0F5805FC0F0C5809D
:101D1000584601F089FB0546019801F0C7FAC20751
:101D200002D4002D40F0B980029801F0BFFA10F003
:101D3000010F58464FD101F08FFB584601F0B0FB20
:101D40000546002D40F0A98004F5E0570F373846CE
:101D50000BAB0DF126022946FEF774FB002893D148
:101D6000019801F0A3FAC307B6D5584601F05CFB11
:101D70009DF82630814600283AD1002BACD00125B1
:101D8000CDF814A0DDF80CA006940BAB0AAA2946E6
:101D90003846FEF757FB00287FF476AFBDF8288061
:101DA000ADF82A0028F4FF73BAF1010F23F0010304
:101DB00023D0B3F5D05F23D041460DF12A03002292
:101DC0005046FFF7C9FE002864D040F20725284698
:101DD0000FB0BDE8F08F01F0F3FA584601F03CFB7C
:101DE000584601F05DFB0546584601F0F7FAA8E7B2
:101DF000002B52D0A9460125C2E7B3F5B05FDBD175
:101E00000DAB0DF1270200214046FEF71BFB002819
:101E1000DBD19DF8274044B30446064607950136BA
:101E2000F6B20DAB31460CAA4046FEF70BFB0DF1A6
:101E30002A030028C9D10C995046C1F3C405C1F347
:101E40000722090CADF82A500D95FFF785FE0028F2
:101E5000BBD1BDF82A300D9A1C449342A4B2B4D130
:101E60009DF82730B342DAD8079D9DF8263001351A
:101E7000EDB2A144AB421FFA89F986D25846DDF88B
:101E800014A0069C01F0D0FA81457FF625AF9CE7AF
:101E9000049DFBE6BDF82A40E7E74FF40275F5E63E
:101EA0002C35FF1F2DE9F047DFF870A0DFF87090A8
:101EB000DFF87080DAF80070B9F80C30B8F800502C
:101EC00082B01F449DB10024254608EBC4060123BF
:101ED00032897068394601F037FA01343389B8F82D
:101EE0000020E4B21D44A242ADB21F44EDD8B9F8BF
:101EF0000E30AB420CD9B9F80C20DAF800101344BC
:101F00005A1E012311440DF107001A4601F01CFA74
:101F100004F010FC02B0BDE8F08700BFEC85FF1FA5
:101F2000F085FF1F2C35FF1F08B5822242F2107189
:101F3000034801F061FCFFF7B5FF002008BD00BFBA
:101F4000A435FF1F2DE9F047DFF86CA0DFF86C9097
:101F5000DFF86C80DAF80070B9F81230B8F82C505D
:101F600082B01F449DB10024254608EBC40601231E
:101F7000B28E316B384601F0E5F90134B38EB8F812
:101F80002C20A4B21D44A242ADB21F44EDD8B9F832
:101F90001430AB420CD9B9F81220DAF8000013441F
:101FA0005A1E012310440DF107011A4601F0CAF927
:101FB00002B0BDE8F08700BFEC85FF1FF085FF1F72
:101FC0002C35FF1F08B5FFF7BDFF022001F0F8F91F
:101FD000032001F0F5F9022001F026FA20B90220D1
:101FE00001F03AFB002008BD012001F035FB002084
:101FF00008BD00BF2DE9F04F89B088469346019394
:10200000074600285AD18DF810200025AA465C46C4
:102010004FF0010906AB07AA21464046FDF728FF0D
:10202000012F064603461BD0B6BB05AB0DF11202CD
:1020300021464046FEF72EFCBDF8143013F4805FB5
:1020400008BF4FF00009012F11D0069B9DF810200A
:102050001D44B246ADB20134E4B29442DAD913E081
:1020600040F215229042DFD19DF81020F3E7BDF831
:102070001230012B14D0B246069B1D44ADB29DF820
:102080001020002CE7D1B2B9B9F1010F129B2BD06F
:10209000AB422BD940F20313184609B0BDE8F08FCC
:1020A000BAF1080F1ED00AF1010A5FFA8AFABAF1F2
:1020B000010FE4D8E0E70135ADB2CCE704AB0DF198
:1020C0000F020DF112014046FEF7D0FB0346002837
:1020D000E2D19DF810305B4597D2129B002BD9D1ED
:1020E0000023D9E7BA46C7E7AB42D3D15A45F7D365
:1020F000DFF84091DDF804A001265C4606AB07AA94
:1021000021464046FDF7B4FE012F15D0002873D1BB
:10211000FEF750FF214602464046FEF759F910F0FF
:10212000380FADF8140012D1002F38D140F205134A
:10213000184609B0BDE8F08F40F215239842E5D16A
:1021400001349DF81030E4B2A342D7D2C8E75FBB98
:10215000BDF81850D34601263B465A462146404614
:10216000FEF7DAFB002847D1BDF8143013F4805F86
:10217000079B39D159462A46184605F097FE224654
:102180004146384604F0DCFA002842D1069B9A44C6
:10219000002FD5D0002CD3D10AF1010AD0E7069B3D
:1021A0009A44002CCCD1F7E70DF116030DF1120281
:1021B00021464046FEF76EFBF0B9BDF81250012DE6
:1021C000C6D1012E1ED01AF8013C1E4214BF0123B5
:1021D0000023802E0AF1FF3A8DF811300ED07600E0
:1021E000F6B20DF1110BB7E719462A46484601939E
:1021F00005F05CFE019BBDE703464DE72E460DF161
:10220000110BA9E79AF8003003F001038DF81130A3
:10221000E5E7012803463FF43FAFBDF81420D204A0
:102220007FF53AAF01902A460249079805F03EFE35
:10223000019B31E7B435FF1F70B582B0054601A898
:102240000E46FFF71FFB38B100210846FEF716FDCA
:102250000225284602B070BD019BAA889A800A22F6
:1022600004465A809868AA799A7106304FF4004162
:10227000FFF764FC019B9A68072111729A689472B7
:10228000986821460A30FFF759FC019B986831464F
:102290000C30FFF757FC03210198FFF70BFB0546B5
:1022A00048B1019B204621461C70FEF7E7FC022541
:1022B000284602B070BD01460820FEF7DFFC284624
:1022C00002B070BD2DE9F041904D2B8982B05BB911
:1022D000044680680C30FFF72DFC0528688167D81C
:1022E000A288A379AA81EB8101A8FFF7CBFA044663
:1022F00040B100210846FEF7C1FC0224204602B08E
:10230000BDE8F081019BA9899868EA899980062136
:1023100059809A7108444FF40041FFF70FFC019A6D
:102320002B8991684FF0020881F8088091688C72BF
:10233000976807F10C06002B48D0013B2B816B8975
:1023400023B1E98A0020FEF7DBF9E0B9019B298976
:102350005A88986814445C800A30FFF7EFFB2B8999
:102360000198EBB92B760321FFF7A4FA044640B39A
:10237000019B002108461970FEF780FC02242046CC
:1023800002B0BDE8F08101463046FFF7D7FB0234CA
:102390002B69A4B2B4EB430F06F10206D1D1D5E705
:1023A0008268137A012163F07F0313722976DAE7DA
:1023B00020465749FFF740FF0446204602B0BDE8DB
:1023C000F08129890620FEF759FC97E7012001F0EA
:1023D0002BF80C38430869892B613046FFF7AEFBB8
:1023E0006C8907F10E0634B3012C64D0022C0ED098
:1023F000032C6BD0042C72D0052C7BD0A88A4446C9
:102400002B69421C9A420AD800232B8197E740216E
:102410000120FEF775F94023A882EB82F0E7C3F1B3
:1024200001021044B0FBF3F203FB120392B203B1BA
:1024300001322A8183E705234FF6FF710120AB8229
:10244000FEF75EF9034601463046AB82FFF776FBA6
:1024500040210120FEF754F90346014607F1100020
:10246000AB82FFF76BFB80210120FEF749F90346A1
:10247000014607F11200AB82FFF760FB4FF4807159
:102480000120FEF73DF90346014607F11400AB8237
:10249000FFF754FB4FF400710120FEF731F90346BA
:1024A000014607F11600AB8207F11806FFF746FB5D
:1024B0000C24A88AA4E720464FF6FF71FEF720F906
:1024C0004FF6FF734446A882EB8299E780210120F2
:1024D000FEF716F980234446A882EB8290E74FF47A
:1024E00080710120FEF70CF94FF480734446A882F6
:1024F000EB8285E74FF400710120FEF701F94FF4FC
:1025000000734446A882EB827AE700BFB435FF1F10
:10251000430004062DE9F0415D4C638B82B03BBB68
:10252000054680680C30FFF705FB0DF101036A4694
:102530000DF10201A083FEF799F938B904F11E02EA
:1025400004F12001A08BFEF791F840B128465149D3
:10255000FFF772FE0546284602B0BDE8F081AA8862
:10256000AB79A2840120E38400F05EFF0C38A06206
:1025700001A8FFF787F9054640B100210846FEF79C
:102580007DFB0225284602B0BDE8F081019BA18CAD
:102590009868E28C9980062159809A7108444FF41A
:1025A0000041FFF7CBFA019B668B9A6804211172F8
:1025B0009A6895729F6807F10C00002E3BD0013E8F
:1025C000B6B26683A846A26AE38B216A551B9D4278
:1025D00028BF1D462A4605F069FC019F226A7B88B8
:1025E000B8681FFA85FE43441544E28B25627344A4
:1025F0007B800A30A2EB0E033146E383FFF79EFA9D
:10260000638B0198002B39D08268137A022163F022
:102610007F03137221760321FFF74CF9054678B347
:10262000019B002108461970FEF728FB0225284669
:1026300002B0BDE8F081E38BA26A991D914208D9EE
:102640009B1A0633B3FBF2F102FB113389B2E3B9F3
:102650006183A18BFFF772FA07F10E00BDF802103B
:10266000FFF76CFA06259DF801209DF800303A74BA
:102670007B7407F11200A846668BA4E72376CAE7AD
:10268000618B0620FEF7FAFA7CE70131E0E700BF34
:10269000B435FF1F000002062DE9F041B04DAC8DAE
:1026A00086B0002C41D1064680680C30FFF742FA14
:1026B000B368E885997BDF7B85F8301005F132033C
:1026C0000DF1060285F83170FEF7E4F8C0B1A549B6
:1026D000234640F2031205E00133172B00F001817D
:1026E00031F833209042F7D19E4A02EBC303596878
:1026F0003046FFF7A1FD0446204606B0BDE8F08154
:102700006B8EB188B279A98613F4805F95F8313069
:10271000EA8608BF03F08F0323F06003012085F8E9
:10272000313000F081FE0C38A86302A8FFF7AAF848
:10273000044640B100210846FEF7A0FA02242046D4
:1027400006B0BDE8F081029BA98E9868EA8E998058
:1027500006269A715E8030444FF40041FFF7EEF98F
:10276000029AAB8D91680E7291688C72976807F12E
:102770000C06002B46D0013BAB8595F8313019078C
:1027800004D5AA6B271D974240F2CC80DA0629D4E3
:10279000002B00F0AE80029BA98D5A8898681444E3
:1027A0005C800A30FFF7CAF9AB8D0298002B00F06D
:1027B00096808268137A032163F07F03137229766F
:1027C0000321FFF777F80446002800F08D80029B74
:1027D000002108461970FEF751FA0224204606B07F
:1027E000BDE8F08103AB05AA95F83010E88DFDF740
:1027F000BFFE039AAB6BA118994240F2B78095F8DF
:102800003130C5E73046E98DFFF798F995F830206B
:1028100095F83130BA7307F11000FB73BDF806105C
:10282000FFF78CF9BDF80600012807F1120875D0F2
:10283000FDF7B4FD04460490002840F0AA8005AEE0
:10284000324604AB95F83010E88DFDF711FB0028F7
:1028500040F0A280BDF810104046FFF76FF9698E76
:1028600007F11400C1F30901FFF768F900243246AB
:1028700003AB95F83010E88DAC87FDF7F9FA95F8C1
:1028800031301A0707F1160602D5AA8F0432AA873B
:10289000DF0603D5A98F039A0A44AA879C0603D5AD
:1028A000A98F039A0A44AA87580603D5AA8F039BC7
:1028B0001344AB872C4B95F83010E88D9A1CFDF72C
:1028C000EDFEAB8FE98FAA6B0B449BB203F10A01BB
:1028D0009142AB8736D80023AB850A244DE72B768F
:1028E0006EE74FF0006103E7A98D0620FEF7C6F9F9
:1028F00025E7AB6BEA8F296C1F1B974228BF174651
:102900003A46304605F0D2FAAA8F2B6CB9B20C4485
:10291000521A1F44A4B2AA872F643CE704900146D0
:1029200005AE99E730460021FFF70CF9AA8F95F81C
:102930003130043A03F0F703BCB20436AA8785F8B5
:10294000313023E7C2F10A011944B1FBF2F302FB73
:1029500013129BB202B10133AB850A240DE700BF0D
:10296000B435FF1F808E0100F235FF1F05993046F8
:1029700005F09CFA0399AA8F95F8313088B2044487
:10298000121A03F0EF030E44A4B2AA8785F831307F
:10299000FEE681B205AE5FE7049421465CE700BF26
:1029A00010B50C4C237E012B09D0022B0DD0032B2C
:1029B00000D010BD0020BDE81040FFF76DBE002024
:1029C000FFF780FC237E022BF1D10020FFF7A2FD50
:1029D000237EECE7B435FF1F2DE9F04182B00446B9
:1029E00001A8884617461E46FEF74CFF40B100215D
:1029F0000846FEF743F90224204602B0BDE8F08104
:102A0000019BA2889A800A225A8005469868A2797A
:102A10009A7106304FF40051FFF790F8019B9A68C5
:102A200080211172986841460930FFF787F8019BB1
:102A30009A68D772986831460C30FFF783F8032103
:102A40000198FEF737FF044650B1019B28462946FE
:102A50001D70FEF713F90224204602B0BDE8F08194
:102A600001460820FEF70AF9204602B0BDE8F081D1
:102A70002DE9F0430446806885B009308846FFF7A9
:102A800059F8A3681A7ADD7A12F01007064602D0C8
:102A9000012D4DD80127B8F1010F30D003F10C0002
:102AA000B4F80290FFF748F8A36802461033B8F173
:102AB000000F05D1A9F10A0E1FFA8EFE704543D80A
:102AC000009231462A463846FFF794FA20B344492B
:102AD00040F20312002304E00133172B31D031F808
:102AE00033208242F8D13E4A02EBC3035B682A4698
:102AF00031462046FFF770FF05B0BDE8F083C2F312
:102B00008102C2F1040200920C332A463146384653
:102B1000FFF770FA0028DAD103A8FEF7B3FE50B32E
:102B200000210846FEF7AAF8022005B0BDE8F083B0
:102B300001462A4620462B4BFFF74EFF05B0BDE865
:102B4000F0834FF00063D2E7DFF89CC01946CCF861
:102B500048200CF155007246ACF844608CF84650A1
:102B6000CCF84CE08CF8547005F0A0F903A8FEF7FF
:102B700089FE0028D4D1039BA2889A800A225A8019
:102B80009868A2799A714FF440510630FEF7D6FF4B
:102B9000039B9A6860211172E7B998683146093041
:102BA000FEF7CCFF03988368DD7283680024DC6045
:102BB0000321FEF77FFE38B1039B204621461C709F
:102BC000FEF75CF8022097E701200021FEF756F897
:102BD000002091E799680A7A42F010020A72DCE755
:102BE000808E010043000406B435FF1F2DE9F04F2D
:102BF00091B0164603939DF8703004939DF874309D
:102C00000790DDF8688000930D46002940F04F8161
:102C10009DF80C308DF82B304FF0000ACDF868800D
:102C2000039C0DF138090DF1340BD0460CE000285F
:102C300040F02581BAF1010F40F21E8101349DF868
:102C40002B30E4B2A34228D34B465A4621463046A5
:102C5000FDF70EF9012D0746E9D140F21523984200
:102C6000ECD0002840F00B810CAB0DF12E02214678
:102C70003046FDF70FFEBDF82E30012B00F00A8123
:102C8000BA460E9B9844002CD8D101349DF82B30C5
:102C9000E4B2A34208F10108D6D201204446CDF89F
:102CA0002080DDF8688000F0BFFB042C834640F2F2
:102CB0001581103883B209930FA800230693FEF7FD
:102CC000E1FD0590002840F01781049B052B00F0E2
:102CD0002381089B042B0F9B9A6800F27E8102F1EE
:102CE0000C0A9DF82B2003998A4238BF00277AD31B
:102CF0000DF1340B0023CDF804B0039CDDF824B0B3
:102D000002931F460DF138094B46019A2146304681
:102D1000FDF7AEF8012D00F0F980002840F0608149
:102D2000B8F1000F06D00D9A0E9B4244A3EB0803A6
:102D30000D920E93FEF73EF9214602463046FDF70E
:102D400047FB4207ADF8300040F0EB80002D00F06B
:102D5000A181009B012B00F0F5804FF001080DF1DF
:102D600032030DF12E0221463046FDF793FD002877
:102D700040F03681BDF82E30012B00F00C810D990A
:102D80000E9A0290BB185B4511D9AD4BA3F8446075
:102D900083F8464083F85450049BABEB0702052BA5
:102DA0000E92A74B00F0F0801A6500230693B8F14D
:102DB000000F40F0C280504605F078F80E9B1F448B
:102DC000BFB29A4425B11CB901370AF8014BBFB212
:102DD000BB4507D04FF0000801349DF82B30E4B21A
:102DE000A34291D20F9B079998688A889A800A22F9
:102DF0005A808A799A7106304FF44051FEF79EFE50
:102E0000049B052B00F022810F9B9A6840211172D0
:102E100099680A7A012D42F001020A7200F03E819F
:102E2000069A002A00F0E98099680A7A42F00202C4
:102E30000A72089A9968C2F10402087A920002F0B4
:102E40000C0202430A72986831460930FEF776FE9A
:102E50000F989DF80C2083680321DA72FEF72AFD93
:102E6000002800F0E9800F9B002119700846FDF74B
:102E700005FF0223059309E00E9B9844DEE62246F7
:102E8000314607986F4BFFF7A7FD0590059811B0E5
:102E9000BDE8F08FBAF1080F00F09D800AF1010A39
:102EA0005FFA8AFABAF1010F7FF6EBAEEBE60DF1AD
:102EB0002B030BAA0DF12E013046FDF7D7FC03467C
:102EC000002840F098809DF82B2003998A42BFF497
:102ED000A3AE0120089300F0A7FA8346ABF10C0BD8
:102EE0001FFA8BF309930FA801230693FEF7CAFC80
:102EF000059000283FF4E9AE00210846FDF7BEFE2C
:102F000002230593059811B0BDE8F08F40F2152318
:102F100098427FF402AF5FE70F9B9A6802F1090ABB
:102F2000DFE6009B012B00F0D480002D40F0CE8026
:102F30000D990E9A0295A84624E70021504604F008
:102F4000C0FF3BE722463146284603F031FC00280B
:102F50003FF403AF0F9A3C490023137040F2031271
:102F600005E00133172B00F0AE8031F833208242A8
:102F7000F7D1354A02EBC3035B6807982246314616
:102F8000FFF72AFD059081E71B6D2D48134403656B
:102F9000002306930BE70D9A02981278003218BFAF
:102FA000012210F0F70F8DF82D20014611D01AF8EC
:102FB000013C824001311A43013FCBB2BFB20293C0
:102FC0008DF82D200AF1FF3A01220E920DF12D010C
:102FD000D8E60293F8E7AA4653E602F1100A80E623
:102FE0000F9D0798174B0027224631462F70FFF799
:102FF000F3FC05904AE7039A42E75A8898680899D3
:103000003A445A800C30FEF79DFD0F9B986831467C
:103010000930FEF793FD0F989DF80C20836803217B
:10302000DA72FEF747FC00287FF41DAF089B0420EE
:10303000D91BFDF723FE29E701460320F9E700BF6E
:10304000B435FF1F11000906808E01000F988368B8
:1030500000221A72079B9B681B7ADB0604D58268E4
:10306000137A43F0100313721B9B9F4225D0072F46
:103070001AD94388073B3B4443800321FEF71AFCDF
:10308000059000287FF4EFAE1B9B0520D91BFDF7B0
:10309000F5FDFBE60F9A134B15706EE799680A7AF7
:1030A00042F010020A72BBE68268FB1F117A5B00D5
:1030B00003F00E030B431372DFE78268137A43F0C9
:1030C00001031372D3E74FF0006356E74FF0000897
:1030D00045E622463146284603F06AFB00283FF4C5
:1030E00024AF37E70100010630B585B0084C0191E7
:1030F00094F84630B4F8442094F85410246D0094A9
:103100000025052403950294FFF770FD05B030BD3E
:10311000B435FF1FF0B50546806885B00930FEF76D
:1031200009FDAB681C7ADB7A14F0100418D0012B6F
:103130000DD80121002401270426024603972846C2
:10314000029601940094FFF751FD05B0F0BD1A46B8
:10315000044B0146284605B0BDE8F040FFF73CBCF3
:103160002146E7E74300040670B544880A2C84B082
:1031700006465AD0033CA4B2494DE86C23180A2BEA
:1031800043D8B168284422465530093104F08EFEF8
:10319000EB6CB2681C44EC64137ADA070CD403A815
:1031A000FEF770FB002845D000210846FDF766FDBC
:1031B0000224204604B070BDAB6C95F84620B5F8EB
:1031C000441095F85400009305F15503FEF712FFE3
:1031D0000028E4D0B5F8441095F84620314D40F26F
:1031E0000314002304E00133172B51D035F833408A
:1031F000A042F8D12B4800EBC3035B683046FFF7D1
:10320000EBFB0446204604B070BD00210846FDF7E4
:1032100035FD3046244B95F84620B5F84410FFF7AD
:10322000DBFB0446204604B070BD83681C7AC4F3FF
:103230004204A1E7039BB2889A800A225A809868C8
:10324000B2799A7106304FF44051FEF777FC03983B
:10325000836820221A72B3681B7ADB0604D5826861
:10326000137A43F01003137283680025C3F80950E2
:103270000321DD60FEF71EFB044660B1039B284678
:1032800029461D70FDF7FAFC0224204604B070BDEB
:103290004FF00063B2E701460220FDF7EFFC88E73C
:1032A000B435FF1F808E01000500040500B583B012
:1032B000014601220DF1070000F04EFB9DF80700CA
:1032C00003B05DF804FB00BF00B583B001460222E5
:1032D0000DF1060000F040FBBDF8060003B05DF8FC
:1032E00004FB00BF00B5042283B001460DEB0200D1
:1032F00000F032FB019803B05DF804FB00B583B029
:1033000002AB012203F8011D194600F05BFB03B07C
:103310005DF804FB00B583B002AB022223F8021D66
:10332000194600F04FFB03B05DF804FB00B583B015
:1033300002AB042243F8041D194600F043FB03B01E
:103340005DF804FB00F03EBB00F006BBF8B50520BD
:10335000FFF7ACFF184E0428307029D904233370CE
:10336000164F002403E00134E4B29C421FD204F55E
:103370008075ED00E81D0121FFF7C0FF3378A342FF
:10338000F1D92846FFF7A0FF337804EB4402A342AB
:1033900027F8120005F1020007EB4205E3D9FFF719
:1033A00093FF013433786880E4B29C42DFD3F8BDE8
:1033B0000028D5D1FBE700BF1436FF1FF085FF1FA3
:1033C000054B1B78834200D87047C00000F6070009
:1033D0000021FFF793BF00BF1436FF1F054B1B787A
:1033E000834200D87047C00000F607000121FFF7B4
:1033F00085BF00BF1436FF1F094B1B78834201D8DD
:103400000020704710B5044600F58070C000FFF73B
:103410005BFF04EB4404034B23F8140010BD00BF12
:103420001436FF1FF085FF1F094B1B78834201D81C
:103430000020704710B50446C00000F60200FFF7F8
:1034400043FF044B04EB440403EB4404608010BDD1
:103450001436FF1FF085FF1FF8B500F58076F600E3
:1034600005463046FFF730FF0746B01CFFF72CFF3C
:103470000446301DFFF71AFF830708BF04EB44041E
:10348000064B07F1FF3008BFA4B205EB4505044425
:1034900003EB4505A0B2A880F8BD00BFF085FF1F73
:1034A0002DE9F0411A4F3B785BB31A4D00EB400811
:1034B000064605EB48080024E00000F60600FFF78A
:1034C000F5FEA64204F1010217D06300191910F0AD
:1034D000010F05EB410010D035F81130B8F800109D
:1034E0009942044602D3808888420DD2B8F804106D
:1034F0008B4202D8A3888B4206D23B78D4B2A34237
:10350000DAD80020BDE8F0810220BDE8F08100BFDC
:103510001436FF1FF085FF1F70B5044682B0FDF71B
:1035200049FD022C23D0032C1ED1234B9A78022A6A
:1035300004BF01225A70082836D0042834D01F4B0B
:103540001F4D1C686B8A1C4401231A4620460DF14E
:103550000701FFF7F7FEA88A0123013820440DF187
:1035600007011A46FFF7EEFE002002B070BD124BB5
:10357000012408285C701CD0114E104B1D68B389C3
:103580001D4429460DF1070023462246FFF7DCFEC5
:10359000F18901390DF10700294423462246FFF73E
:1035A000D3FE002002B070BDFEF7CCFC002002B0BC
:1035B00070BDFEF777FCD7E71436FF1FEC85FF1FC1
:1035C000F085FF1F0320FFF7A7BF00BF70B50C4CAD
:1035D0006368012B06D063780BB10123636000237D
:1035E000637070BD6678002EF7D1054603F01EF9B2
:1035F0000220FDF721FD284600F002F96660EAE7A7
:103600001436FF1F38B540F6060440F686052046FE
:103610000834FFF74BFEAC42F9D138BD10B540F687
:103620000E00FFF743FE10F001030FD0094C237A80
:1036300000F0020083420BD02072FEF74BF9217A92
:1036400040F60F00BDE81040FFF758BE014A137264
:1036500010BD00BF1436FF1F014B9870704700BFAC
:103660001436FF1F014B9878704700BF1436FF1FB8
:1036700030B42B4D2C6844B1844203D148E09842C9
:1036800013D01C462368002BF9D122F020030373CA
:1036900012F0200308BF4381224B41601B88B1EB2D
:1036A000C33F0BD9022030BC70470368236090F9F8
:1036B0000C30002BA4BF00234381E6E744890C446F
:1036C000A34221D2B4FBF3F103FB114389B243813E
:1036D00001811BB113065CBF013189B22B792A68C5
:1036E000194489B20181B2B113898B4204D912E025
:1036F0001C89A14203D31A461368002BF8D103603A
:1037000030BC106000207047002343810121E5E7B1
:1037100003682B60CBE7026028600020C3E700BF8E
:103720002036FF1F6415FF1F70B5324E34683379A1
:10373000002C5CD0DBB2228999B2914254D330790B
:10374000C31ADBB233712546002000E02A8991427A
:1037500096BF521A28812A812D68002DF6D123891F
:10376000BBB9207B20F08003022B24D0316849B301
:10377000A14236D00A4602E0A3420BD01A46136893
:10378000002BF9D110F0C00F0CD10C462389002B6F
:10379000E7D070BD23681360030658BF658110F041
:1037A000C00F04D0616800F0BF00207399B934687D
:1037B000002CD4D170BD2046FFF708FF3168207B74
:1037C0000029D5D110F0C00FE3D0616800F0BF0030
:1037D00020730029EBD040F020022046FFF748FF7D
:1037E000E5E723683360D7E7092BA8D870BD3471AB
:1037F00070BD00BF2036FF1F01B139E701207047BF
:103800000C4B1A684AB1824203D110E0984205D0AD
:103810001A461368002BF9D170477047036813608C
:1038200090F90C30002BF8DB0023438170470268CD
:103830001A60F5E72036FF1F70B5104E336813B9D4
:1038400011E01B687BB19842FBD10D460C490389FE
:10385000098803FB01F1044659B9012032796560FA
:103860009B1A238170BD09B9012070BDBDE870406D
:10387000FEE62046FFF7FCFE2389EFE72036FF1F18
:103880006415FF1F074B1B683BB1834202D106E062
:10389000984204D01B68002BFAD1184670470120CB
:1038A000704700BF2036FF1F034A13790133DBB294
:1038B00001211371517170472036FF1F70B5054605
:1038C0000E46F5F7D3FBC5F3471343F000431F4AF9
:1038D00043F480335363D36A002BFCDA936BD16AD1
:1038E0001B4B1A4CE80000F0F80041F01041034374
:1038F000D1625363E36A002BFCDA2B0A23F01F0327
:1039000043EA8603A26BE16A104ADBB243F000434C
:1039100043F4803341F01041E1626363D36A002BCA
:10392000FCDA936BD36A032E43F01043D36200D0CA
:1039300070BD084B05495363CB6A002BFCDA8B6BD7
:10394000CB6A43F01043CB6270BD00BF00D0024091
:1039500006000180FF00018089B238B50546144693
:1039600008460321FFF7AAFF0CB31349134A012CA1
:103970000DD04A63CB6A002BFCDA8B6B05F8013B58
:10398000CB6A013C43F01043A4B2CB62EFE70A4B91
:103990000B4A5A63DA6A002AFCDA074BDA6AD20069
:1039A000FCD59A6B2A70DA6A42F01042DA62BDE8FE
:1039B0003840F5F753BB00BF00D002400000018043
:1039C000FF00010838B580B20D4614460421FFF708
:1039D00075FF34B3154A16482946012C0ED00B78D2
:1039E000134343630131C36A002BFCDA836BC36A60
:1039F000013C43F01043A4B2C362EEE70B780C4ADB
:103A000043F0006343F480335363D36A002BFCDA42
:103A1000074BDA6AD200FCD59A6BDA6A42F01042A0
:103A2000DA62BDE83840F5F719BB00BF000001803D
:103A300000D00240F0B5114C114F124A124E134BF8
:103A4000134D03CC3860796003CA3060716003CBDA
:103A5000B4F800E01288A7F808E00E4F1C88328105
:103A60000D4B0E4E2C8100226FF0004428606960DF
:103A70003A7010469E64DC64F0BD00BF2CA20100C9
:103A8000BC01FF1F38A20100B001FF1F44A20100CA
:103A9000A401FF1F2636FF1F4400FF1F0100008006
:103AA000014B002018607047EC85FF1F08B54FF4EC
:103AB000A070FFF709FCC0B208BD00BF08B54FF405
:103AC000A070FFF701FCC0B2A0F10500B0FA80F0D1
:103AD000400908BD10B5002002F06AFF002000F088
:103AE0009FFB00F031FC012000F08CFA012000F077
:103AF00057FB012000F004FF002000F083FA0020B3
:103B000001F07EFC002000F04BFB002001F084F867
:103B10000E4C002000F0F4FE0D4B626E1A6000F0B7
:103B2000A7FF002001F0E0FC638803F06F033BB9BE
:103B3000002001F0F1FA638803F06F03002BF7D047
:103B400002F0D2FEBDE8104000F00EBC4400FF1FA2
:103B50006486FF1F08B5FDF7FBFC012000F01EF88E
:103B600002F06AFE02F0B6FE38B9002000F016F846
:103B70000020BDE8084001F0CFBA00F04FFFFFF78A
:103B800021FDF2E7044B588800F06F00A0F1080017
:103B9000B0FA80F0400970474400FF1F2DE9F0475C
:103BA000CD4EC700F319D3E9002352EA030182B0D6
:103BB00024D0840006EB0408D8F8BC50E90700F1D3
:103BC000888015F0020100F08F8030B1C349D1E93F
:103BD000002342F00072C1E9002396F8B8E096F89D
:103BE000B930344425F002057345C4F8BC504FF099
:103BF000000939D1484602B0BDE8F087B74DB84951
:103C00003D443944D5E90045D1E900894D4508BF17
:103C1000444521D0002188EA040889EA05094FF0CB
:103C20003F0E4FF0010CAEF12005CEF120040CFA4E
:103C300005F32CFA04F423430CFA0EF208EA02040A
:103C400009EA030501310EF1FF3E2C43C9B25FFAC8
:103C50008EFE2CD14029E6D196F8B8E096F8B9301E
:103C60004FF001097345C5D09E4906EBCE0301EB29
:103C7000CE010231188AFDF7BBF804460028B9D1FD
:103C800002AA014602F8010D012341F20100FCF7EE
:103C9000FFFB96F8B830142B18BF013348460CBF11
:103CA00086F8B84086F8B83002B0BDE8F0878E4C90
:103CB0004FF0000E2146D1E900894B4508BF42452F
:103CC00001F120015FD00EF1010EBEF1150FF2D10E
:103CD000C2E725F00105C8F8BC5096F8B8E096F8A0
:103CE000B9304FF00009BDE715F0040979D115F09E
:103CF000080A40F0978015F0200964D115F04001C2
:103D000040F09F8015F0800F40F0BE8015F4807960
:103D100040F02381A90500F1FC80680500F11181C4
:103D200015F4006971D115F4805140F09D8015F4AF
:103D3000005940F0DF80690400F1F48015F400417F
:103D400000F03F81002003F040010143634D07D0A4
:103D500005EB070EDEE9000120F01000CEE90001BE
:103D60003D44D5E90089344429EA0309374428EA67
:103D70000208002000210023C5E90089C7E90001ED
:103D8000C4F8BC3068E74FEA400806EB080504EBCE
:103D90004E11840006EB040CB5F8C450D1F80CE0C9
:103DA000CCF8C8106906CCF8BCE003D52EF06C0E38
:103DB000CCF8BCE0B044F11945EA0E05C1E9002396
:103DC000A8F8C450F6E600F0B5F9D8F8BC2096F88B
:103DD000B8E096F8B93022F02002D146C8F8BC20ED
:103DE00040E7424C96F8B8E096F8B930942202FBCE
:103DF000004025F004054288C8F8BC5022F06F024C
:103E000042F00F02894642802CE7384B5B8803F072
:103E10006F03082B42D096F8B8E096F8B9304FF00F
:103E200000091FE7314B942404FB00340121626E2A
:103E300000F04AFA012840D096F8B8E096F8B93078
:103E400010E72A4996F8B8E096F8B930942202FBB8
:103E5000001025F040054288C8F8BC5022F06F02DF
:103E600042F008024280FDE6204B5B8803F06F03BE
:103E7000082BD0D1344425F48055C4F8BC5096F8B2
:103E8000B8E096F8B930EDE625F08005C8F8BC50EA
:103E9000894696F8B8E096F8B930E3E63444144A17
:103EA00096F8B8E096F8B93025F400654FF00009AF
:103EB000C4F8BC5082F80090D4E66188D8F8BC20E1
:103EC00096F8B8E096F8B93041F4806122F0080223
:103ED0006180C8F8BC20C5E62836FF1F1086FF1F8A
:103EE0002086FF1F3836FF1F6815FF1F4400FF1F85
:103EF0000886FF1F414B5B8803F06F03082B8AD1B4
:103F00000120894602F064FD96F8B8E096F8B930D1
:103F1000A8E625F40075C8F8BC5096F8B8E096F805
:103F2000B9309FE6364BD3E90023002302F000723C
:103F300013433FF470AF344425F48045C4F8BC50BB
:103F40007AE7344425F48065C4F8BC5096F8B8E0AC
:103F500096F8B9304FF0000984E696F8B93096F833
:103F6000B8E05F1C774524D0B6F8B820B2F5A05F62
:103F70001FD03119DA00D1F8C8C0B118BCF80880D8
:103F8000A1F8108001289CF80AC081F812C03244C0
:103F900008BFFF20142BC87418BFFBB24FF00001FC
:103FA00011755175917506BF86F8B9100B4686F8E4
:103FB000B930344425F48075C4F8BC504FF0000982
:103FC00050E6E8037FF527AF0D4D96F8B8E03D4485
:103FD000D5E90089344443EA090342EA0802C5E905
:103FE0000023374400230022C7E90023C4F8BC1093
:103FF00096F8B9304FF0010934E600BF4400FF1FC6
:104000002086FF1FF0B40F4B0F4E1049104FC20017
:1040100000240025164411441A44C2E90045C1E9B0
:1040200000450022C6E9004503EB400403EB800392
:1040300008493A70A4F8C420C3F8BC20C3F8C810DB
:10404000F0BC70472836FF1F1086FF1F2086FF1F19
:104050000886FF1F6815FF1F2DE97003124E1349D4
:10406000134AC3001E44D6E900451944D1E900892A
:1040700004F0804405F03C0544F00104C6E9004525
:1040800013440024002502EB400008F0804809F0AA
:104090003C09C3E900450023C1E90089A0F8C43008
:1040A000BDE87003704700BF1086FF1F2086FF1F0A
:1040B0002836FF1F10B5002314460A460146062085
:1040C000F9F728FD2060F8F799FE642814BF4FF433
:1040D0008370002010BD00BF08B513680A46014672
:1040E0000520F9F717FDF8F789FE642814BF4FF48F
:1040F0008370002008BD00BF38B5024604460D4657
:10410000002303210620F9F705FD084B942202FB4A
:104110000434E16A6B1A984205DB29448842CCBF1B
:104120000020012038BD002038BD00BF4400FF1F23
:1041300000F0D2BF10B5044602F03AFC064800EB8E
:104140000410FFF75DFB054A32F8143023F0010339
:1041500022F81430012010BD3486FF1F3086FF1F67
:1041600070B50D4E345C05464CB10C4A32F8100067
:1041700010F0010002D000227255012070BD02F043
:1041800015FC064A012132F8153071550B432046C3
:1041900022F8153070BD00BFF836FF1F3086FF1FB4
:1041A000012803D0024B002223F81020704700BFE3
:1041B0003086FF1F2DE9F041164E174D56F820604E
:1041C000044617469846B04755F824303946064607
:1041D0002046984755F824200746414620469047F8
:1041E0003B46054622460B210520F9F793FC2B465A
:1041F00022460B210520F9F78DFC15B1074B43F83A
:1042000024503346224600210120F9F783FC002088
:10421000BDE8F0814486FF1F5086FF1F6486FF1FA4
:104220000023024619460320F9F774BC2DE9F84330
:104230001A4E1B4D56F820809DF820600446174604
:104240009946C04755F8243039468046204698475D
:1042500055F82420074649462046904743460546E0
:10426000224604210520F9F755FC3B4622460B2146
:104270000520F9F74FFC2B4622460B210520F9F7C4
:1042800049FC15B1074B43F8245022463146099B9F
:104290000420F9F73FFC0020BDE8F8834486FF1FA7
:1042A0005086FF1F6486FF1F38B502460C46054640
:1042B0000B4605200B21F9F72DFC14B1014B43F8F7
:1042C000254038BD6486FF1FF8B51A4D2B180446EB
:1042D0001B798B4215D0184B0E4653F820301146EF
:1042E00098472246074603460B210520F9F712FCA2
:1042F000CFB90023194622460320F9F70BFC2B19EE
:104300001E710023224603210620F9F703FC0B4B04
:10431000014653F8243020469847034638B92C44C8
:1043200001202371F8BD064B43F82470E1E700201B
:10433000F8BD00BFF836FF1F5086FF1F4C86FF1FD9
:104340006486FF1F00F06ABB064B10B441F2F272A4
:104350000124042000219C60D86019615A609A6190
:1043600010BC70478C01FF1F024B4FF480221A6073
:10437000704700BF1823FF1F2DE9F04784B004AB3E
:10438000002502AC43F8045D2246032141F21800E7
:104390000295FCF757F8002838D1029AADF80620AC
:1043A000120CADF804204FF00009DFF86CE0194F53
:1043B0004E460DF1040C4FF02E08052542F2107008
:1043C000B2FBF0F3A7FB00A100FB13229BB292B259
:1043D000C80813B9B9F1000F06D03033711C0EF8BC
:1043E00006304FF00109CEB2013DE9D12CF8022B85
:1043F000A4450EF8068004D00136F6B2BCF80020C1
:10440000DBE70EF8065004B0BDE8F087BDF80420E5
:10441000C9E700BFCDCCCCCCA401FF1F01490020CF
:1044200000F0F8B80818FF1FA0F50053B3F5E06FCF
:1044300010B40AD3A0F5C043B3F5006F14D24FF403
:10444000006422464FF4C04304E04FF40074224657
:104450004FF40053C31A93FBF4F3DBB203FB1200D7
:10446000088010BC184670470123088010BC18460D
:10447000704700BF0B4610B511460446184600F0C1
:1044800073FA28B1014620464B69BDE81040184731
:1044900010BD00BF10B5044600F018FE044A942376
:1044A00003FB04239861204600F0D4FB002010BDDC
:1044B0004400FF1F10B5044600F0E0FD204600F068
:1044C0001FFD204600F00EFD002010BD10B5024675
:1044D0000446497A00230620F9F71CFB034BB4225B
:1044E00002FB04346060002010BD00BFD800FF1F35
:1044F00000207047F0B50A88B1F9044083B004FB8E
:10450000002402AB0026A4B20D460746897843F882
:10451000046D20466A460096FBF794FF08B103B08D
:10452000F0BD03463A46697A0620F9F7F3FAAB790B
:10453000012B0AD0022B10D000906A46A978019B6B
:104540002046FBF7A5FF03B0F0BD054B53F827301D
:104550000146384698470090EFE7024BF6E700BF68
:104560004C86FF1F4886FF1F4FF48870704700BFBE
:10457000034A942303FB00230020DA6D1A66704778
:104580004400FF1F10B50246044600230321062005
:10459000F9F7C0FA154B014653F8243020469847E6
:1045A000002818D00BDD124A942303FB04240020BA
:1045B0006388C3F30E0343F48043638010BD0C4B48
:1045C000942202FB0434002063886FEA83436FEA7D
:1045D0009343638010BD064A942303FB0424002008
:1045E0006388C3F30D03638010BD00BF4C86FF1FBB
:1045F0004400FF1F0B4610B511460446184600F054
:10460000B3F928B1014620460B69BDE810401847B0
:1046100010BD00BF064A942303FB002340F215108F
:104620005B8803F06F03402B08BF0020704700BF7A
:104630004400FF1F00F058BF00207047204A942319
:1046400003FB002393F90E1093F90F308B4224D013
:1046500010B591B1062908D0012920D00A2904D02B
:1046600003290AD04FF4897010BD164CB42303FB04
:10467000004393F87430082B19D0942303FB0022D5
:10468000538803F06F03272B02D0D173002010BD95
:10469000044600F01FFF68B110BD00207047094CB0
:1046A000B42303FB004393F87430082BE5D140F2A8
:1046B000151010BD2046BDE8104000F0BBBE00BF85
:1046C0004400FF1FD800FF1F4FF48870704700BFE1
:1046D0004FF48870704700BF054A942303FB002005
:1046E000B0F90430042B0CBF4FF4847000207047E5
:1046F0004400FF1F0A4A0B4B12689A4202D04FF443
:104700008470704710B500240023E1B21A460720D8
:104710000134F9F7FFF9B4F5807FF5D1002010BD21
:104720001C23FF1F73617665024B01221A60002073
:10473000704700BF1C23FF1FF0B5B1F904500F886C
:1047400083B002AB4FF0000E064605FB00700C462E
:1047500043F804ED8978CDF800E0174680B26A4648
:10476000FBF786FB054670B9E379023B052B2BD896
:10477000DFE803F022260C1C1F0C144B304653F8C4
:10478000263098473860284603B0F0BD009B196872
:10479000A379012BF1D0022B18BF3960F3D10C4B58
:1047A000304653F8263098473860ECE7009B19787C
:1047B000EEE7009B1988EBE7009B93F90010E7E711
:1047C000009BB3F90010E3E70021E1E74486FF1FF7
:1047D0005086FF1F70B5114C942303FB004382B039
:1047E0005B8803F06F03402B18BF40F2151502D011
:1047F000284602B070BD02AA002342F8043D0E46CE
:104800000446FFF799FF05460028F1D12246717A48
:10481000019B0520F9F77EF9EAE700BF4400FF1F7E
:1048200070B582B002AA002342F8043D06460D4648
:10483000FFF782FF044628B93246697A019B0520BA
:10484000F9F768F9204602B070BD00BF70B582B0BC
:1048500002AA002342F8043D05460E46FFF76CFF0E
:10486000044640B90F4A942303FB05235A8802F0FB
:104870006F02272A02D0204602B070BD93F90F3094
:1048800023F00203012BF6D1717A019B2A46052001
:10489000F9F740F928460199FFF706FD204602B0D6
:1048A00070BD00BF4400FF1F30B583B002AA0023D3
:1048B00042F8043D0546FFF73FFF044660B9084A49
:1048C000942303FB05235B8803F06703072B03D1C5
:1048D00028460199FFF7E8FC204603B030BD00BF31
:1048E0004400FF1F10B5044600F0F0FB034B942278
:1048F00002FB0434A061002010BD00BF4400FF1F74
:1049000070B5184E338853B30546344605E00BB1F5
:10491000E368984734F8183F53B1012DA388214626
:104920002846F4D1002BF3D034F8183F002BF4D1F3
:104930003388012D14BF0426072683B1094C02E0F9
:1049400034F8183F63B1237AB342F9D1214628469F
:10495000FFF766FF238B18340BB10028F3D070BD2E
:1049600070BD00BF0818FF1F094B10B41A88044619
:1049700002E033F8182F3AB194421846F9D19A78E8
:104980008A42F6D110BC7047104610BC704700BF79
:104990000818FF1F2DE9F04182B002AB002423F874
:1049A000024D1D4E884619461746FFF73DFD96F805
:1049B0009920BDF806E06AB3012102E08A4216D9C7
:1049C000E1B24B1EDBB24C1C16F833508542F5D1D8
:1049D00006EBC3035D887545F0D11D794545EDD1E2
:1049E0003B44012200205A7102B0BDE8F081541C02
:1049F000E4B206EBC201CB1906F832000122002016
:104A0000A1F802E081F8048086F899405A7102B05A
:104A1000BDE8F0810124ECE70037FF1F38B5124CE8
:104A200094F8983014F8335004EBC30328461A79ED
:104A30005988FFF71FFD94F8983004EBC30146F244
:104A400064024988914208D094F899200133934236
:104A500008BF002384F8983038BD044A942101FB34
:104A60000525AA696A61EFE70037FF1F4400FF1FB1
:104A70002A4900222DE9F0470B4681F8982001F1E0
:104A800098044A800831A1424FF00000F9D1012179
:104A900046F2FD0A46F2620946F2640846F26B0CE1
:104AA00046F26C0E46F2740746F2770642F20D05A6
:104AB000082418701A711A721A731A741A751A76F1
:104AC0001A7783F8202083F8242083F8282083F89D
:104AD0002C2083F8302083F8342083F8382083F8A2
:104AE0003C20A3F802A0997199739975997783F87E
:104AF000261083F82E1083F8361083F83E10A3F8A2
:104B00000A90A3F81280A3F81AC0A3F822E05F85E8
:104B10005E865D8783F89940BDE8F0870037FF1F08
:104B20002DE9F04383B002AB002423F8024D0F4679
:104B300019461646FFF778FC344BBDF8069093F8FB
:104B400099809C466246234608F1010503E0AB428A
:104B500002F108020CD011788142DCB29E4603F1CA
:104B60000103F4D151884945F1D11179B942EED10F
:104B7000444543D04FEACE000CEB00031E44002214
:104B800072715A79B2BB9B79A3BB9CF89870BC42F6
:104B900008F1FF3605D2B64503DA013FFFB28CF8C3
:104BA0009870631CDAB242451AD25FFA86F800E0C8
:104BB0000133DBB2D8000CEB00010CEBC4024D79E1
:104BC00055711CF83350B1F802E00CF83450984598
:104BD0000D798979A2F802E01C4615719171E7D12F
:104BE0000CEB0003F6B20020BE428CF899605880AE
:104BF000187108D0002003B0BDE8F08340F20B101C
:104C000003B0BDE8F0838CF89800F9E70037FF1F88
:104C1000084670470846704770B40849084E094D69
:104C2000094C0A4A0A4B46F8202045F8202044F84F
:104C3000203041F8203070BC704700BF4886FF1F0D
:104C40004486FF1F4C86FF1F5086FF1F114C01003A
:104C5000154C01002DE9F047DFF858E1942101FBE4
:104C600000E191F90F90B9F1060F7ED04300DFF813
:104C70003CC189691A180CEB8202D2F808A0514590
:104C80003CDD494EC2001644D6E9004545F0040516
:104C9000C6E9004503440CEB830CDCF804308B427E
:104CA00058DCDFF8148108EB0203D3E90045002645
:104CB00005F0080756EA07031DD03C493C4E00EBBF
:104CC000400301EB8301942303FB00EE4B6856F88D
:104CD0002000DEF81810034499420CDB324B1344D9
:104CE000D3E90001424425F0080521F00801C2E99A
:104CF0000045C3E900010020BDE8F087DFF8B88077
:104D0000C20008EB0204D4E90045002605F00407C0
:104D10003E43BFD0264E56F82060AAEB060A514506
:104D2000B8DC214B1344D3E9006725F0040508EBF8
:104D3000020A27F00407B9F1060FCAE90045C3E9E2
:104D400000672CD0430003440CEB830CDCF80430E8
:104D50008B42A6DD144B1A44D2E9000141F0080150
:104D6000C2E900010020BDE8F087DFF84C80C200F6
:104D700008EB0203D3E90045002605F0040756EAD4
:104D8000070394D00A4BDFF824C053F820608969E8
:104D90000C2303FB00C39B689B1B9942C1DD08EBFE
:104DA0000203D3E9004582E71086FF1F5886FF1FE4
:104DB0006C86FF1F4400FF1F2086FF1F012930B4AF
:104DC0001FD0022902D0002030BC7047234C244958
:104DD0009422B42302FB004203FB0013D26CD3F8ED
:104DE000B0306FF000418D1A5C42A5422DDB1D49A9
:104DF00000EB400001EB8000D21A826030BC002042
:104E00007047164D164C9422B42302FB005203FB4C
:104E10000043926CD3F8B03001F100418D1A5C422E
:104E2000A54208DD0F4B00EB400003EB800030BCD7
:104E30004160002070470B4900EB400001EB80000F
:104E4000D21A426030BC00207047064B00EB400095
:104E500003EB800030BC8160002070474400FF1FDE
:104E6000D800FF1F5886FF1F08B58978FFF7A6FFF7
:104E7000002008BD0B4A08B5942303FB0023897862
:104E80009A6CDB6C9A4203DB012905D0022906D01B
:104E9000FFF794FF002008BD4FF4877008BD40F273
:104EA0000D1008BD4400FF1F10B58C78013CE1B225
:104EB000002301220F20F8F72DFE024B43F82400B7
:104EC000002010BD0023FF1F08B500231A46FF2154
:104ED0000F20F8F71FFE024B1860002008BD00BF2E
:104EE0002023FF1F054A942303FB00230020D3F84F
:104EF000842022F00402C3F8842070474400FF1F7E
:104F00002DE9F04702460446002314210620F8F755
:104F100001FE22460023152105460620F8F7FAFD7A
:104F2000524A534E4FF0940EB4230EFB042E03FB53
:104F300004F3DEF88410F35821F0030C9907CEF83F
:104F400084C040D4690001F0020141EA0C0113F071
:104F50000103CEF8841005D100F0010C4CEA0101E8
:104F6000CEF88410002D66D0942101FB04214D88D9
:104F700005F02F0565B191F90F1006295BD03D4969
:104F800001EBC401D1E9006747F01007C1E90067F0
:104F9000002B37D1002835D0942303FB04225388FB
:104FA00003F02F0363B192F90F30062B2AD0314B57
:104FB00003EBC404D4E9002343F02003C4E9002335
:104FC0000020BDE8F0872C49E5004E1913F00103DD
:104FD000D6E900673CD04FF0000807F0100958EA06
:104FE000090E11D0DFF88CE0AE44DEE900892944D7
:104FF00027F0100729F01009C1E90067CEE9008900
:10500000002BC7D01C49E5004C19D4E9002300202F
:1050100003F020010143D3D016480544D5E900012F
:1050200023F0200321F02001C5E90001C4E9002399
:105030000020BDE8F0871049E5004E19D6E9006769
:105040004FF0000807F0100958EA090ECAD19FE78F
:1050500000F0010A4FF0000807F010094AEA0C0CB2
:10506000CEF884C058EA090EBCD193E74400FF1F74
:10507000D800FF1F1086FF1F2086FF1F054A9423BC
:1050800003FB00230020D3F8842022F00802C3F899
:10509000842070474400FF1F38B50546FFF7BAFA71
:1050A000044678B9B423084A03FB05F30520D35816
:1050B000590801F00201C3F3C0030B432A46A6219D
:1050C000F8F728FD204638BDD800FF1F0246002310
:1050D00001210620F8F71EBD002070470020704710
:1050E0000C4A942303FB002393F90F30013B092B57
:1050F0000CD8DFE803F0090B070B0B050B0B0B0CAF
:1051000001F0CEBA00F044BE00F0BCBD704700F024
:1051100087BB00BF4400FF1F2DE9F041B54D35F8B6
:105120001030D907044639D49A0700F184805F070C
:105130003FD41E0700F1918013F0200640F0A580B7
:1051400059064BD4DA0500F1D6809F0500F1B780EF
:105150005E0500F1A480180500F10781D90400F173
:1051600014819A0400F121815B0400F12E81A24A8E
:10517000942303FB04235A8802F06F02272A23D1C9
:1051800093F90F30012B00F03081062B00F02881BD
:10519000D3B92046BDE8F04100F010BC0121FEF774
:1051A000C7FF98B101280FD0002325F81430BDE8BF
:1051B000F081914B942606FB00360321726EFFF7B7
:1051C00083F8012800F08B80BDE8F08135F81430B9
:1051D00023F0010325F81430BDE8F081FEF7C0FF8D
:1051E00001280746F0D12046FFF71AF8824B4FF00E
:1051F000940808FB043898F90E300A2B13D0324675
:1052000046F264012046FFF735F93146D8F81830E8
:1052100022460520F8F77EFCD8F818303946224699
:105220000520F8F777FC35F8143023F0400325F813
:105230001430BDE8F08101F0C3FB6F4A35F814105B
:10524000942303FB042321F002015A8825F814104B
:1052500042F480625A80BDE8F081684B032153F824
:105260002020FFF731F80128AED1634A35F8141039
:10527000942303FB042321F008015A8825F8141015
:1052800042F480625A80BDE8F081FEF753FF35F8A2
:10529000143023F0200325F81430BDE8F08156497E
:1052A000942202FB001223F48061538825F8101029
:1052B00023F06F0343F021035380BDE8F0814E4992
:1052C000942202FB001223F40071538825F8101079
:1052D00023F06F0343F040035380BDE8F0817288F0
:1052E00035F8143042F4806223F00403728025F80C
:1052F0001430BDE8F0814049942202FB001292F97B
:105300000E200A2A0ED8DFE802F02B230D1B0D0D0C
:10531000130D0D0D060000F089FA204600F06AFA20
:1053200035F8143023F4807325F81430BDE8F0818B
:1053300001F0EAF9204600F055FE35F81430F1E7A7
:1053400000F032FD204600F00DFD35F81430E9E79D
:1053500000F0C4FC204600F0F9FB35F81430E1E71A
:1053600000F046FB35F81430DCE72349942202FBB9
:10537000041223F40061538825F8141023F06F03FE
:1053800043F023035380BDE8F0811B49942202FBC4
:10539000041223F48051538825F8141023F06F036E
:1053A00043F027035380BDE8F0811349942202FBA8
:1053B000041223F40051538825F8141023F06F03CE
:1053C00043F007035380BDE8F0812046FFF788FED5
:1053D00035F8143023F4804325F81430BDE8F0810B
:1053E0002046BDE8F04100F07FBF2046BDE8F04117
:1053F00000F028BC9C37FF1F4400FF1F6486FF1F7E
:1054000038B50A4B03EB40024FF6FF710025044606
:1054100023F81050918001F043F9054B942202FBD0
:1054200004344FF40473638038BD00BF9C37FF1F02
:105430004400FF1F38B5264D0446FFF751FE942364
:1054400003FB045393F90E300A2B3ED8DFE803F038
:1054500013333D1C3D3D293D3D3D0600204600F0F7
:10546000E5F9204600F0C6F988BB942303FB0454F9
:105470000A23E37338BD204600F0BAFA942303FBF5
:1054800004540020E07338BD204600F08DFC204617
:1054900000F068FCD8B9942303FB04540323E3739E
:1054A00038BD204601F014F988B9942303FB045455
:1054B0000623E37338BD204600F0F0FB38B994238F
:1054C00003FB04540123E37338BD4FF4847038BDEB
:1054D0004400FF1F032905D00A2901D100F0B2B909
:1054E0000020704700F06CBC2DE9F84FB84DB94F63
:1054F000942303FB00F3EE1835F803E0738827F8D4
:1055000010E013F06F01024607D1B34B4FF40C7457
:10551000084623F81240BDE8F88FDFF8BC924FEA46
:10552000400809EB080A4029BAF804C004460EF006
:105530008F020CF08F0B0CD10EF0870EBEF1060F10
:1055400000F089805A4514BF4FF489700020BDE8EF
:10555000F88F212919D023293AD0272947D00729A4
:1055600059D0082974D11EF0800FEBD0FEF774FDDE
:10557000738837F81420AAF8042023F06F0343F04F
:10558000400373800020BDE8F88F072A16D00F2A49
:105590004FD00EF08601022902D01EF0820FD1D129
:1055A0009422C84402FB045423F06F0343F04003E9
:1055B000A8F804E063800020BDE8F88F23F06F03B3
:1055C00043F023037380AAF804E00020BDE8F88FBD
:1055D0000F2A2ED00EF087010629DAD14FF484630A
:1055E00029F81030AAF804E00020BDE8F88F072A57
:1055F00051D00EF08703062B56D01EF0820042D009
:105600000EF08603022B58D05A4500F0A9804FF4C3
:105610008970BDE8F88F1EF082002CD00F2A91D13E
:105620004FF48853AAF804E029F814300020BDE8AC
:10563000F88F96F90F10FFF74DFF50B937F8143077
:10564000AAF804304FF48E5329F81430BDE8F88FCF
:105650000020BDE8F88F0021FEF76AFD0128F8D888
:1056600037F81430AAF8043040F2014329F8143016
:105670000020BDE8F88F4FF40C73AAF804E029F875
:105680001430BDE8F88F44F23823AAF804E029F872
:105690001430BDE8F88F44F6380329F81030AAF822
:1056A00004E00020BDE8F88F44F2384329F81030B8
:1056B000AAF804E00020BDE8F88FB6F90430013BF9
:1056C000062BA4D801A252F823F000BF4D570100C9
:1056D00039570100255701000F56010011570100ED
:1056E000FD560100E9560100C84446F20203A8F83D
:1056F00004E029F814300020BDE8F88FC84446F2D1
:105700000403A8F804E029F814300020BDE8F88F5D
:10571000C84446F20803A8F804E029F81430002031
:10572000BDE8F88FC84444F23223A8F804E029F811
:1057300014300020BDE8F88FC84444F23423A8F8A0
:1057400004E029F814300020BDE8F88FC84444F282
:105750003823A8F804E029F814300020BDE8F88FB9
:105760000EF45C7E0CF45C7CE6453FF471AF942350
:1057700003FB045595F90F300A2B24D8DFE803F01A
:105780001F1B23172323132323230600204600F087
:1057900031F800287FF45DAFC84437F81430A8F81A
:1057A0000430BDE8F88F204600F01CFCF1E72046ED
:1057B00000F0D8FAEDE7204600F0C8F9E9E7204606
:1057C00000F0FAF8E5E74FF48470BDE8F88F00BF09
:1057D0004400FF1F6886FF1F9C37FF1F044B33F8F0
:1057E000100000F00E00003018BF0120704700BF0D
:1057F0009C37FF1F10B50446FFF7F0FF58B9074B61
:10580000942101FB04312246086BCB6F9B2103449A
:105810000520F8F77FF9002010BD00BF4400FF1FEE
:10582000024600239B210520F8F774B9044A94230B
:1058300003FB0020438843F480534380704700BF3C
:105840004400FF1F284B03EBC003D3E9002330B40F
:10585000002403F0040554EA050121D0234C9421CF
:1058600001FB0041096B00291ADD002403F010053B
:1058700054EA050140F2151127D1002203F020035C
:10588000134322D0194A942303FB002040F215133E
:10589000026B31EA220128BF1946084630BC704726
:1058A000002403F0080554EA050111D10021002469
:1058B00003F010052C43E0D00C4D942404FB00545D
:1058C000246B002CD9DD40F21511084630BC70471E
:1058D0000649942404FB001440F21511246B002C9B
:1058E000A8BF0021E3E700BF1086FF1F4400FF1F91
:1058F00070B582B002AA002342F8043D0646FEF7C6
:105900001BFF134A019B942404FB06240546E26F07
:105910001344019348B93046FFF794FF054620B978
:10592000638803F06F03272B02D0284602B070BDB6
:1059300094F90F300A2BF8D13046FFF74FFF0028BB
:10594000F3D13246019B9B210520F8F7E3F8ECE701
:105950004400FF1F70B582B002AA002342F8043D44
:105960000646FEF7E9FE134A019B942404FB062435
:105970000546226B1344019348B93046FFF762FF96
:10598000054620B9638803F06F03272B02D0284611
:1059900002B070BD94F90F300A2BF8D13046FFF7F2
:1059A0001DFF0028F3D13246019B9B210520F8F70B
:1059B000B1F8ECE74400FF1F002070470A4A10B519
:1059C000942404FB00246288530500D510BD074AC7
:1059D000072152F82020FEF777FC0128F6D16388D2
:1059E00043F48063638010BD4400FF1F6486FF1F83
:1059F000044A942303FB0020438823F4505343803C
:105A0000704700BF4400FF1F402A22D01F4B00EB0D
:105A1000400203EB82039A68914202DB40F21510C8
:105A200070475B689942F9DD194B03EBC003D3E97A
:105A3000002330B4002403F010052C4311D0154D81
:105A4000942404FB0054A469A1420ADB40F215101F
:105A500017E0104A942303FB00239A69196C114440
:105A6000D4E7002203F0200313430CD0094B942207
:105A700002FB003040F2151380698142D4BF184602
:105A8000002030BC70470020FBE700BF5886FF1F96
:105A90001086FF1F4400FF1F10B50446FEF72AFDC5
:105AA0000449054A942303FB04131B6A42F824307B
:105AB00010BD00BF4400FF1F6C86FF1F0E4A9423D9
:105AC00003FB002310B51A6A531C0FD0002A0ADB0F
:105AD0000A4C44F8202013460246497A0520F8F77C
:105AE00019F8002010BD4FF4877010BD034A002341
:105AF00042F82030F0E700BF4400FF1F6C86FF1F14
:105B000070B582B002AA002342F8043D05460E4655
:105B1000FEF712FE044640B90B4A942303FB05230B
:105B20005A8802F06F02272A02D0204602B070BDC8
:105B300093F90F30012BF8D12A46717A019B052089
:105B4000F7F7E8FFF1E700BF4400FF1F2DE9F0433E
:105B50002A4B2B4E33F81020942712F0400283B0CA
:105B6000044607FB00670BD1D7F840804146FFF79A
:105B70004BFF0546002836D0284603B0BDE8F08329
:105B8000D7F8408040224146FFF73EFF0546814658
:105B90000028F1D1FB6D796DCDF8048001201A4603
:105BA00000902046FEF742FB4B46054622464946FA
:105BB0000620F7F7AFFF002DDED11248942101FB3C
:105BC000046130F814204B8822F0020242F00102F6
:105BD00023F4806343F4805320F8142028464B803C
:105BE00003B0BDE8F083FB6D796D1A468DE82001A6
:105BF0002046FEF71BFB0546DDE700BF6886FF1F5A
:105C00004400FF1F7086FF1F0D4A942303FB0023EF
:105C10005A8802F06F02272A01D00020704793F9BA
:105C20000F30012BF9D110B50446FFF7D7FD08B1AD
:105C3000002010BD2046BDE81040FFF787BF00BF21
:105C40004400FF1F0D4B33F8103013F0020300D057
:105C50007047024610B59C2104460620F7F75AFF0C
:105C6000074B942202FB04340009638800F480602F
:105C700023F480631843608010BD00BF7086FF1F4F
:105C80004400FF1F044A942303FB0020438823F4AD
:105C900040534380704700BF4400FF1F0C4A0D4B28
:105CA00032F81020D20648BF03224FF0020123F839
:105CB000101048BF23F81020074B942202FB00333A
:105CC00000205A8822F4405242F480625A80704781
:105CD0006886FF1F7086FF1F4400FF1F084B09499D
:105CE000942202FB003210B4538823F44053022460
:105CF00043F4806321F81040538010BC704700BF0C
:105D00004400FF1F7086FF1F10B502460446497A03
:105D100000230620F7F7FEFE104B014653F824300F
:105D2000204698470E4B942202FB04346388E062BD
:105D300003F06F02272A01D0002010BD94F90F2034
:105D4000032AF9D1D4F8882090420CBF43F4806331
:105D500023F480636380002010BD00BF4C86FF1FCA
:105D60004400FF1F10B50446FFF738FD08B10020BE
:105D700010BD064B942202FB04322046D36DD2F8AC
:105D80008810BDE810401A46FEF714BA4400FF1F01
:105D9000044A942303FB00230021DB6D1A46FEF71F
:105DA00009BA00BF4400FF1F044A942303FB0020EC
:105DB000438823F450534380704700BF4400FF1FC3
:105DC0002A4B03EBC003D3E9002330B4002403F0D3
:105DD000040554EA050123D0254C942101FB004120
:105DE000D1F8881000291BDD002403F0100554EAC7
:105DF000050140F2151129D1002203F020031343BD
:105E000024D01B4A942303FB002040F21513D0F842
:105E1000882031EA220128BF1946084630BC704765
:105E2000002403F0080554EA050112D100210024E2
:105E300003F010052C43DFD00D4D942404FB0054D7
:105E4000D4F88840002CD7DD40F21511084630BC4C
:105E500070470749942404FB001440F21511D4F84C
:105E60008840002CA8BF0021E1E700BF1086FF1F7B
:105E70004400FF1F30B583B002AA002342F8043D5E
:105E80000546FEF759FC044668B92846FFF798FF17
:105E9000044640B90D4A942303FB05235A8802F0B7
:105EA0006F02272A02D0204603B030BD93F90F308D
:105EB000032BF8D12846FFF791FC0028F3D12A469E
:105EC000019B02210520F7F725FEECE74400FF1FA8
:105ED00070B582B002AA002342F8043D05460E4682
:105EE000FEF72AFC044640B90B4A942303FB052322
:105EF0005A8802F06F02272A02D0204602B070BDF5
:105F000093F90F30062BF8D12A46717A019B0520B0
:105F1000F7F700FEF1E700BF4400FF1F1C4A94237F
:105F200003FB002393F96830232B2DD8DFE803F01F
:105F3000122C2C2C2C2C2C2C2C2C2C2C2C2C2C2CBB
:105F40002C20142C2C2C2C2C2C2C2C2C2C2C2C2CB5
:105F50002C2C2C1200207047B42303FB00F00D4BB7
:105F60001B5813F0020F40F2151008BF00207047B5
:105F7000B42303FB00F0074B1B5813F0010F40F252
:105F8000151008BF002070474FF48470704700BFA1
:105F90004400FF1FD800FF1F70B582B002AA002383
:105FA00042F8043D05460E46FEF7C6FB044618B906
:105FB0000B4B5A5D012A02D0204602B070BD5A191F
:105FC000B17812799142F7D103EB850301989B6870
:105FD000717A00FB03F32A460520F7F79BFDEBE7F8
:105FE000A437FF1F9E4B33F8103013F01003F0B5A9
:105FF00004D09C4B1A5CC2B10020F0BD994A115CE0
:106000000029F9D0984C1354942101FB0041151834
:106010004C882B7102EB800024F440524FF40004B2
:10602000836004614A800020F0BD8F4D942404FBFE
:1060300000548100D4F884E094F968605F181C185B
:10604000C7F80CE0BA602271232E3AD8DFE816F0C8
:10605000D500AA00B70085003900C6003900390014
:106060003900390039003900390039003900390068
:10607000390099002400700039005C0039003900B3
:106080003900390039003900390039003900390048
:1060900039005200490044005A18744C14611EF033
:1060A000020F4FF00204546100F0CF80704C146175
:1060B0004FF0FF34946119444FF0FF340122CC615A
:1060C0000A62942202FB0052012451881C5421F4DC
:1060D000505353800020F0BD19444FF440020A6130
:1060E000EFE719444FF4E006002401220E614C61F1
:1060F0000A62E6E719444FF4E00600244FF0FF324D
:106100000E614C610A62DCE75A18584C14611EF0AB
:10611000020F4FF00404546174D04FF0FF36554C19
:1061200096611461194401240022CC610A62C8E717
:106130005A184E4C14611EF0020F4FF004045461C3
:106140007BD04FF0FF364B4C9661146119444FF0F1
:10615000FF340022CC610A62B3E75A18464C14613E
:106160001EF0020F4FF00404546159D04FF0FF3677
:10617000424C9661146119444FF0FF32CA610A62C1
:106180009FE75A18394C14611EF0010F4FF00104BB
:1061900054615FD0364E9461166119440122CA6180
:1061A0000A628EE75A18344C14611EF0010F4FF04A
:1061B000010454612ED0324E94611661EDE75A18F5
:1061C0002D4C14611EF0020F4FF0020454612FD0C9
:1061D0002B4C14614FF0FF349461CCE75A18264CD5
:1061E00014611EF0020F4FF00404546152D04FF0BE
:1061F000FF36224C96611461CFE719444FF4000238
:106200000A615EE71EF0010F5CD00126194C966111
:10621000146187E74FF0FF361A4C96611461BCE7B2
:106220001EF0010F56D00126144C96611461A2E7AE
:106230000126154C966114619DE71EF0010F31D0C7
:1062400001260C4C9661146180E701260F4C966183
:10625000146130E74FF0FF360D4C966114619CE7F6
:106260006886FF1FA437FF1F4400FF1FF303400091
:1062700000034000EF034000F3037000EF037000E1
:1062800000037000E7037000EB037000EB034000B5
:10629000E70340001EF0010F0CD00126114C96615F
:1062A00014617AE71EF0040F0CBF01244FF0FF3495
:1062B00094614BE71EF0040F0CBF4FF0FF34012434
:1062C00094616AE71EF0040F0CBF4FF0FF34012405
:1062D000946127E71EF0040F0CBF01244FF0FF3438
:1062E000946148E7EF0370002DE9F043B84E870052
:1062F000F41983B0226912F0F30F05460FD112F49E
:10630000407178D112F4401F58D112F4000340F0CC
:10631000A880520200F1DB8003B0BDE8F083D30710
:1063200000F10081910740F1B080DFF8ACE2E16854
:106330006369942000FB05E0D0F8840080EA010E38
:106340001EEA030F1CBF22F01E022261820740F1E9
:10635000FF800B4313F0020313D1F419226912F0EA
:10636000040F00F089819B4A236102EBC504D4E944
:10637000002343F01003C4E90023F31941F00201A4
:10638000D960C20740F10581CB07C5D4F219536922
:1063900013F00103C0D11069040740F173818D48E7
:1063A000136100EBC505D5E9002343F02003C5E9DF
:1063B00000233E4441F00101F160ADE712F4801387
:1063C00040F00E819002A7D59C212A460620F7F7BF
:1063D000A1FBC106A0D52846FDF722FF7E49226910
:1063E000942303FB051522F400126B88226143F409
:1063F00080536B8090E7D10500F1D38092058BD557
:10640000754A63694FF0940909FB0029D9F8841093
:1064100011EA030800F00E818B070ED5F2195369BB
:1064200013F0020309D16B48136100EBC500D0E9FA
:10643000002343F01003C0E90023CC077FF56CAFC5
:106440003E44736913F001037FF466AF614A336120
:1064500002EBC505D5E9002343F02003C5E900237D
:106460005AE75D4A942303FB002506216A6FFDF776
:106470002BFF01287FF450AF6A88236942F48062C1
:1064800023F400036A80236146E7D30600F1BD8050
:10649000910665D412F0400940F0D88013067FF5CC
:1064A0003BAF4D4A63694FF0940808FB0028D8F8C9
:1064B00084101942B0D000F083FA2269D8F8841011
:1064C000731922F08002226183F80490A4E7024647
:1064D00003210620F7F71EFB00287FF41DAF3E4B7B
:1064E0003E4A942606FB0536B42303FB0523726C53
:1064F000C3F8B02001212846FEF760FC022128469F
:10650000FEF75CFC736C2A465B4201210520F7F71D
:1065100001FB7288236942F4A05223F48003728045
:106520002361F9E62C4BA169942202FB0032354429
:10653000536FD26E01FB02F11A46FDF73BFE236951
:10654000A269A26023F0010301222A712361E3E61C
:106550008C077FF516AFF31921F00201D96010E71F
:106560001D4A942303FB002505216A6FFDF7ACFE4D
:1065700001287FF4D1AED5F8842063691A4200F077
:106580008780236923F0C0033E4423F02003336156
:10659000C2E6CA077FF5C0AE3E4421F00101F160BA
:1065A000BAE60D4BE169942202FB00323544536F89
:1065B000126F01FB02F11A46FDF7FCFD2369E26947
:1065C000A26023F4807302222A712361A4E600BF33
:1065D000A437FF1F1086FF1F4400FF1FD800FF1FB6
:1065E0002E4B0191942202FB00320091536F116FE8
:1065F0001A46FDF71BFE2369226AA2603544022277
:1066000023F480132A71236186E6244A942303FB32
:10661000002504216A6FFDF757FE01287FF47CAE48
:106620002369A26923F0100343F00303524223615C
:10663000A26171E600F0C4F92269D9F884107319D7
:1066400022F40072226183F80480E5E6134BA1690D
:10665000942202FB00323544536F126F01FB02F1AA
:106660001A46FDF7A7FD2369A269A26023F0400343
:1066700002222A7123614FE622F0020343F00C0349
:1066800023617AE620F0020343F00C03136190E6E5
:10669000A26923695242A26176E700BF4400FF1F4E
:1066A000094B942270B402FB0032084C5188261822
:1066B000002304EB800521F4405133712354AB6077
:1066C0002B61518070BC70474400FF1FA437FF1F2F
:1066D0000A4B0B4A33F810300A4913F0100318BF65
:1066E00001231354942303FB001302EB8002598807
:1066F000002021F450511061598070476886FF1FB7
:10670000A437FF1F4400FF1F084A942330B403FB43
:106710000023074C5A8804EB8005002122F45052D4
:10672000215429615A8030BC704700BF4400FF1FCC
:10673000A437FF1F014B01221A707047C837FF1F93
:1067400030B583B002AB002023F8020D084619468D
:106750001446FDF769FEBDF80610B1F5005F0CD2D6
:10676000B1F5B05F06D041F61243994202D0002045
:1067700003B030BD00F0B8F8F9E722460546FDF752
:1067800039FF0028F4D1BDF8062046F240039A42B2
:10679000EDD1054B0549942202FB05F203EB4505BB
:1067A0008B5AAB80E4E700BFC837FF1F4400FF1FD0
:1067B00030B583B002AB002423F8024D08461946D9
:1067C0001546FDF731FEBDF80610B1F5005F02D2A7
:1067D000204603B030BD2A46FDF74CFE03B030BD65
:1067E000431E032B14D8DFE803F002020202094B18
:1067F0009A79082A01D098717047074A30B4D2E9D3
:106800000245987144F00064C2E9024530BC70470B
:10681000004BF0E7C837FF1F1086FF1F024B012215
:10682000DA710020704700BFC837FF1F704700BFF4
:1068300000207047704700BF2DE9F041214E3378AA
:1068400082B093B3204C214FDFF88480002304F101
:106850002005337010E046F26003994228D0A278F8
:10686000FDF7C8FE28B1D7E9022342F00402C7E9C8
:1068700002230434AC4218D02088B0B10DF10601D7
:10688000FDF7D2FDBDF8061046F240039942E2D171
:10689000942303FB00F306EB400238F80330B2F810
:1068A00004E09E45E5D09380D9E702B0BDE8F081D1
:1068B000942303FB008393F90E2093F90F309A423F
:1068C000CDD1D6E7C837FF1F7486FF1F1086FF1F84
:1068D0004400FF1F034BD87910B10022DA71012068
:1068E000704700BFC837FF1F2DE9F043DFF8B880BD
:1068F00085B00024434608F120021C809C700433BC
:106900009342FAD104AF01AA47F8044D00213B4657
:1069100041F612400194F9F795FDC0B9019BB3B15E
:106920000546012400E0144602AA3B46E1B241F6C6
:10693000124002950395F9F785FD621C064618B9C9
:106940000298B0F5B05F05D0019BA342EBD805B02B
:10695000BDE8F08331463B4602AA02960396F9F75A
:1069600071FD0028F3D1029E002EF0D0054681462D
:10697000012401E0A642EAD302AA3B4621464FF495
:10698000B050CDF80890F9F75DFD08EB850230B9FD
:10699000029B190C1B0A28F825109370013501344D
:1069A000072DE4B2E6D9D2E77486FF1FF2F708BAE2
:1069B00008B5F8F73DFABDE80840F2F719BA00BF8C
:1069C00008B5F8F735FABDE80840F2F711BA00BF8C
:1069D000F6F7A8BDF3F7F4BAF3F718BBF7F746B824
:1069E000034613F8012B002AFBD1181A013870470F
:1069F00081F0004102E000BF83F0004330B54FEA70
:106A000041044FEA430594EA050F08BF90EA020FDC
:106A10001FBF54EA000C55EA020C7FEA645C7FEA6F
:106A2000655C00F0E2804FEA5454D4EB5555B8BF92
:106A30006D420CDD2C4480EA020281EA030382EA03
:106A4000000083EA010180EA020281EA0303362D95
:106A500088BF30BD11F0004F4FEA01314FF4801C68
:106A60004CEA113102D0404261EB410113F0004F7A
:106A70004FEA03334CEA133302D0524263EB430331
:106A800094EA050F00F0A780A4F10104D5F1200ECF
:106A90000DDB02FA0EFC22FA05F2801841F100012A
:106AA00003FA0EF2801843FA05F359410EE0A5F1FE
:106AB00020050EF1200E012A03FA0EFC28BF4CF02F
:106AC000020C43FA05F3C01851EBE37101F00045E5
:106AD00007D54FF0000EDCF1000C7EEB00006EEBF2
:106AE0000101B1F5801F1BD3B1F5001F0CD349087C
:106AF0005FEA30004FEA3C0C04F101044FEA4452D3
:106B000012F5800F80F09A80BCF1004F08BF5FEA59
:106B1000500C50F1000041EB045141EA050130BD39
:106B20005FEA4C0C404141EB010111F4801FA4F1DC
:106B30000104E9D191F0000F04BF01460020B1FA31
:106B400081F308BF2033A3F10B03B3F120020CDA69
:106B50000C3208DD02F1140CC2F10C0201FA0CF047
:106B600021FA02F10CE002F11402D8BFC2F1200CAC
:106B700001FA02F120FA0CFCDCBF41EA0C01904062
:106B8000E41AA2BF01EB0451294330BD6FEA0404AB
:106B90001F3C1CDA0C340EDC04F11404C4F1200296
:106BA00020FA04F001FA02F340EA030021FA04F3A8
:106BB00045EA030130BDC4F10C04C4F1200220FAFF
:106BC00002F001FA04F340EA0300294630BD21FA3D
:106BD00004F0294630BD94F0000F83F4801306BF03
:106BE00081F480110134013D4EE77FEA645C18BFF7
:106BF0007FEA655C29D094EA050F08BF90EA020F8E
:106C000005D054EA000C04BF1946104630BD91EA85
:106C1000030F1EBF0021002030BD5FEA545C05D188
:106C20004000494128BF41F0004130BD14F58004C7
:106C30003CBF01F5801130BD01F0004545F0FE413B
:106C400041F470014FF0000030BD7FEA645C1ABF70
:106C5000194610467FEA655C1CBF0B46024650EAA7
:106C6000013406BF52EA033591EA030F41F40021D3
:106C700030BD00BF90F0000F04BF0021704730B559
:106C80004FF4806404F132044FF000054FF000012E
:106C900050E700BF90F0000F04BF0021704730B5EF
:106CA0004FF4806404F1320410F0004548BF4042C4
:106CB0004FF000013EE700BF42004FEAE2014FEA19
:106CC00031014FEA02701FBF12F07F4393F07F4FF4
:106CD00081F06051704792F0000F14BF93F07F4F26
:106CE000704730B54FF4607401F0004521F0004169
:106CF00020E700BF50EA010208BF704730B54FF0EF
:106D000000050AE050EA010208BF704730B511F0F3
:106D1000004502D5404261EB41014FF4806404F12B
:106D200032045FEA915C3FF4DCAE4FF003025FEAAD
:106D3000DC0C18BF03325FEADC0C18BF033202EB35
:106D4000DC02C2F1200300FA03FC20FA02F001FA8F
:106D500003FE40EA0E0021FA02F11444C1E600BF2E
:106D600070B54FF0FF0C4CF4E06C1CEA11541DBFE1
:106D70001CEA135594EA0C0F95EA0C0F00F0DEF8AC
:106D80002C4481EA030621EA4C5123EA4C5350EA91
:106D9000013518BF52EA033541F4801143F48013E2
:106DA00038D0A0FB02CE4FF00005E1FB02E506F073
:106DB0000042E0FB03E54FF00006E1FB03569CF0C8
:106DC000000F18BF4EF0010EA4F1FF04B6F5007FCE
:106DD00064F5407404D25FEA4E0E6D4146EB060640
:106DE00042EAC62141EA55514FEAC52040EA5E50C9
:106DF0004FEACE2EB4F1FD0C88BFBCF5E06F1ED873
:106E0000BEF1004F08BF5FEA500E50F1000041EBA9
:106E1000045170BD06F0004646EA010140EA020056
:106E200081EA0301B4EB5C04C2BFD4EB0C0541EA78
:106E3000045170BD41F480114FF0000E013C00F38D
:106E4000AB8014F1360FDEBF002001F0004170BDB1
:106E5000C4F10004203C35DA0C341BDC04F11404CA
:106E6000C4F1200500FA05F320FA04F001FA05F256
:106E700040EA020001F0004221F0004110EBD37023
:106E800021FA04F642EB06015EEA430E08BF20EA4F
:106E9000D37070BDC4F10C04C4F1200500FA04F3F2
:106EA00020FA05F001FA04F240EA020001F0004184
:106EB00010EBD37041F100015EEA430E08BF20EAF7
:106EC000D37070BDC4F1200500FA05F24EEA020E3F
:106ED00020FA04F301FA05F243EA020321FA04F06E
:106EE00001F0004121FA04F220EA020000EBD37025
:106EF0005EEA430E08BF20EAD37070BD94F0000F25
:106F00000FD101F00046400041EB010111F4801F58
:106F100008BF013CF7D041EA060195F0000F18BF09
:106F2000704703F00046520043EB030313F4801F45
:106F300008BF013DF7D043EA0603704794EA0C0FFF
:106F40000CEA135518BF95EA0C0F0CD050EA410615
:106F500018BF52EA4306D1D181EA030101F0004192
:106F60004FF0000070BD50EA410606BF10461946BA
:106F700052EA430619D094EA0C0F02D150EA0136C6
:106F800013D195EA0C0F05D152EA03361CBF104607
:106F900019460AD181EA030101F0004141F0FE41A6
:106FA00041F470014FF0000070BD41F0FE4141F42A
:106FB000780170BD70B54FF0FF0C4CF4E06C1CEA2A
:106FC00011541DBF1CEA135594EA0C0F95EA0C0FDF
:106FD00000F0A7F8A4EB050481EA030E52EA03359A
:106FE0004FEA013100F088804FEA03334FF08055BB
:106FF00045EA131343EA12634FEA022245EA1115E8
:1070000045EA10654FEA00260EF000419D4208BF98
:10701000964244F1FD0404F5407402D25B084FEA45
:107020003202B61A65EB03055B084FEA32024FF4F1
:1070300080104FF4002CB6EB020E75EB030E22BF4E
:10704000B61A754640EA0C005B084FEA3202B6EB0E
:10705000020E75EB030E22BFB61A754640EA5C00BD
:107060005B084FEA3202B6EB020E75EB030E22BF4D
:10707000B61A754640EA9C005B084FEA3202B6EB4E
:10708000020E75EB030E22BFB61A754640EADC000D
:1070900055EA060E18D04FEA051545EA16754FEA6F
:1070A00006164FEAC30343EA52734FEAC2025FEA8D
:1070B0001C1CC0D111F4801F0BD141EA00014FF01C
:1070C00000004FF0004CB6E711F4801F04BF0143ED
:1070D0000020B4F1FD0C88BFBCF5E06F3FF6AFAE09
:1070E000B5EB030C04BFB6EB020C5FEA500C50F199
:1070F000000041EB045170BD0EF0004E4EEA11311C
:1071000014EB5C04C2BFD4EB0C0541EA045170BD22
:1071100041F480114FF0000E013C90E645EA060E66
:107120008DE60CEA135594EA0C0F08BF95EA0C0F94
:107130003FF43BAF94EA0C0F0AD150EA01347FF4DC
:1071400034AF95EA0C0F7FF425AF104619462CE7B3
:1071500095EA0C0F06D152EA03353FF4FDAE104616
:10716000194622E750EA410618BF52EA43067FF467
:10717000C5AE50EA41047FF40DAF52EA43057FF4F7
:10718000EBAE12E74FF0FF3C06E000BF4FF0010C02
:1071900002E000BF4FF0010C4DF804CD4FEA410C66
:1071A0007FEA6C5C4FEA430C18BF7FEA6C5C1BD033
:1071B00001B050EA410C0CBF52EA430C91EA030FB4
:1071C00002BF90EA020F0020704710F1000F91EA11
:1071D000030F58BF994208BF90422CBFD8176FEADF
:1071E000E37040F0010070474FEA410C7FEA6C5CAD
:1071F00002D150EA013C07D14FEA430C7FEA6C5CB4
:10720000D6D152EA033CD3D05DF8040B704700BFDF
:107210008446104662468C461946634600E000BF2D
:1072200001B5FFF7B7FF002848BF10F1000F01BDFF
:107230004DF808EDFFF7F4FF0CBF012000205DF8CA
:1072400008FB00BF4DF808EDFFF7EAFF34BF01204F
:1072500000205DF808FB00BF4DF808EDFFF7E0FFE8
:1072600094BF012000205DF808FB00BF4DF808ED39
:10727000FFF7CEFF94BF012000205DF808FB00BFA0
:107280004DF808EDFFF7C4FF34BF012000205DF882
:1072900008FB00BF4FEA410C7FEA6C5C02D150EA68
:1072A000013C0AD14FEA430C7FEA6C5C02D152EAFE
:1072B000033C02D14FF0000070474FF001007047CF
:1072C0004FEA4102B2F1E04324BFB3F5001CDCF108
:1072D000FE5C0DD901F0004C4FEAC0024CEA507040
:1072E000B2F1004F40EB830008BF20F0010070476F
:1072F00011F0804F21D113F13872BCBF01F0004072
:10730000704741F480114FEA5252C2F11802C2F1A3
:10731000200C10FA0CF320FA02F018BF40F0010024
:107320004FEAC1234FEAD32303FA0CFC40EA0C00D6
:1073300023FA02F34FEA4303CCE77FEA625307D113
:1073400050EA01331EBF4FF0FE4040F4400070474A
:1073500001F0004040F0FE4040F40000704700BFE4
:1073600080F0004002E000BF81F0004142001FBFFA
:107370005FEA410392EA030F7FEA226C7FEA236C03
:107380006AD04FEA1262D2EB1363C1BFD2184140F8
:1073900048404140B8BF5B42192B88BF704710F08E
:1073A000004F40F4000020F07F4018BF404211F031
:1073B000004F41F4000121F07F4118BF494292EA99
:1073C000030F3FD0A2F1010241FA03FC10EB0C00C5
:1073D000C3F1200301FA03F100F0004302D5494252
:1073E00060EB4000B0F5000F13D3B0F1807F06D3FF
:1073F00040084FEA310102F10102FE2A51D2B1F1F7
:10740000004F40EBC25008BF20F0010040EA0300EB
:107410007047490040EB000010F4000FA2F1010298
:10742000EDD1B0FA80FCACF1080CB2EB0C0200FA22
:107430000CF0AABF00EBC25052421843BCBFD04070
:107440001843704792F0000F81F4000106BF80F4EA
:1074500000000132013BB5E74FEA41037FEA226CAD
:1074600018BF7FEA236C21D092EA030F04D092F078
:10747000000F08BF0846704790EA010F1CBF0020AC
:10748000704712F07F4F04D1400028BF40F0004009
:10749000704712F100723CBF00F50000704700F029
:1074A000004343F0FE4040F4000070477FEA226250
:1074B00016BF08467FEA23630146420206BF5FEA21
:1074C000412390EA010F40F4800070474FF0000321
:1074D00004E000BF10F0004348BF40425FEA000CE8
:1074E00008BF704743F0964301464FF000001CE090
:1074F00050EA010208BF70474FF000030AE000BFE6
:1075000050EA010208BF704711F0004302D5404223
:1075100061EB41015FEA010C02BF84460146002095
:1075200043F0B64308BFA3F18053A3F50003BCFAB0
:107530008CF2083AA3EBC25310DB01FA02FC63445D
:1075400000FA02FCC2F12002BCF1004F20FA02F264
:1075500043EB020008BF20F00100704702F1200257
:1075600001FA02FCC2F1200250EA4C0021FA02F2B8
:1075700043EB020008BF20EADC7070474FF0FF0CBD
:107580001CEAD0521EBF1CEAD15392EA0C0F93EAB8
:107590000C0F6FD01A4480EA010C400218BF5FEA5A
:1075A00041211ED04FF0006343EA501043EA5111CD
:1075B000A0FB01310CF00040B1F5000F3EBF4900C7
:1075C00041EAD3715B0040EA010062F17F02FD2ACB
:1075D0001DD8B3F1004F40EBC25008BF20F00100AE
:1075E000704790F0000F0CF0004C08BF49024CEAC5
:1075F000502040EA51207F3AC2BFD2F1FF0340EA57
:10760000C250704740F400004FF00003013A5DDCC7
:1076100012F1190FDCBF00F000407047C2F1000208
:10762000410021FA02F1C2F1200200FA02FC5FEAF5
:10763000310040F1000053EA4C0308BF20EADC703F
:10764000704792F0000F00F0004C02BF400010F4B1
:10765000000F013AF9D040EA0C0093F0000F01F05E
:10766000004C02BF490011F4000F013BF9D041EA80
:107670000C018FE70CEAD15392EA0C0F18BF93EA82
:107680000C0F0AD030F0004C18BF31F0004CD8D1AC
:1076900080EA010000F00040704790F0000F17BF33
:1076A00090F0004F084691F0000F91F0004F14D079
:1076B00092EA0C0F01D142020FD193EA0C0F03D1D1
:1076C0004B0218BF084608D180EA010000F00040D4
:1076D00040F0FE4040F40000704740F0FE4040F4AF
:1076E000400070474FF0FF0C1CEAD0521EBF1CEA4E
:1076F000D15392EA0C0F93EA0C0F69D0A2EB03026C
:1077000080EA010C49024FEA402037D04FF0805305
:1077100043EA111143EA10130CF000408B4238BFCA
:107720005B0042F17D024FF4000C8B4224BF5B1AD8
:1077300040EA0C00B3EB510F24BFA3EB510340EA26
:107740005C00B3EB910F24BFA3EB910340EA9C00D4
:10775000B3EBD10F24BFA3EBD10340EADC001B0144
:1077600018BF5FEA1C1CE0D1FD2A3FF650AF8B42E8
:1077700040EBC25008BF20F0010070470CF0004CF5
:107780004CEA50207F32C2BFD2F1FF0340EAC25020
:10779000704740F400004FF00003013A37E792F0E1
:1077A000000F00F0004C02BF400010F4000F013A3F
:1077B000F9D040EA0C0093F0000F01F0004C02BF3A
:1077C000490011F4000F013BF9D041EA0C0195E7A3
:1077D0000CEAD15392EA0C0F08D142027FF47DAF3C
:1077E00093EA0C0F7FF470AF084676E793EA0C0F2C
:1077F00004D14B023FF44CAF08466EE730F0004C2A
:1078000018BF31F0004CCAD130F000427FF45CAFB9
:1078100031F000437FF43CAF5FE700BF4FF0FF3C27
:1078200006E000BF4FF0010C02E000BF4FF0010C7A
:107830004DF804CD4FEA40024FEA41037FEA226C43
:1078400018BF7FEA236C11D001B052EA530C18BF65
:1078500090EA010F58BFB2EB030088BFC81738BFCA
:107860006FEAE17018BF40F0010070477FEA226CB8
:1078700002D15FEA402C05D17FEA236CE4D15FEAB4
:10788000412CE1D05DF8040B704700BF84460846E8
:107890006146FFE70FB5FFF7C9FF002848BF10F1A9
:1078A000000F0FBD4DF808EDFFF7F4FF0CBF0120EE
:1078B00000205DF808FB00BF4DF808EDFFF7EAFF78
:1078C00034BF012000205DF808FB00BF4DF808ED33
:1078D000FFF7E0FF94BF012000205DF808FB00BF28
:1078E0004DF808EDFFF7D2FF94BF012000205DF8AE
:1078F00008FB00BF4DF808EDFFF7C8FF34BF0120BB
:1079000000205DF808FB00BF4FEA4002B2F1FE4FD5
:107910000FD34FF09E03B3EB12620DD94FEA002351
:1079200043F0004310F0004F23FA02F018BF40422A
:1079300070474FF00000704712F1610F01D1420211
:1079400005D110F0004008BF6FF0004070474FF0C5
:10795000000070477BB972B90029BEBF00204FF00C
:10796000004106E008BF00281CBF6FF000414FF047
:10797000FF3000F0FFB9ADF1080C6DE904CE00292D
:1079800009DB002B1ADB00F087F8DDF804E0DDE905
:10799000022304B07047404261EB4101002B1BDB26
:1079A00000F07AF8DDF804E0DDE9022304B040429B
:1079B00061EB4101524263EB43037047524263EB78
:1079C000430300F069F8DDF804E0DDE9022304B0C8
:1079D000404261EB41017047524263EB430300F0C8
:1079E0005BF8DDF804E0DDE9022304B0524263EB0A
:1079F0004303704753B94AB9002908BF00281CBF88
:107A00004FF0FF314FF0FF3000F0B4B9ADF1080C8A
:107A10006DE904CE00F040F8DDF804E0DDE9022372
:107A200004B0704710B500210446FFF745FF20B9A8
:107A30002046BDE8104000F009B804F1004000F015
:107A400005F8404261EB410110BD00BFD0B5FFF722
:107A500033F900220E4B06460F46FFF781F900F07E
:107A60008BF90446FFF706F900220A4BFFF778F975
:107A700002460B4630463946FEF7BEFF00F07CF961
:107A80002346002242EA000210461946D0BD00BF3C
:107A90000000F03D0000F0412DE9F0478C460D4616
:107AA0000446089E002B51D18A4217466DD9B2FA7E
:107AB00082FEBEF1000F0BD0CEF1200C01FA0EF5C4
:107AC00020FA0CFC02FA0EF74CEA050C00FA0EF450
:107AD0004FEA174A250CBCFBFAF81FFA87F90AFB94
:107AE00018CC45EA0C4508FB09F3AB420AD9ED195D
:107AF00008F1FF3280F02381AB4240F22081A8F1EF
:107B000002083D44ED1AA4B2B5FBFAF00AFB105589
:107B100044EA054400FB09F9A14509D9E41900F13B
:107B2000FF3380F00A81A14540F2078102383C44CE
:107B3000A4EB090440EA08400021002E61D024FA99
:107B40000EF4002334607360BDE8F0878B4207D9E0
:107B5000002E54D0002186E821000846BDE8F087B9
:107B6000B3FA83F1002940F08E80AB4202D3824207
:107B700000F2FA80841A65EB03050120AC46002E62
:107B80003FD086E81010BDE8F08712B90127B7FB97
:107B9000F2F7B7FA87FEBEF1000F34D1EB1B3A0CB7
:107BA0001FFA87FC0121B3FBF2F8250C02FB183306
:107BB00045EA03450CFB08F3AB4207D9ED1908F180
:107BC000FF3002D2AB4200F2D1808046ED1AA3B260
:107BD000B5FBF2F002FB105543EA05440CFB00FC38
:107BE000A44507D9E41900F1FF3302D2A44500F2FD
:107BF000B8801846A4EB0C0440EA08409DE73146E3
:107C00003046BDE8F087CEF1200405FA0EF307FAFE
:107C10000EF720FA04F83A0C25FA04F448EA0308AF
:107C2000B4FBF2F14FEA184502FB11441FFA87FC3E
:107C300045EA044501FB0CF3AB4200FA0EF409D906
:107C4000ED1901F1FF3080F08A80AB4240F287806D
:107C500002393D44EB1A1FFA88F5B3FBF2F002FB40
:107C6000103345EA034500FB0CF3AB4207D9ED198D
:107C700000F1FF386FD2AB426DD902383D44EB1AA8
:107C800040EA01418FE7C1F1200722FA07F88B4053
:107C900005FA01F448EA030320FA07FE4FEA134C01
:107CA000FD404EEA040EB5FBFCF94FEA1E440CFB06
:107CB00019551FFA83F844EA054509FB08F4AC425C
:107CC00002FA01F200FA01FA08D9ED1809F1FF30C1
:107CD00043D2AC4241D9A9F102091D442D1B1FFA20
:107CE0008EFEB5FBFCF00CFB10554EEA054400FB84
:107CF00008F8A04507D9E41800F1FF3529D2A045BE
:107D000027D902381C4440EA0940A4EB0804A0FB30
:107D100002894C45C6464D4615D312D056B1BAEB32
:107D20000E0364EB050404FA07F7CB401F43CC4075
:107D3000376074600021BDE8F0871846F8E6904689
:107D4000E0E6C245EAD2B8EB020E69EB0305013862
:107D5000E4E72846D7E7404691E78146BEE701467B
:107D600078E702383C4445E7084608E7A8F10208EE
:107D70003D442BE7704700BF4A0011D212F50012B4
:107D800011D20DD56FF47873B3EB62520ED44FEA73
:107D9000C12343F0004343EA505323FA02F07047F3
:107DA0004FF00000704750EA013002D14FF0FF3031
:107DB00070474FF00000704738B5F1F7C7FD62B665
:107DC000F0F748FDF0F764FDF0F7C8FD344C0546C8
:107DD000F1F7BEFDF1F76CF932492A462046F2F779
:107DE000A1FAF1F7B9F92078F1F744FB2079F1F71E
:107DF0008BFBF0F781FEF1F7E3F82B4B01221A70B1
:107E0000F1F73CF9F1F7B8FD0446F1F7B5FD031BB6
:107E1000002BB8BF5B42B3F5FA7FF6DBF1F736F91A
:107E2000F1F7AAFD0446F1F7A7FD031B002BB8BF2D
:107E30005B42B3F5FA6FF6DBF4F7B4FFF6F77CF8C4
:107E400040F21670F3F7DAF80125FBF7F3FD002492
:107E5000FBF726FE0DE0BDB1FBF728FE0446E4B2B9
:107E6000F7F700FC052C13D00024F1F785FDF7F798
:107E70002FFFF7F759FF0120F5F7ACFCF6F702FBEF
:107E8000092CE8DC0134F0E7FBF764FE2C46ECE754
:107E90000025F9F729FB2C46FBF71CFEE5E700BFA0
:107EA0005438FF1FD037FF1F5038FF1F10B5431E37
:107EB0000A44914200D110BD11F8014B03F8014F63
:107EC000F7E702440346934200D1704703F8011BD1
:107ED000F9E700002DE970438AB004460D4600F032
:107EE00077F8354B93F90060731C804689460DD0B6
:107EF00022462B4620462946FFF7CCF930B900220E
:107F0000002320462946FFF7BBF920B140464946E9
:107F10000AB0BDE87083294B0890CDE90245CDE950
:107F20000445019320462946CEB9254D4FF06044C3
:107F300000220023CDE90645FFF77AF9002833D067
:107F400002230093684600F037FAA8B1089BC3B932
:107F5000DDE90689404649460AB0BDE87083194DFF
:107F6000002400220023CDE90645FFF761F968B13E
:107F700002239E420093E5D100F026FA22230360FB
:107F8000E4E700F021FA089B0360E1E70123022EF9
:107F900000930BD100F018FA212303600A4800F087
:107FA0000DFACDE90601D1E701230093684600F000
:107FB00003FA0028F2D1EDE72421FF1F50A20100AF
:107FC000FFFFEFC70000F0FF488F01000000000036
:107FD0002DE9F04FB1F5801F85B006460F460B46E0
:107FE0005ADA024621F00044224300F0F8800029CA
:107FF000C0F27A810022D64BFEF7B2FED54A0B467C
:10800000934206460F466FF0350C4ADCC3F3130566
:1080100005F5152E0EF6647E0EF4801E8EF07F524E
:1080200082F440121C1542EA0507A4F2FF346444AE
:108030000022C94B3046394604EB1E54FEF7DCFCE7
:10804000AB1CC3F31303022B82468B464FF0000296
:1080500030DC0023FFF7ECF8002800F0C980002C8A
:1080600000F04B812046FEF715FEA5A3D3E90023BF
:1080700006460F46FEF774FEA3A3D3E90023044689
:108080000D4630463946FEF76BFE02460B4620464B
:108090002946FEF7B3FC0AE0AE4A93424FF0000CCB
:1080A000B4DD32463B4630463946FEF7A7FC05B004
:1080B000BDE8F08F4FF08043FEF7A0FC02460B4670
:1080C00050465946FEF776FF064620460F46FEF715
:1080D000E1FD3246CDE900013B4630463946CDE967
:1080E0000267FEF73DFE02460B4680468946FEF7D4
:1080F00037FE87A3D3E9002306460F46FEF730FE7E
:1081000085A3D3E90023FEF779FC32463B46FEF710
:1081100027FE83A3D3E90023FEF770FC32463B46DB
:10812000FEF71EFE80A3D3E90023FEF767FC42465C
:108130004B46FEF715FE7EA3D3E900238046894611
:1081400030463946FEF70CFE7BA3D3E90023FEF749
:1081500055FC32463B46FEF703FE79A3D3E90023E4
:10816000FEF74CFC32463B46FEF7FAFD0B46024654
:1081700049464046FEF742FCA5F5C223C5F5D72582
:10818000A3F27A4351351D43002D8046894656DDC2
:108190000022724B50465946FEF7E2FD52465B46BE
:1081A000FEF7DEFD06460F46002C68D132463B4600
:1081B00040464946FEF722FCDDE90223FEF7D0FDEA
:1081C00002460B4630463946FEF716FC02460B4681
:1081D00050465946FEF710FC05B0BDE8F08F00226E
:1081E000002300205E49FEF7E5FE05B0BDE8F08FF4
:1081F00055A3D3E9002350465946FEF7B1FD024688
:108200000B4600205549FEF7F7FB524606460F463F
:108210005B4650465946FEF7A3FD02460B463046E4
:108220003946FEF79DFD06460F46002C40F09A8029
:1082300002460B4650465946FEF7DEFB37E7002C58
:1082400000F0A4802EA3D3E90023DDE90001FEF7AE
:1082500087FD42464B4604460D4650465946FEF7BA
:10826000CBFBDDE90223FEF77BFD27A3D3E9002347
:1082700006460F46DDE90001FEF772FD21E020A36E
:10828000D3E90023DDE90001FEF76AFD32463B46F3
:1082900004460D4640464946FEF7B0FBDDE90223A1
:1082A000FEF75EFD18A3D3E9002380468946DDE989
:1082B0000001FEF755FD02460B4640464946FEF7D3
:1082C0009DFB02460B4630463946FEF795FB52466B
:1082D0005B46FEF791FB02460B4620462946FEF719
:1082E0008BFB05B0BDE8F08F02460B46FEF784FB22
:1082F00000220023FEF75EFED9E600200021D6E62C
:108300000000E0FE422EE63F763C7935EF39EA3D4B
:1083100044523EDF12F1C23FDE03CB966446C73FB4
:10832000599322942449D23F935555555555E53FCD
:108330009FC678D0099AC33FAF788E1DC571CC3FD8
:1083400004FA97999999D93F555555555555D53FA3
:1083500000005043FFFFEF7F0000F03F0000E03FD0
:10836000000050C32046FEF795FC0FA3D3E900237D
:1083700080468946FEF7F4FC0DA3D3E900230446AA
:108380000D4640464946FEF7EBFC9AE702460B468F
:1083900050465946FEF730FBDDE90223FEF7E0FCCC
:1083A00014E700BFAFF300800000E0FE422EE63F7E
:1083B000763C7935EF39EA3D0020704700200149CD
:1083C000704700BF0000F87F014B1868704700BF7E
:1083D000C020FF1F8025000040380000004B000037
:1083E000807000000096000000E10000002C0100F9
:1083F00000C201005515AC6A004001C0ABEA5795B8
:108400000010161B2023272A2D30323537393B3DEB
:108410004041434547494B4C4E5051535456575990
:108420005A5B5D5E60616263656667686A6B6C6D0E
:108430006E707172737475767778797A7B7C7D7ED5
:1084400080808182838485868788898A8B8C8D8EC3
:108450008F9090919293949596969798999A9B9BCA
:108460009C9D9E9FA0A0A1A2A3A3A4A5A6A7A7A8E8
:10847000A9AAAAABACADADAEAFB0B0B1B2B2B3B415
:10848000B5B5B6B7B7B8B9B9BABBBBBCBDBDBEBF51
:10849000C0C0C1C1C2C3C3C4C5C5C6C7C7C8C9C996
:1084A000CACBCBCCCCCDCECECFD0D0D1D1D2D3D3E2
:1084B000D4D4D5D6D6D7D7D8D9D9DADADBDBDCDD38
:1084C000DDDEDEDFE0E0E1E1E2E2E3E3E4E5E5E694
:1084D000E6E7E7E8E8E9EAEAEBEBECECEDEDEEEEF7
:1084E000EFF0F0F1F1F2F2F3F3F4F4F5F5F6F6F75C
:1084F000F7F8F8F9F9FAFAFBFBFCFCFDFDFEFEFFCC
:108500006B7FD87EB87DA07C8F7B857A82798578D9
:108510000878147726763D7559747B73A17236728C
:1085200064719670CC6F076F456EE66D2A6D726C44
:10853000BE6B0D6B5F6AB5696169BB681968796765
:10854000DC664266AB656065CC643B64AD6320630A
:1085500096620F62CB614761C4604460C65F495F49
:10856000CE5E925E1A5EA45D2F5DBD5C4B5CDC5BF3
:10857000A55B385BCC5A625AF95992592C59F95873
:1085800095583358D15771571257B4560000C90047
:1085900092015B022403ED03B6047F054806110730
:1085A000D907A2086A09330AFB0AC40B8C0C540DC4
:1085B0001C0EE30EAB0F72103A110112C8128F138A
:1085C00055141C15E215A8166E173318F918BE19A4
:1085D000821A471B0B1CCF1C931D571E1A1FDD1F31
:1085E0009F2061212322E522A62367242825E82550
:1085F000A82667272628E528A329612A1F2BDC2B1C
:10860000992C552D112ECC2E872F4130FB30B531B2
:108610006E322633DF3396344D350436BA366F3733
:108620002438D9388C39403AF23AA53B563C073DBC
:10863000B83D683E173FC53F73402141CE417A4265
:108640002543D0437A442445CD4575461C47C3474E
:1086500069480F49B449584AFB4A9D4B3F4CE04C8E
:10866000814D204EBF4E5D4FFB4F97503351CE5141
:10867000685202539B533254C9546055F5558A567B
:108680001D57B0574258D3586459F359825A0F5B5B
:108690009C5B285CB35C3E5DC75D4F5ED75E5D5FF3
:1086A000E35F6860EB606E61F0617162F16270635C
:1086B000EE636C64E8646365DD655666CF664667A5
:1086C000BC673268A66819698B69FD696D6ADC6AE6
:1086D0004A6BB76B236C8E6CF86C616DC96D306E34
:1086E000966EFB6E5E6FC16F22708370E270407198
:1086F0009D71F9715472AE7207735E73B5730A742B
:108700005F74B27404755575A575F37541768D76F1
:10871000D87622776B77B377FA773F788478C77803
:1087200009794A798979C879057A417A7C7AB67A61
:10873000EE7A267B5C7B917BC57BF87B297C597C20
:10874000887CB67CE37C0E7D397D627D897DB07D41
:10875000D57DFA7D1D7E3E7E5F7E7E7E9C7EB97ECF
:10876000D57EEF7E097F217F377F4D7F617F747FCC
:10877000867F977FA67FB47FC17FCD7FD87FE17F43
:10878000E97FF07FF57FF97FFD7FFE7F488F010055
:108790004C8F0100588F0100688F0100848F010009
:1087A000A48F0100C48F0100D88F0100E48F010065
:1087B000F48F010004900100149001002890010042
:1087C0003890010048900100589001006890010025
:1087D0001490010028900100389001004890010099
:1087E0005890010068900100789001008890010085
:1087F00098900100A890010014900100B890010029
:10880000DC900100009101002491010048910100D9
:108810006C91010088910100B0910100CC910100A0
:10882000F091010018920100649201003092010061
:108830003C9201005C920100709201008492010060
:10884000989201008C920100A8920100B892010058
:10885000C8920100E0920100F89201000C9301001F
:10886000249301003C93010058930100749301008C
:10887000F091010018920100649201003092010011
:108880003C9201005C9201007092010098920100FC
:108890008C920100A8920100B8920100C8920100D8
:1088A000E092010074930100809301009493010011
:1088B000AC930100BC930100D0930100E093010050
:1088C000D0930100EC930100F8930100049401009F
:1088D000D093010014940100289401002494010015
:1088E0003894010044940100509401006094010008
:1088F0007494010084940100D093010098940100C5
:10890000AC940100A8940100BC94010038940100CB
:1089100044940100D0940100E4940100D09301003C
:10892000FC940100109501000C95010038940100A1
:1089300020950100349501004C95010064950100DB
:1089400078950100D09301008C9501009895010065
:10895000D09301008C950100A8950100B495010009
:10896000D09301008C950100C4950100D8950100B9
:10897000E0950100EC950100F895010004960100D6
:10898000D09301001496010028960100389601004A
:10899000D093010044960100609601006C9601009E
:1089A0007496010088960100A0960100B49601001B
:1089B000C4960100DC96010014900100E8960100C5
:1089C000F0960100F8960100009701000897010059
:1089D00010970100149001001897010024970100DE
:1089E0003897010044970100509701005C970100FF
:1089F0006897010074970100809701009897010023
:108A0000B0970100D0970100E497010000980100A1
:108A100014980100309801004898010068980100FE
:108A20007898010090980100A0980100B898010082
:108A3000D0980100E8980100F89801000899010019
:108A40001499010028990100389901004899010002
:108A500054990100709901008C990100A8990100B6
:108A6000C0990100DC990100EC990100049A010011
:108A70001C9A0100349A010054990100449A0100A3
:108A8000589A01006C9A0100809A0100909A0100A6
:108A9000A09A0100B4960100B89A0100C89A01009A
:108AA000E09A0100488F01004C8F0100588F0100AF
:108AB000688F0100848F0100A48F0100F49A0100E7
:108AC000049B0100249B0100489B0100689B01005E
:108AD000889B0100A89B0100C89B0100E89B010046
:108AE000009C0100209C0100389C0100549C010066
:108AF0006C9C01007C9C0100989C0100B89C0100CA
:108B0000D89C0100F09C01000C9D0100289D0100F3
:108B1000449D0100609D0100809D0100949D010025
:108B2000B4960100C4960100DC960100B09D0100DE
:108B3000C09D0100D09D0100E49D0100F89D010051
:108B4000189E0100349E0100589E0100709E010095
:108B5000949E0100B09E0100D49E0100F09E010091
:108B6000189F0100309F0100509F0100689F010085
:108B7000849F0100A09F0100BC9F0100D49F0100C1
:108B8000E89F0100FC9F010018A001002CA001003B
:108B900044A0010058A0010078A0010094A00100A9
:108BA000B8A00100CCA00100E8A0010004A10100D0
:108BB00024A1010038A101004CA1010068A101001D
:108BC00080A1010094A10100B4A10100CCA1010089
:108BD000E4A1010000A2010000000000BC01FF1F91
:108BE000B001FF1FA401FF1F0000000000000000F3
:108BF00000000000D800FF1FDC00FF1FE800FF1F7F
:108C0000EC00FF1FF000FF1F2001FF1F4401FF1FAA
:108C10004801FF1F5401FF1F7401FF1F7801FF1F50
:108C20007C01FF1F8001FF1F2023FF1F1C23FF1F4C
:108C30001823FF1F8C01FF1F0023FF1F6000FF1F71
:108C40006400FF1F7800FF1F9400FF1F9800FF1FA4
:108C50009C00FF1FA000FF1FA400FF1FA800FF1F14
:108C6000B000FF1FB800FF1FC800FF1FD000FF1F8C
:108C7000D400FF1FE000FF1F0001FF1F0201FF1FC4
:108C80002401FF1F2601FF1F3C01FF1F5E01FF1F84
:108C90006001FF1F6401FF1F6E01FF1F7001FF1FB6
:108CA0004400FF1F4600FF1F6800FF1FC400FF1F96
:108CB000E400FF1F4C01FF1F4D01FF1F5A01FF1F62
:108CC0005B01FF1F6201FF1F6301FF1F6C01FF1F9C
:108CD0008401FF1FF400FF1FF800FF1FFC00FF1FAF
:108CE0000401FF1F0801FF1F0C01FF1F1001FF1FE0
:108CF0001401FF1F1801FF1F1C01FF1F2801FF1F88
:108D00002C01FF1F3001FF1F3401FF1F3801FF1F1F
:108D10004001FF1F6801FF1F8801FF1F5400FF1F54
:108D20005800FF1F5C00FF1F6C00FF1F7000FF1F3B
:108D30007400FF1F7C00FF1F8000FF1F8400FF1FC7
:108D40008800FF1F8C00FF1FBC00FF1FC000FF1F1B
:108D5000CC00FF1FE200FF1F5001FF1F5801FF1F43
:108D60005C01FF1F4800FF1F4A00FF1F4C00FF1F50
:108D70004E00FF1F5000FF1F6A00FF1F5200FF1F21
:108D80005300FF1FAC00FF1F488F0100488F0100F8
:108D90001CA2010028A20100000000000001000048
:108DA0000000704192017AFFFFFFFFFF000000000A
:108DB00000000000A0000000250200008602000064
:108DC0008C0C000000000100905F0100A0860100F3
:108DD000400D030092010400FFFFFF01FFFFFF0FA2
:108DE00020000D201000406010004160080060600D
:108DF00008006160200062602000646020006B60F9
:108E000020006C602000716020007460200077609A
:108E100020007A602000FF600000000002000300D4
:108E2000070022003200F4010016FF17001AFF1B92
:108E3000FF7FFFFFFF00000102030405060708098A
:108E40002040FEFF00000080C0F2FCFF70A0FEFF8B
:108E50000000000000000000905F0100400D0300D2
:108E6000FFFFFF7F0080FFFF000000000100020005
:108E700004000800FF7F00008000000A24000000BA
:108E800003010000100007060C01000000000305AC
:108E900016010000000004050001000001000405A7
:108EA00008010000000001060401000001000106A5
:108EB0000501000002000106010100000000020699
:108EC00009010000410004060A0100000300010638
:108ED0000F010000420004060601000043000406E2
:108EE0001001000000000606110100001000070636
:108EF00002010000110009061201000030000906FD
:108F00000E010000310009060D01000032000906C3
:108F10000B01000000000008130100002000000801
:108F200014010000210000081501000022000008C3
:108F3000070100004700040656312E3100000000F2
:108F400043313630563430300000000044657669D5
:108F500063652054797065004572726F72205265A6
:108F600067697374657200004D616E756661637444
:108F70007572657220446576696365204E616D6522
:108F8000000000004D616E756661637475726572F4
:108F90002048617264776172652056657273696FEB
:108FA0006E0000004D616E75666163747572657266
:108FB00020536F6674776172652056657273696FAE
:108FC0006E0000006E756D626572206F6620656EC2
:108FD000747269657300000056656E646F72204993
:108FE0006400000050726F6475637420436F6465A1
:108FF000000000005265766973696F6E206E756DB2
:109000006265720053657269616C206E756D626590
:10901000720000004E756D626572206F6620456EAD
:1090200074726965730000004D617070696E67202D
:10903000456E7472792031004D617070696E6720E1
:10904000456E7472792032004D617070696E6720D0
:10905000456E7472792033004D617070696E6720BF
:10906000456E7472792034004D617070696E6720AE
:10907000456E7472792035004D617070696E67209D
:10908000456E7472792036004D617070696E67208C
:10909000456E7472792037004D617070696E67207B
:1090A000456E7472792038004D617070696E67206A
:1090B000456E747279203900436F6D6D756E69630A
:1090C0006174696F6E20547970652053796E6320E6
:1090D0004D616E616765722031000000436F6D6DF8
:1090E000756E69636174696F6E2054797065205381
:1090F000796E63204D616E616765722032000000F9
:10910000436F6D6D756E69636174696F6E2054791C
:1091100070652053796E63204D616E6167657220C2
:1091200033000000436F6D6D756E69636174696F24
:109130006E20547970652053796E63204D616E61A5
:109140006765722034000000436F6D6D756E696352
:109150006174696F6E20547970652053796E632055
:109160004D616E6167657220350000004E756D625D
:109170006572206F662061737369676E6564205243
:109180007850444F0000000050444F204D617070F3
:10919000696E6720696E646578206F6620617373FD
:1091A00069676E656420527850444F730000000078
:1091B0004E756D626572206F662061737369676EAC
:1091C000656420547850444F7300000050444F2091
:1091D0004D617070696E6720696E646578206F6696
:1091E0002061737369676E656420547850444F0042
:1091F0004E756D626572206F662053796E6368727A
:109200006F6E697A6174696F6E20506172616D650D
:10921000746572730000000053796E6368726F6E3C
:1092200069736174696F6E20547970650000000085
:1092300053686966742054696D65000053796E63E4
:1092400068726F6E697A6174696F6E2054797065A7
:109250007320537570706F72746564004D696E6928
:109260006D756D204379636C652054696D650000F0
:1092700043616C6320616E6420436F707920546990
:109280006D6500004D696E696D756D2044656C619A
:10929000792054696D650000476574204379636CDB
:1092A000652054696D65000053796E633020437901
:1092B0006C652054696D6500534D2D4576656E745F
:1092C000204D6973736564004379636C652054694C
:1092D0006D6520546F6F20536D616C6C0000000051
:1092E00053686966742054696D6520546F6F20530C
:1092F000686F727400000000527850444F20546F21
:1093000067676C65204661696C6564004D696E69CC
:109310006D756D204379636C652044697374616E6B
:10932000636500004D6178696D756D204379636CEC
:10933000652044697374616E636500004D696E69F0
:109340006D756D20534D2053796E6320446973749D
:10935000616E6365000000004D6178696D756D2078
:10936000534D2053796E632044697374616E636555
:109370000000000053796E63204572726F72000026
:1093800053776974636820506172616D65746572AA
:109390007300000053746174757320616E6420451E
:1093A00072726F7220466C61677300005375707043
:1093B0006C7920566F6C7461676500004472697641
:1093C00065722054656D7065726174757265000018
:1093D0004E756D4F66456E747269657300000000CE
:1093E0004D6F746F72506F6C657300004D617854EF
:1093F0006F727175650000004D617856656C6F6322
:10940000697479004D6178416363656C657261745C
:10941000696F6E0041637475616C43757272656E3D
:109420007400000052616D70546172676574437519
:109430007272656E74000000505F506172616D65FC
:1094400074657200495F506172616D657465720088
:1094500050495F546F727175655F4572726F72002B
:1094600050495F546F727175655F4572726F725FBC
:1094700053756D0050495F466C75785F4572726F29
:109480007200000050495F466C75785F4572726FDC
:10949000725F53756D00000041637475616C5665B1
:1094A0006C6F63697479000052616D70546172670A
:1094B000657456656C6F6369747900004D6F746FE5
:1094C0007248616C74656456656C6F636974790089
:1094D00050495F56656C6F636974795F4572726F4E
:1094E0007200000050495F56656C6F636974795F64
:1094F0004572726F725F53756D0000004163747541
:10950000616C506F736974696F6E000052616D70A9
:10951000546172676574506F736974696F6E00008F
:1095200050495F506F736974696F6E5F4572726FF7
:10953000720000005461726765745265616368650A
:109540006456656C6F6369747900000054617267DA
:1095500065745265616368656444697374616E63C0
:1095600065000000436F6D6D75746174696F6E20E6
:109570004D6F64650000000056656C6F6369747917
:109580002052616D70204D6F6465000041637475F9
:10959000616C416E676C65004F70656E4C6F6F70EB
:1095A00043757272656E7400496E76657273696F89
:1095B0006E000000496E746572706F6C6174696F43
:1095C0006E0000005374657073506572526F746161
:1095D00074696F6E000000004F666673657400006A
:1095E000446972656374696F6E000000496E697446
:1095F0004D6F646500000000496E697444656C61DC
:1096000079000000496E697456656C6F63697479FE
:1096100000000000456E61626C654272616B6543DB
:10962000686F707065720000566F6C746167654C8E
:10963000696D697400000000487973746572657320
:1096400069730000546865726D616C57696E646976
:109650006E6754696D65436F6E7374616E7400005C
:109660004949744C696D697400000000494974539C
:10967000756D0000494974457863656564436F758D
:109680006E74657200000000436C65617249497434
:109690004578636565646564466C61670000000039
:1096A000486F6D65204F66667365742044697370FA
:1096B0006C6179004469676974616C20496E7075EA
:1096C0007473000053746F72652041786973205081
:1096D0006172616D657465720000000048414C2044
:1096E00056657273696F6E00696E666F2031000097
:1096F000696E666F20320000696E666F203300006D
:10970000696E666F20340000696E666F2035000058
:10971000696E666F203600004144435F494E5F30FA
:10972000000000004144435F53494E474C455F539E
:1097300048554E54000000004144435F7068617317
:10974000655F41004144435F70686173655F42003B
:109750004144435F56537570706C79004144435FD8
:1097600054656D7000000000436F6E74726F6C770B
:109770006F726400537461747573776F7264000064
:10978000517569636B2053746F70204F7074696FEB
:109790006E20436F6465000053687574646F776E64
:1097A000204F7074696F6E20436F64650000000085
:1097B00044697361626C65204F7065726174696F92
:1097C0006E204F7074696F6E20436F6465000000F7
:1097D00048616C74204F7074696F6E20436F6465CC
:1097E000000000004661756C742052656163746905
:1097F0006F6E204F7074696F6E20436F6465000058
:109800004D6F646573206F66204F70657261746977
:109810006F6E00004D6F646573206F66204F70653A
:10982000726174696F6E20446973706C61790000B5
:10983000506F736974696F6E2044656D616E64204A
:1098400056616C7565000000506F736974696F6EC6
:109850002041637475616C20496E7465726E616C31
:109860002056616C75650000506F736974696F6E86
:109870002041637475616C00466F6C6C6F77696E24
:1098800067204572726F722057696E646F770000AF
:10989000506F736974696F6E2057696E646F7700DB
:1098A000506F736974696F6E2057696E646F7720AB
:1098B00054696D650000000053656E736F7220532C
:1098C000656C656374696F6E20436F6465000000AA
:1098D00056656C6F636974792044656D616E6420B0
:1098E00056616C756500000056656C6F636974792C
:1098F0002041637475616C00546172676574205413
:109900006F727175650000004D617820546F72713F
:1099100075650000546F727175652044656D616EE8
:10992000642056616C756500546F727175652041D5
:10993000637475616C000000546172676574205037
:109940006F736974696F6E00486F6D65204F66664E
:109950007365740048696768657374207375622D58
:10996000696E64657820737570706F7274656400D9
:109970004D696E20536F66747761726520506F7306
:109980006974696F6E204C696D6974004D6178204F
:10999000536F66747761726520506F736974696F75
:1099A0006E204C696D6974004D61782050726F664D
:1099B000696C652056656C6F6369747900000000FE
:1099C00050726F66696C652056656C6F6369747957
:1099D00020696E2070702D6D6F646500456E642087
:1099E00056656C6F636974790000000050726F6691
:1099F000696C6520416363656C65726174696F6E43
:109A00000000000050726F66696C652044656365F4
:109A10006C65726174696F6E000000005175696356
:109A20006B2053746F7020446563656C657261745C
:109A3000696F6E00486F6D696E67204D6574686F61
:109A4000640000004661737420486F6D696E672082
:109A50005370656564203100536C6F7720486F6DDB
:109A6000696E67205370656564000000486F6D691A
:109A70006E6720416363656C65726174696F6E0027
:109A8000506F736974696F6E204F666673657400FA
:109A90004F666673657420746F727175650000009F
:109AA000506F736974696F6E696E67204F70746967
:109AB0006F6E20436F646500546172676574205651
:109AC000656C6F6369747900537570706F7274653B
:109AD00064204472697665204D6F646573000000F0
:109AE00053696E676C6520446576696365205479B7
:109AF000706500004964656E74697479204F626A0C
:109B000065637400526563656976652050444F2033
:109B10004D617070696E6720506172616D6574652A
:109B2000722031005472616E736D69742050444F1D
:109B3000204D617070696E6720506172616D65744F
:109B4000657220310000000053796E63204D616E14
:109B50006167657220436F6D6D756E6963617469CD
:109B60006F6E20547970650053796E63204D616E7D
:109B70006167657220322050444F204173736967DA
:109B80006E6D656E7400000053796E63204D616EDA
:109B90006167657220332050444F204173736967B9
:109BA0006E6D656E7400000053796E63204D616EBA
:109BB0006167657220322053796E6368726F6E69D7
:109BC0007A6174696F6E000053796E63204D616E27
:109BD0006167657220332053796E6368726F6E69B6
:109BE0007A6174696F6E0000417869733020537731
:109BF0006974636820506172616D65746572730089
:109C000041786973302053746174757320616E6498
:109C1000204572726F7220466C616773000000000D
:109C2000417869733020537570706C7920566F6C71
:109C300074616765000000004178697330204472E8
:109C4000697665722054656D7065726174757265B0
:109C5000000000004178697330204D6F746F7220EE
:109C600053657474696E677300000000417869730E
:109C700030204C696D69747300000000417869738D
:109C80003020546F72717565204D6F646520536587
:109C90007474696E6773000041786973302056658B
:109CA0006C6F63697479204D6F64652053657474BB
:109CB000696E677300000000417869733020506F4F
:109CC000736974696F6E204D6F6465205365747499
:109CD000696E677300000000417869733020436F3C
:109CE0006D6D75746174696F6E204D6F64650000F1
:109CF00041786973302056656C6F636974792052BE
:109D0000616D70204D6F64650000000041786973DB
:109D100030204F70656E204C6F6F702053657474E7
:109D2000696E6773000000004178697330204861F4
:109D30006C6C2053656E736F722053657474696E1A
:109D40006773000041786973302041424E20456EB0
:109D5000636F6465722053657474696E6773000085
:109D60004178697330204272616B652043686F707F
:109D70007065722053657474696E6773000000002B
:109D80004178697330204949542053657474696E71
:109D900067730000417869733020486F6D65204F0C
:109DA000666673657420446973706C6179000000A5
:109DB000434C20496E666F726D6174696F6E00006E
:109DC000416E616C6F6720496E707574730000009E
:109DD000417869733020436F6E74726F6C776F7265
:109DE00064000000417869733020537461747573A6
:109DF000776F7264000000004178697330205175FC
:109E000069636B2053746F70204F7074696F6E209C
:109E1000436F646500000000417869733020536827
:109E20007574646F776E204F7074696F6E20436F26
